:100000000100000000000000000400000094511AEC
:100010001CF09FE51CF09FE51CF09FE51CF09FE5A0
:100020001CF09FE51CF09FE51CF09FE51CF09FE590
:1000300024440ECBC8750200A0750200A47502000E
:10004000A8750200AC750200B0750200B47502001C
:10005000C1750200000000EAEC8500EA28008FE28A
:10006000000C90E800A08AE000B08BE001704AE24A
:100070000B005AE1E585000A0F00BAE814E04FE2F0
:10008000010013E303F0471013FF2FE1387C020057
:10009000787C02000030A0E30040A0E30050A0E321
:1000A0000060A0E3102052E27800A128FCFFFF8A44
:1000B000822EB0E13000A128003081451EFF2FE1E3
:1000C00004309FE503308FE013FF2FE1851A020013
:1000D0000020704710B5144C206800280CD100F0A7
:1000E00027FD2060114A2021A0600BF3A4F9104ADB
:1000F000606820210BF39FF910BD10B50A4C2068F1
:10010000002808D0002213210BF395F920680BF387
:1001100076F90020206010BD0200034810B5006889
:1001200068210BF388F910BDB0F500C0851B0200F3
:10013000A31B020010B527F094EA05F33FFF00204F
:1001400010BDB64810B5006800022FD5B44CB54AB2
:100150000020C11C09016161236981005350031D06
:100160001B01636123698918801C0C284B60F0DB3C
:10017000AD48FFF7D1FF27F0D8EAFF21AB4A2D3178
:1001800002E0401C8842FCDB50780028F9D0A848E7
:100190006061A8482061012040036061A648206199
:1001A000A348E03860610520206105E09E48401CBE
:1001B000FFF7B2FF27F0B8EA012010BD9B4910B548
:1001C000486000F03DFF10BD202800D3FEE79B4AA9
:1001D00080001358002B00D0FEE71150002070471C
:1001E000964A002180001150080070470268836819
:1001F000C1681000184770B5052804D2904D8400DE
:100200002B59002B01D0012070BD2C238C4E434371
:10021000DC3E9B192B5135000401F0352851601943
:10022000C2608160002141608649196158610020E7
:1002300070BDFEB50E001700052815D280490201D9
:100240001431551869687E4B840000290DD10122B4
:1002500001970096029218594369026907F390FAD0
:10026000002801D101206860FEBD18591D0007F368
:10027000C3FA28593A00310007F370FA285907F3F6
:100280005DFAFEBD694970B50878401C0006000E95
:100290000870012149044018FFF73EFF6A4D6C6A5F
:1002A000E00705D003F388EF0BF318F9A81768628D
:1002B000664EA0070CD5A86A02218843A8622020B8
:1002C000F060491F6962B1680143B1600BF3FEF849
:1002D000600705D5A86A04218843A8620BF31FFCB8
:1002E00020070AD5A86A08218843A8628020F06008
:1002F000C9436962B1680143B160012070BD70B546
:100300000124524D8440EC60002022F037FCA868A4
:100310002043A860012070BD01214C4A814010B5E6
:10032000D1600F3800D5FEE7022800DBFEE7484C1D
:100330000023800004192360454C403400190362F7
:10034000906808439060012010BDF8B5414DEC68FD
:10035000E00702D0A817E8600440200606D58020F8
:10036000C043E8608020844300F03DFD200407D5B1
:100370000126F603300000F036FDF043E860B44398
:100380006003400F06D00720000421000140C9434C
:10039000E96084432002000F09D00F273F052600A3
:1003A0003E40300000F0D4FCF043E860BC43E00085
:1003B000400F09D00727BF0626003E40300000F05E
:1003C0005FFCF043E860BC43E0060FD51020C0435B
:1003D000E8601020844322F0C1FA002806D004F01F
:1003E000EDFE002802D0102000F0ACFB002C05DA56
:1003F0000120C00700F05FFC1748E86013498868D7
:100400000122920510438860F8BD104B3AF3F46462
:1004100001000000FC030000000400005AEF5E131E
:100420000122920510B5DA60FFF799FF012010BD97
:100430000031008080290080006102C0400001007E
:10044000F47C0200F0200000FF0C0000070080FF99
:10045000D0430004D87E0200DD010000003400809B
:100460000030008040E8008080220080FFFFFF7F96
:1004700030B504002020208165692018AD7A057010
:100480006469E47A44700171090A4171110A827148
:10049000C171190A8370C17030BDF7B50700487883
:1004A0000E00097805020D43203528003430010480
:1004B000090C0022FF481DF36BF8040021D028002E
:1004C0001430A08067612027E019142127811CF3D4
:1004D0009EEB2B04029A1B0C14212000FFF7C8FF8F
:1004E0003420208120182A0031001CF3CAEA0021A0
:1004F000200021F0F2FB207B202804D1200021F0F5
:10050000DDFB0020FEBD278124F0E5F8002802D0A5
:1005100005200AF0B4F921F095FBE84B0500E64808
:1005200021001C68002200680523A047280021F054
:100530008DFB0120FEBDFFB50120904083B0039FDD
:100540000406240EFF374137F8790E0015002042CB
:100550002FD1FF229132462301A902A805F0E9F824
:10056000002826D0F87917212043F871019C103417
:1005700020001CF34CEB0698002801D1052000E078
:100580000D20607225722000627A0C990A301CF3EB
:1005900078EA310006220C31A01C1CF372EA607A62
:1005A00001990A308872000AC8720299039805F00E
:1005B0008BF807B0F0BDFFB59FB0060008003768A4
:1005C0000021179121997C69002910D040301E909C
:1005D0001CF398EB229905004118C07820314006A1
:1005E00002D4B88823B0F0BD2888682801D800203C
:1005F000F8E719AA18910092219918981AAA17AB2E
:1006000010F308F9280010F32CF9002853D0AC4857
:10061000002104AA01AB07C318ABAA4A00921D79B6
:1006200010AB1A7F38002B001AA90EF34CFB050003
:100630002DD12000FF304130C179090624D5002C8E
:100640000CD00521C90161180968002906D018AB32
:100650001A79920068328B585B1C8B50C17949061D
:10066000490EC1711E981CF34EEB18AB1D792199F0
:100670002A01521B52180E320092010010AB1B7F50
:100680002A002000FFF757FF00203060AFE73560F9
:1006900028891E9940191CF346EB0088A880200089
:1006A000FF30413018AB1B7901263200C1799A40E6
:1006B0009143C1711DE010AB197F009101952A880B
:1006C00018991898643A091D1AAB12F3A8FD060090
:1006D0001CD0200018AB1A79FF3041300123C179BA
:1006E00093409943C171288808382880B888083811
:1006F000B880002C08D00520C00120180068002810
:1007000002D0416E491C416630006BE7002C14D0CA
:100710000520C0012018016800290ED018AB1A79F5
:10072000920068328B585B1C8B5001680A69521C1E
:100730000A610068C168491CC1601E981CF3E2EAA6
:10074000010018AB1879219A03011B1A9A180E326E
:100750000092020010AB1B7F2000FFF7ECFED3E7F6
:1007600000280CD00521C90141180868002806D0CE
:100770000269521C02610868C16C491CC16470475F
:10078000FFB583B004001E000C9F0E9D24F054FDA5
:10079000002820D0607A02281DD0082E1BD3082FF5
:1007A00001D3012005E738001DF378FB030080002A
:1007B00055250019ED00119A109940196D4607C58D
:1007C000580057210019C90043180D9A059904983B
:1007D0000FF374FFEDE60FA807C86C462B0007C4A3
:1007E000F3E7F7B592B014000F00129800680D906F
:1007F00000200A900D9845690800403011901CF3C4
:1008000082EA06002430099028000CF0F9FF21004C
:100810002C311091091D203700280F91F976C9421B
:1008200001000000F80700000004000009358D7F7A
:1008300022D0109807AA08A903AB07C36B46E0793A
:100840000F9A0107387E090F4007400F07C30021A8
:10085000B078099A03092800FFF79CFF00280BD005
:10086000002D08D00520C001281800680028F8D005
:10087000016D491C016595E030886828FBD922008C
:100880004C3268380304111F081F0692021F05919D
:10089000049003920C3938381C3A0291019000926E
:1008A000387E1B0C47077F0F1A00099930003B0068
:1008B00012F3D7FB070030000FF3DDFF002849D00B
:1008C00000200BAA0AA909E078040004B4F500C0CE
:1008D000F0F500C0306102C0782401C0009101929F
:1008E0000A900D9B099A310038000FF3A4FE0028EE
:1008F00058D0934A0092934A934B0D9831001CF3C1
:1009000053FF002802D1129908604BE012990600AB
:1009100008600189081811991CF30EEA0E900A98D4
:1009200000284AD00BAA009209990E9823003200A1
:100930000FF3B0FE070040D1002D08D00520C00104
:1009400028180068002802D00168491C01600E9830
:10095000807922E0002F28D03807800F0FD0002D9B
:1009600020D00520C0012918086800281AD0C26CC0
:10097000521CC26408680169491C016112E0B80791
:1009800010D5002D08D00520C001281800680028C7
:1009900002D00168491C0160B079C107C90F280065
:1009A00026F0DAEE002015B0F0BD30881438308023
:1009B0000D980D99808814388880079C6B461A8C96
:1009C00010990F9823000FF380FE002F0AD1002DFD
:1009D00008D00520C00128180068002802D0416E08
:1009E000491C41660120DEE7F7B582B0140007001C
:1009F0000068009001900398002540301CF38CE9BA
:100A000006000198F1784069490605D42030807EBF
:100A1000400731D401252FE0002C02D1002005B081
:100A2000F0BDA17AC90720D0E0790007000F0128A6
:100A300005D1039922006846FFF7DDFE05E0039922
:100A4000220004236846FFF7C0FD050000983860C7
:100A5000B079C00710D1002D0ED0A07980070BD53A
:100A6000A07AFD210840A07206E00521C9014018C6
:100A700000688168491C81602800D0E7F3B589B01F
:100A800005000A98002814D02C896E69611920226B
:100A900001A81CF300E86B46987901AF0007810FAD
:100AA0000120884029490988084204D1280021F002
:100AB0000FF90BB0F0BD200020216C1820382981DF
:100AC0002071000A6B466071988B00092072000A41
:100AD0006072B07A2070F07A6070A0360E20305EBE
:100AE00023F017FB20730A20305E23F005FB6073B0
:100AF000FF20A0720A9A3B002100280021F0F8F99B
:100B00000520A0710020E071012060742074A88885
:100B1000A070000A22000B32E0700A98D11C1DF36D
:100B200062F821F099F80B4B060009481C68002276
:100B3000290000680523A047300021F091F8B8E7AC
:100B40006C2401C0742401C0306102C02C04000474
:100B5000B4F500C0F0F500C0010002A010B50AF322
:100B600032FC10BD7364696F0000000010B5040012
:100B7000C0200DF076FA00F00AFAE00602D50BF07C
:100B800048F810BD0AF0E9FF10BD0020EEE70000B4
:100B9000052803D259498000085C7047FF20704740
:100BA0000A00032010B5FFF7F3FF904201D1FFF7D1
:100BB000ECFF10BDFF280BD0504A00218B00D35C06
:100BC000834202D10806000E7047491C0529F5D35F
:100BD000FF207047FF280CD0484A00218B009B184B
:100BE0005B78834202D18800105C7047491C05295C
:100BF000F4D3FF207047052804D2404980004018F4
:100C000040787047FF207047FF280CD03B4A0021F6
:100C10008B00D35C834203D18800801840787047F2
:100C2000491C0529F4D3FF207047FF2840C36148C1
:100C300001000000F40B000000040000FD5AF8CB96
:100C40000CD0334A00218B00D35C834203D188004F
:100C5000801880787047491C0529F4D3FF2070471D
:100C60002B4A00218B00D35C834206D18800801878
:100C7000C0784007C017401C7047491C0529F1D3B4
:100C80000020704770B505000C00100000F043F91B
:100C9000200000F0C6F82800FFF7A6FF022805D0C4
:100CA000032803D0042801D0052803D1200000F038
:100CB0006DF870BD20000DF010FA70BD70B5040025
:100CC000144DC00004D52A00A9040C20FFF7DAFF58
:100CD000200105D50122D20211040B20FFF7D2FF1B
:100CE000600105D501212A0089060A20FFF7CAFF05
:100CF00070BD0120C00310B500F00DF90120C00740
:100D000000F08FF80449C86880229043C86010BD85
:100D10007CF800C00004000000280080F3B581B01A
:100D20000F000198FFF750FF05000198FFF776FFCD
:100D300006000198FFF783FF0400032D07D1042E5E
:100D400005D1102000F0E7F8B00400F073F8002F90
:100D500016D10198FFF784FF002811D0231F1CF340
:100D6000C0E8060F0F0F0F07040F0021102005E049
:100D70002649A8004018C0780021C00809F321FEC8
:100D8000FF2201991000FFF715FFFEBD10B504000A
:100D9000C00203D501210220FFF7C0FFA00203D546
:100DA00001210320FFF7BAFF600203D501210420CF
:100DB000FFF7B4FF200203D501210520FFF7AEFFA6
:100DC00001200007844205D04010844202D0401028
:100DD00084421AD1FF208206A11808D0891804D0B5
:100DE000C206891804D10C2002E00B2000E00A2082
:100DF000FFF7FAFE022805D0032803D0042801D00B
:100E0000052802D10121FFF789FF10BD7CF800C041
:100E100013490A6802430A608A6802438A60012013
:100E200070470F490A6882430A608A6882438A6071
:100E3000012070470A49C043C8600120704710B5BF
:100E4000074C8034216962690F23DB0199439A437F
:100E5000002801D01A4300E019432161626110BDEE
:100E60008022008083480068416801225204914337
:100E7000416070477F480068416801225204114375
:100E8000416070477B480068816B0901090C01D003
:100E900000207047816B002904DA816B0906090F75
:100EA000FBD100E0806B01207047724909688A69B4
:100EB000120C120402438A6170476E480068816B0D
:100EC000C907FCD041680122D203914341607047B9
:100ED000684909680A6B086348680122D203104315
:100EE0004860704763480068406A70476149096814
:100EF00080314A6A0001120F1207000902434A6258
:100F000070475C480068C06A70475A490968CA69F6
:100F10008243CA61704757490968CA690243CA6176
:100F20007047544909680A6A02430A627047514986
:100F300009680A6A82430A6270474E480068803036
:100F4000416849084900416070474A48006880305C
:100F50004168012211434160704770B5454D2868D2
:100F6000803001680122114301600168424C49024E
:100F700005D50168A14301600A2026F08AEB2868A4
:100F8000803001682143016070BD3A48006801006B
:100F900080310A68520852000A60816BC900FCD493
:100FA00070473448006880300168334A91430160DB
:100FB0007047304800688030C068704770B52D4D6C
:100FC00029680E690C00012109040E4326612100E5
:100FD00080310E69086148694B618869F020886139
:100FE000C869CA61A06810210843A060A0682022D7
:100FF0009043A0602868416B436B8B42FCD0FFF7A5
:10100000D8FF0028F6D128688168114381604168C3
:10101000012252031143416070BD164800688030C0
:10102000006970471348006881682022114381607D
:10103000704710480068816820229143E3BF075041
:1010400001000000F00F000000040000AE802BA79C
:10105000816070470C49096880310A681F23DB05ED
:10106000C0069A43000902430A6008680122120779
:101070001043086070470448006880300168FF2210
:10108000521C114301607047C4F500C000004000CD
:1010900038B500240C4D01E08047641CA00028589E
:1010A0000028F9D109480B4902680092084A0A4809
:1010B0000A4B07F355FC0AF07AFC0948016800293D
:1010C00001D00020884738BD60B602C0A8F800C033
:1010D000704F00047004000464040004008002C027
:1010E000C8F500C0FEB50D001600089F0A9A0999C0
:1010F000002800D1FEE70468002C00D1FEE7029230
:10110000019132002900200000970EF0DDFCFEBDA9
:1011100010B506F319FA0006000E10BD10B506F35F
:10112000A5F90006000E10BD002810B501D006F389
:10113000D9F910BD38B514006A4606F333F90098A2
:101140002070002038BD10B5040006F385F820603B
:10115000002010BD10B506F355F910BD7CB50D008B
:101160001600079A0699002800D1FEE70468002CB3
:1011700000D1FEE7019200913200290020000EF01C
:1011800081FD002800D165637CBD10B5416B0EF078
:1011900090FD10BD7CB50C001500069A002800D10A
:1011A000FEE70068002800D1FEE7002101920091CF
:1011B0002A0021000EF0B6FC7CBD10B50EF0D1FC6B
:1011C00010BD002810B500D1FEE70068002800D14E
:1011D000FEE70EF03DFD10BD002810D00521C9012D
:1011E0004218116800290AD00B695B1C0B61116859
:1011F000CB685B1CCB6011680A6E521C0A66FF301C
:101200004130C17980221143C1717047704706484F
:10121000142110B51BF3EEEC0448012101700021EC
:101220008160C16010BD0000306102C06C2401C04B
:101230009048416810221143416070477047F1B5F2
:1012400082B0002620F01CFD00908B480021006831
:10125000012806D18848029A00694369934200D167
:10126000416186484468019425001BE0A00087186E
:10127000B868029B4169994206D1761C002120F092
:10128000EFFC0020B86008E0A90089188860002001
:10129000102D019500D0681C05000020102C00D0F6
:1012A000601C0400754A00201168102900D0481CF9
:1012B000A042DBD1002E07D070484168A94201D17D
:1012C000446001E0019901606B484068012807D142
:1012D0006B480299006842698A4201D1002141614C
:1012E00066484C30446801942500002728E02420FB
:1012F0006043029B8618F0684169994208D17F1CBF
:1013000021F0CEFD30000C3024211BF374EC12E0F0
:10131000242169438B18D8603069186131001800A6
:10132000143114301C221BF334EC0020372D0195AE
:1013300000D0681C05000020372C00D0601C040081
:101340004E4A00204C321168372900D0481CA04278
:10135000CDD1002F08D049484C304168A94201D175
:10136000446001E001990160009820F08DFCFEBD11
:10137000F8B50500002420F083FC3F490A68012AE3
:1013800004D109694969A94200D101243B4F0026D3
:101390003B6879680BE08A00D21992685269AA42C8
:1013A00000D101243200102900D04A1C1100002C69
:1013B00005D13200102B00D05A1C8A42EBD120F00C
:1013C00063FC2000F8BD70B50E0004981D00018973
:1013D0000C1820784007400F90420FD1E06D290093
:1013E000FF31801D06224A3120F06EF9002805D118
:1013F000682006552100280021F0ACFD70BDFFB526
:1014000081B01E001C480168012906D1026901A8AB
:10141000009207C83300FFF7D6FF184900270D6870
:101420003800102D00D0681C4C68A04215D00EE08A
:101430001249A0004018826801A8009207C8330032
:10144000FFF7C1FF3800102C00D0601C3A7F30DE5F
:1014500001000000EC1300000004000011450E1410
:1014600004003800102D00D0681CA042EAD105B05D
:10147000F0BD07480021C943002206C04430426045
:10148000016004498160704700A000903C040004A2
:1014900098060004504400040020704710B512F074
:1014A00071F910BD0722010010B5FF48406921F015
:1014B0009DFA002010BDF7B584B000242500FC483B
:1014C0000194FA4E42690499430619430A43426162
:1014D000F74980310A6907231B041A430A61F44B58
:1014E000C0331968082291431960F2490B6893438D
:1014F0000B60806902900AF301F80090EE480F003B
:10150000FEF73CFEE8482AE009F3F8FF009A0023C2
:10151000801AE54AB941D1649064E84A121A8B41B5
:1015200009D2E1488168491C8160E1494869049A0F
:101530009043486116E0DE486D1C80690290E048E7
:1015400000697F214905084003D001214905411A5E
:1015500003D1864201D1641C00E0002406000698F5
:101560008442D1D3D04E0120B1680004002907DDA8
:1015700006998C42F16801D3491C00E00918F1601A
:10158000FEF7FCFD09F3BAFF009A801AB941F16435
:10159000B06402990498884301D001200190C549A4
:1015A0000868082210430860C149C0310868104328
:1015B0000860BF4A8032116907200004814311612D
:1015C00005980560019807B0F0BDF8B50700B64D65
:1015D00009F394FF0E00B8490400F13938000FF305
:1015E00070F909F38BFF041B686CB1410B000021FB
:1015F000001B994100D36C6C6C64F8BDF1B584B0EC
:10160000A94C206B401C206309F378FFA94F0D0003
:10161000403F0290FE6AAB48F862A548406921004D
:101620000190A9481E222431FFF745FF002802D06F
:10163000206C401C2064FE629D488069E06209F3D2
:101640005DFF029AE76B861AA9410D007A1C002003
:10165000A06BE16B002348430021801969411BF313
:1016600016E8A063E06B401CE063606B0021801B08
:10167000A94100D3666B6663606AA16A884201D99A
:10168000606A00E0A06AA062049A01998E48114342
:10169000884301D0FFF799FF226C616B112018F08D
:1016A00049FE05B0F0BD89480088002804D088496B
:1016B00001200978042900D0002070472020F1E69D
:1016C000F8B50024784D6868002801D12000F8BDE5
:1016D00020F0E0FA0090286A01273B00002800D0A3
:1016E00000230020390081402A6A0E00164202D1F0
:1016F0000C000A432A62401C002C01D11F28F1DD96
:10170000002B04D010F3DFFBFF20FFF777FF0098DA
:1017100020F0C4FADAE770B5040020F0BBFA050047
:10172000614800224168002901D1226070BD236810
:10173000016A99430162226007D1FF20FFF745FF4C
:1017400010F3B9FB0120FFF7ADFE280020F0A6FA48
:1017500070BD38B5040041696A4622F0A1FE002838
:1017600002D12000FFF79AFE002802D120001BF3CF
:101770000DFF38BD38B505224B4C0021606921F0C2
:1017800035F9544805220068002121F02FF902E0C4
:1017900000981BF3FBFEA06904220023694621F098
:1017A00021F90F28F4D14C48002505704B4812212F
:1017B0001BF32AEA4A4865700560002038BD6023A3
:1017C0005843484A10B58418A088E288824201D163
:1017D000012010BD8200A21892680A601421401CEA
:1017E0001BF3C6EEA180A06D401EA065002010BDB9
:1017F00070B50C00417A160002290AD105F045FFA8
:10180000012806D130001C3802210AF022F90128F3
:101810000BD06021614333480C18E5881421681C03
:101820001BF3A6EEA088884201D1012070BDA8005C
:1018300020188660E180A06D401CA065002070BD6E
:101840002848602110B51BF3E0E917490020C86162
:1018500010BD001F10B50406240E042CA80A992FF1
:1018600001000000E817000000040000429FDD783E
:1018700013D2602060432049401860211BF3CEE959
:101880000E4A0120D169A04008431021A140014324
:10189000FF20401CA0408143D16110BDF8B5041F5A
:1018A000042C45D220F000FA0600044DFF20401C15
:1018B000E969A04008422BD024E00000D0030004D6
:1018C0004523010040A2008000A70080F000010035
:1018D000A086010080A80080FF7FFF7FFF0300003B
:1018E0001C3E01C0C5F700C0687D02006004000412
:1018F0001C4600045C7D02009C44000400981C38D7
:1019000021F05CFB20006946FFF763FF0028F5D05B
:10191000FF211231E869A1408843E86160206043FB
:101920003949401860211BF37AE9300020F0C0F9F2
:10193000F8BDF8B5041F042C25D220F0B5F9060037
:10194000324DFF20401CE969A04008420BD004E062
:10195000009800211C3820F097F920006946FFF715
:1019600038FF0028F4D0FF211231E869A1408843F4
:10197000E861602060432449401860211BF34EE970
:10198000300020F095F9F8BDF8B5002425001E4E72
:10199000FF277F1C602060431C4935543800C9690B
:1019A000A040084202D00120FFF786FD641C042CF1
:1019B000F0DBF8BDF8B5050020F076F90600144913
:1019C000144825F0F6EEFFF785FE00902800FFF79B
:1019D0004AFC00242006000E290011F07BFB641C49
:1019E000042CF7DB6846FFF7A0FE300020F060F91A
:1019F000F8BD09480088002805D008480178032967
:101A000001D10421017070479C440004D0030004FC
:101A10001111FFFFBBBBBBBB1C3E01C0C5F700C023
:101A2000FF49002048607047FD49002088607047EA
:101A3000F7B582B00600FA4DA86800284AD1FF2108
:101A4000F84800222D311BF3D5FD040042D00120BF
:101A50000221A86021736661617B0143F2486173D2
:101A6000A061AC202081FF205130825BEF480092C2
:101A70000068320003795920C00031187E322000FE
:101A80000EF397FD07001C202518208170212800E7
:101A90001BF3C4E8280060300499019041723000C3
:101AA000EF6511F08AFFE34AA8701279E0499206C7
:101AB00005D4002803D0A8684A071043A8600198FD
:101AC00003220272200011F0DBFE002805D1200065
:101AD0001BF366FD002005B0F0BD0120FBE7FFB55C
:101AE00087B00700002004900A98002803D0CC4853
:101AF000406800287ED1FF242D3402E00120FFF74A
:101B000027FB2100380004F082FB0500F6D028896D
:101B10004619380023F0C2FB002801D00C2000E059
:101B2000042059210590387AC9003A0079187E328C
:101B30000628019200910AD11300059ACB330221A5
:101B400030000EF373FDF0784008400008E0130009
:101B5000059A022130000EF369FDF0780121084357
:101B6000F070F078EF21084008992C00C907C90EE1
:101B70000843F070FF20C01C3071000A7071002013
:101B8000307070701C2028810220290028733031A9
:101B90001C340391702120001BF340E821006031C8
:101BA000119806917728487201D0782804D1A0684E
:101BB000012149060843A060E6650A9800280AD07A
:101BC0000120C0079649A06001204860697B01435D
:101BD00099486973A8610020208005980C2821D1BC
:101BE0000999380023F066FB41072078490FC008A7
:101BF000C00000E06CE0084341072070490F380046
:101C000023F074FC0101E06D028B1207120F0A43EE
:101C10000283E06D017E09090901017620789F2188
:101C200008402070099A21003800002323F070FB3F
:101C30001098804E002806D10699092008723800B5
:101C400011F0BBFE1FE00021380016F027FD03282D
:101C5000A0701CD93079C00604D576484030807D0C
:101C600040060CD5787A022811D10B20DD1BA0E5A7
:101C700001000000E41B000000040000B6F0A8CC46
:101C800080013818006A13214901401800790007C3
:101C900007D50321380011F044FEA0700120000395
:101CA00004903079800607D4A078002804D0A0687A
:101CB000012189070843A06003990498C86139008D
:101CC000280002AA22F000FC01280BD00499280069
:101CD00011F0E0FD002805D128000CF003F92800E0
:101CE0001BF368FC0BB0F0BDFFB5FF212D310600E2
:101CF00085B004F096FA07007ED03000FF30317ACC
:101D00004A300129049002D0707A022804D1049943
:101D1000300023F0C2FA02E0300023F0C9FA6B462B
:101D20000390187EF32108400830187603990029A3
:101D300003D00007000FC03002E00007000F403062
:101D40006B46187638893200C5195920C0007E329A
:101D50003118019200911C7E049B2007810F2209FB
:101D600028000EF36DFCFF20C01C2871000A68716A
:101D70006B46AC70587EE870707A02280DD1022153
:101D8000300025F024EDE9788A06D20F1043C00711
:101D9000DF22800E11400143E9701C2038813C187D
:101DA0003800BD6708997C3041720E990172039822
:101DB000002835D06B46988B2080707A032820D17C
:101DC00030001CF04BF90100300023F07DFA410790
:101DD0002078490FC008C000084341072070490F10
:101DE000300023F09DFB0101E06D028B1207120F02
:101DF0000A430283207800E033E09F2108402070EE
:101E00000EE00C4A50880101401C5080687E2A7EFA
:101E1000000210430007000F08432876000A687686
:101E20000021300016F044FCA070089831281BD027
:101E300002AA0DE07C2401C0A8040004A11900003E
:101E4000F4FB00C0021400003A5C00049919000081
:101E50003100380022F038FB012805D10298002813
:101E60000CD0012009B0F0BD0021380011F012FDA6
:101E7000012803D038001BF39DFBF2E70020F1E7B7
:101E80000200894810B5006804210023FFF7B3F968
:101E9000002804D10220FFF719FB002010BD01200B
:101EA00010BD70B50400814D28680079A04201D0B2
:101EB00000F073FB286804717D48446170BD10B563
:101EC00022F03DFC002801D1012010BD002010BDF2
:101ED000784970B50125096B490719D5FF2804D148
:101EE000002411F03CFF010001E001000400724BEE
:101EF0001E1F0AE0E000C2181268801900688242C2
:101F000000D00025641C012D08D18C42F2D905E0D7
:101F10006A48816AC06A814200D00025280070BDED
:101F2000FF2010B5FFF7D4FF002801D011F088FD85
:101F300010BD634870B5007800284BD1614800227D
:101F40000068082109F3BDFA002843D1FFF7E8FF34
:101F500000283FD05C4806F370FD04005A48082171
:101F600006F3FAFC05005848102106F3F5FC281882
:101F700084422FD1554806F360FD040053480821E0
:101F800006F3EAFC05005148102106F3E5FC281889
:101F900084421FD14E4806F350FD04004C480821EE
:101FA00006F3DAFC05004A48102106F3D5FC281890
:101FB00084420FD1474806F340FD040045480821FC
:101FC00006F3CAFC05004348102106F3C5FC281897
:101FD000844201D0002070BD012070BD70B5012089
:101FE0000BF04FF900285ED13B4C354D354E08E0E3
:101FF0002078401C20700120FFF768FA0120FFF7CD
:10200000B1F828780028F3D130680022082109F3BC
:1020100058FA0028ECD102E00120FFF7A3F8FFF7FF
:102020007FFF0028F8D0284806F307FD0400264863
:10203000082106F391FC05002348102106F38CFCCF
:1020400028188442E8D1214806F3F7FC04001F4811
:10205000082106F381FC05001C48102106F37CFCD6
:1020600028188442D8D11A4806F3E7FC040018481F
:10207000082106F371FC050015481021398B525BCD
:1020800001000000E01F000000040000E52A7BA022
:1020900006F36CFC28188442C8D1134806F3D7FC19
:1020A00004001148082106F361FC05000E481021C8
:1020B00006F35CFC28188442B8D170BDE803000424
:1020C000F4FB00C040A6008040A3008034A900803B
:1020D00000A0008060040004B0F500C064040004A7
:1020E000A804000488050004380500047C2401C00D
:1020F000FF305D3089080E2210B516F324FE8000F3
:1021000010BD10B504000C235843FF4940180021AE
:102110000A000B000EC0200010F36EF8200010F330
:1021200076F8200010F35DF810BDF7B586B0040016
:102130001600F64A002500920798310004AA03AB66
:1021400004950EF34EF86B46187C001F032859D8EF
:102150003006000E05901BF3E7FE1BF3F6FE0600AB
:10216000607A032806D16B461B7B0599320020005C
:102170001BF08DFF6B46187C31001CF00BF81FF034
:10218000A7FD0700FFF7BAFA6B460290187BA4235D
:10219000DD4958433031401880306B460576DC4AC3
:1021A000187C68390DF3D3FF6B46197C187B11F34B
:1021B0002CFB6B46187CFFF785FB6B46187C059A59
:1021C00031002300FFF743F96B46197B300011F310
:1021D0002AFA6B46187C2200310010F0CFFF02A8CB
:1021E000FFF7B7FA38001FF077FD6B46197B079AA7
:1021F000200012F04BFA6B46187BFFF782FF01209C
:1022000009B0F0BD0020FBE7F7B584B0050016006B
:10221000BE4A009200240598310003AA02AB039441
:102220000DF3DFFFBC4FBB49380025F0D6EA6B4603
:10223000187B001F032847D8F913380025F0CCEA93
:102240003006000E1BF370FE1BF37FFE01006B4691
:10225000187B1BF09FFF1FF03BFD0600FFF74EFAB7
:102260006B460190187AA423A7495843303140188F
:1022700080306B460476A64A187B68390DF367FFF9
:102280006B46197B187A11F3C0FA6B46187BFFF77F
:1022900064FB2800FEF7FBFF6B46187A11F35DFA2A
:1022A0006B46187B290010F029FF01A8FFF751FAAF
:1022B00030001FF011FD6B46197A059A280012F0C4
:1022C000E5F9012007B0F0BD0020FBE7F8B50D00EF
:1022D000060000241FF0FCFC8C4A07002906090EAA
:1022E000603230001BF37AFB0A280DD2874A0021A6
:1022F0000001603211548018C1602900300011F3D0
:10230000CEFB0AF062FF012438001FF0E5FC20003C
:10231000F8BDF0B50500002085B0019008780C00EC
:102320000007400F16D111F35DF80700042811D003
:1023300077480DF33EFF0600401C0BD03806000E18
:102340003106090E020004900F00200011F307F976
:10235000002802D1002005B0F0BD687A022831D1F2
:10236000280022F0C1FE132149014018807B80071C
:1023700006D56320405D8007002801DA0120019026
:102380000199049810F022FF2200049914322800C9
:1023900012F066F9201D1AF3FCEC0006000E1BF388
:1023A000C3FD1BF3D2FD0290687A03280DD1201DD6
:1023B0001AF3EEEC0106049B090E3A0028001BF00C
:1023C00066FE08E0E8680006D6E7022803D1029915
:1023D00030001BF0E9FE02201BF3B7FD01003000C6
:1023E0001BF0D8FE4D484E4A416A029840003030FA
:1023F000085A904200D1886A0104090C380010F094
:102400008CFF380011F3C2FA300011F3B1FA3E4AE2
:102410000120B100383A50503C4A0092049A3B00E7
:10242000210028000DF3C4FD3800FFF730FA1FF03B
:102430004FFC0600FFF762F90390201D1AF3A8EC89
:1024400002060298120E2B003900FFF700F8201D3B
:102450001AF39EEC02060299120E2B00380010F0BF
:1024600099FE03A8FFF775F930001FF035FC012035
:1024700071E7F3B581B006001FF02AFC234F00245A
:10248000009018206043395C00290BD0C96A8C1F6A
:1024900001000000DC23000000040000CDBBFE1D95
:1024A000C51968781BF34AFD1BF359FDB04203D1EF
:1024B000E878029910F03BFF641C2406240E042CDB
:1024C000E9D300981FF012FCFEBDF8B50025144FAB
:1024D00018206843395C002933D0C419201D22F02C
:1024E0008DFE06002DD06178002230000BF0D1F86F
:1024F0006B46198800010907090F014300911878FC
:10250000000900011870A078009910F3FEFF6B46D7
:10251000188800096081002020730DE0D48102003A
:102520009C800200507D02006666FFFFBBBBBBBB08
:10253000F0580004FFFF000060732900300001F034
:10254000E8F96D1C2D062D0E042DC1D3F8BD70B514
:1025500005000C000FF365FE0C2169434E4B5A58E1
:1025600012185A50226070BD70B505000C000FF3B0
:102570004DFE0C226A43484951188A6812188A6035
:10258000226070BD70B505000C000FF334FE0C2204
:102590006A43414951184A6812184A60226070BD66
:1025A00010B504001FF09EFB3C4A01211368A140B6
:1025B000194311601FF09AFB01208002FEF79AFF79
:1025C00010BD36490F2010B5086001208002FEF7CB
:1025D00091FF10BD70B51FF085FB2F4D00212F4ED0
:1025E0000C0030353268D30704D0A4234B435B1969
:1025F00080331C765208491C04293260F2D31FF044
:1026000075FB70BDA42324495843303140187047EE
:10261000F7B505000026204F34003037A420604372
:10262000C0198030017E01291ED16978027D914256
:102630001AD12978827D914216D1297B427D91421F
:1026400012D1C17D002902D1697BC90608D5016973
:102650000198FF314A3106221FF068F8002803D1A3
:1026600002980126047002E0641C042CD6D33000CA
:10267000FEBD30B51C00A4235843074B4D783033C2
:10268000C018030080331D750D789D751A61097B94
:102690005975DC7530BD0000D48102004C7D02000C
:1026A000F8B503242600032801D1002439E00328CB
:1026B00037DA0400461C34E0FC4861010A18822025
:1026C0006043FB4B95680021C0188173C173417C46
:1026D000F84B4906490E417401211888A1408843EE
:1026E0001880202110001AF3B8EA002D18D00B2012
:1026F00080012F1878690021FF30C94321304181C2
:10270000280000F0DFFA002804D0E868012109045D
:102710008843E8607869FF3021304189E54881606D
:10272000641CB442C8DBF8BDF0B50C000700012002
:10273000002985B003D10320FFF7B2FF75E0E178EF
:10274000A278090211430A00FF3A193A6ED1617A60
:102750004D066D0E032D69DAD44A6901891803917B
:102760008968002901D0B94260D1E07AA17A0002DB
:1027700008430B21890179180028029103D1280010
:10278000FFF78EFF4AE082216943C9480E1860793D
:10279000217902020A433000921D210008301AF309
:1027A000C0E9F17BB27B080210437D23DB00584374
:1027B0000090C11701910822300069461AF3B0E970
:1027C000039820211AF348EA0398BA498760012048
:1027D0000A88A84010430880607AC0091ED0F07BA8
:1027E000B17B0002084319D0F868012109040843AD
:1027F000F860F07BB27B0102029811434469E01D4E
:10280000F930806B1AF3DCEEFF3421346189AA4A77
:102810000004000C914200D00818608102984069C1
:10282000FF3021304189A3488160002005B0F0BD10
:10283000F8B506009D4F0024822161439C4808188A
:10284000C17B827B0802104307D06001C519A868CC
:10285000B04202D10FF330FA03C5641C032CEBDB4A
:10286000F8BD032010B5FFF71BFF90480021603032
:102870000A000B000EC00EC008008E494860886038
:10288000C86010BDF0B5002089B0040007900FF3B8
:1028900013FA0E00069082216143854892918401CB
:1028A00001000000D8270000000400009E612D7187
:1028B00008180890C27B817B1002084345D08048ED
:1028C00061010D182A6806986B683100801A9941D9
:1028D00006D32A6806986B683100801A994106E091
:1028E00028686968069AC043C943801871417D22EF
:1028F0000023D20019F3FCEE049006980F0041C5A6
:102900000822089902A81AF316E902A807C83B0092
:10291000121A8B4110D20899082202A81AF30AE968
:1029200002A807C8801AB9410191009008980822AE
:1029300069461AF300E908E00898082264A11AF32E
:10294000FAE80798012108430790641C032CACD3D4
:10295000079809B0F0BDF3B581B08E1C0A2700249A
:1029600057486101081881680198814217D1822176
:10297000614354480D18687B297B02020A432900F1
:10298000121D0A3130001AF3D6E8687B297B000259
:102990000843361D86193F1DC01907043F0C641CEF
:1029A000032CDDDB3800FEBDF8B54201822344492B
:1029B000584354184349A6684018407CC009404217
:1029C000304253D00B208001351868693F4AFF30F0
:1029D00021308189914249D02269A169914232D83E
:1029E000E1686069884237D90FF370F96A69364F38
:1029F000FF32213293895B1C1B041B0C93816A6993
:102A00007B6029D0D31DF9339F6B334BFF325F437B
:102A100031320CCA801A994100233A1A8B411BD2D9
:102A200029490122C8680223401CC8606869002146
:102A3000FF30C943213081813100FF314A313000FC
:102A400016F078FE08E0002181810FF33FF96A69F2
:102A5000FF32521C516310636069E060A06920611D
:102A60006869FF302130818917484160F8BDF7B5AA
:102A700082B00D0014000298410111480F18BE6881
:102A8000002D7ED0002C7CD0002E7AD00298FFF74B
:102A90008BFFFF21114800222D311AF3D3FD0028AE
:102AA000206008D1FF210E4800222D311AF3CAFD03
:102AB0000028206065D0687AC009786912D113E0D7
:102AC000503801C0C83601C0D4F500C0FFFF000077
:102AD000000000000000000040420F00A8040004B5
:102AE00038050004401C78610299944A89005050CE
:102AF0002068466121680220087321681C20088133
:102B000020685A217C3041722168AC2008812468F9
:102B10001221AC3420001AF3D4E8142027180190B5
:102B2000B07A2070F07A21006070083100201AF32A
:102B300054E90020A073A071E07101982071000A8F
:102B40006071E87AA97A00020843010AA0700E2891
:102B5000E1700CD2E87AA97A000208430E21091A22
:102B6000C0191AF3AEE80E20A0700020E07030000B
:102B700022F0BCFB002800D0287A2073607B40083C
:102B800000E02BE04000F12108406073E87AA97A68
:102B900002020A4329000C310C00380019F3CAEF75
:102BA000200017F061FE5924E40000280BD0687A59
:102BB000C00902D00622311902E0062231007E311E
:102BC000380019F3B8EF2800123017F04DFE002836
:102BD00004D006223119B81D19F3ACEF30E6FEB56A
:102BE0000027574E3C000297822060438519E87BFE
:102BF000A97B0002084322D008222900684619F365
:102C00009AEF019900987940084318D182206043D7
:102C100002AA811908312000FFF729FFE87BA97B70
:102C200000027D230843DB0058430090C117019147
:102C300008222800694619F37EEF0298FEBD641C45
:102C4000032CD1D30020FEBD3E48008870473D4A8A
:102C5000010012880020002A05D0002903D0C9688D
:102C6000C90400D50120704770B500281BD0334C33
:102C70000C34002918D121680022491C21600B2145
:102C8000890144186069FF30213082810FF31EF8FA
:102C90006269FF32521C5163106360692949FF3039
:102CA00021308089486070BD244D00210442651D9B
:102CB00001000000D42B0000000400006A0E58C57B
:102CC000603D4B015B199E6886420BD19E69761C64
:102CD000002A9E6103D063685B1C636002E0A36806
:102CE0005B1CA360491C0329EBDB70BDF8B5060033
:102CF0000B20800130184569012700241448610128
:102D0000603808188068B0421CD1822161431148A4
:102D10000818417CC90915D0C17B807B00270902B6
:102D200001430FD0E81DF930806B1AF35EEC01040B
:102D30002800FF3021304289084B090C9A4200D00C
:102D400051184181641C032CD8DB3800F8BD000009
:102D5000B03801C0C83601C0D4F500C0FFFF000084
:102D600070B50500002422F0DDF90600280009F006
:102D700091FC2B7A1AF304E907050F0505181814BE
:102D80001800697A022902D13400643413E0002962
:102D900011D004680FE00B2080012818046A0AE0B3
:102DA000172040012C1806E01EF0B0FFFF48FDF789
:102DB00021FA24F028ED200070BD70B50500002434
:102DC00009F068FC297A002908D0012908D00329D4
:102DD0000CD1697A032901D001290FD144680DE093
:102DE0000B2080012818046A183407E01EF08EFFBB
:102DF000EE48401CFDF7FEF924F004ED200070BD04
:102E000070B50500002409F045FC297A002908D096
:102E1000012908D003290CD1697A032901D001299D
:102E20000FD1C4680DE00B2080012818046A2534F6
:102E300007E01EF06BFFDD48801CFDF7DBF924F096
:102E4000E2EC200070BD017A012905D10B21890136
:102E50004018006A353070476130704770B5040023
:102E6000FFF77EFF0500200022F05CF9617A02295D
:102E700004D1132149014018807B0CE003F00EF9C6
:102E80000B21890161180128486902D160308078DE
:102E900001E060300078C006C10F08D02000290092
:102EA00061300DF3C9FD002801D0012070BD002064
:102EB00070BD70B504000D0022F034F9617A02296A
:102EC00004D1132149014018807B12E0207A0628A2
:102ED00002D16320005D0CE003F0E0F80B218901D2
:102EE00061180128486902D16030807801E06030C3
:102EF000007881064006C30FCA0F20002900613008
:102F00000DF3A8FD70BD10B50400407A022802D070
:102F1000207A062805D12000FFF722FFC07840075D
:102F20000DE003F0BBF80B21890161180128486905
:102F300002D16030807801E0603000788007C00FF7
:102F400010BD603040798007800F7047C068400630
:102F5000C00F70470100C96800204A0602D5090663
:102F600000D501207047F7B584B0002406000F009B
:102F7000FFF7F6FE05003000FFF71FFF039030005B
:102F8000FFF73EFF02003000FFF75DFF0300F0682F
:102F90004006C00F0AD0039800216E4607C61A00EB
:102FA000069938002B000DF36CFD0400200007B0DB
:102FB000F0BD08B50168836A01290AD100220260C8
:102FC00001007B4A180000927A4A7B4B1C310DF3BA
:102FD000CFFD08BDF8B50D00FF21040017002D310D
:102FE00003F047F90028286011D001892200461813
:102FF0007E325921C90000923A0061180D2303F076
:103000008DF90320203630702968AC200881F8BD86
:10301000F7B5FF2105000600FF364A362D3182B094
:1030200003F027F904001BD020892A007E325921A1
:103030002718C90000922000320069180D2303F000
:103040006DF9042020373870AC202081049A039950
:1030500020000EF3E7F8200003F0B6F905B0F0BD4C
:103060000020C043FAE7FFB587B01C00060000202F
:10307000069052484068002802D0504817F3DEFB03
:103080004E4F08981837002830D12079E178000297
:1030900008432BD1307A012804D0717A022901D05B
:1030A000062807D1607900228006010F30000AF05F
:1030B00004FB05E060798006010F30002ABA17DDB5
:1030C00001000000D02F00000004000039D48BA9BB
:1030D0000AF064FF050060796B461875A079587591
:1030E000384A5920C00003923749099A3018029192
:1030F000019000927A89059B290030000DF3B4FEFF
:10310000300024F09AEB05006079C3210840397A39
:1031100023008906090F890008436071069A00920E
:10312000099A089928000DF370FE280024F088EB16
:103130000BB0F0BD7CB504001EF0F2FD2549050082
:1031400048686B46401C4860E0799870207AD870D7
:10315000A07A617A000208439880E068631C01222B
:10316000694624F072EB28001EF0DEFD7CBD7FB5C1
:1031700004001EF0D5FD0500164A210001A80EF33B
:1031800045F8002807D0012200922069621C022124
:1031900001ABFFF772FF28001EF0C6FD7FBDF8B53A
:1031A0000D000124417A022922D10B218901411805
:1031B000496801291CD121F0E6FF060028000BE038
:1031C00003000100C72E00009C800200FC8002006A
:1031D000106402C0882401C01AF3CEFE7D21895DEF
:1031E00000910100009804F0FDF9002800D00024AF
:1031F0002000F8BDFEB50400401C22F01DF80500BB
:10320000FF4F57D0E8684006C00F53D0207A8006A1
:10321000010F2800FFF7C3FF00284BD0207A80065B
:10322000010F0191687A032801D001280BD12800F1
:1032300022F07CF8217A0600C32001403007800E7E
:103240000143217200E00E00EE49320020000DF330
:10325000ADFE411C46D0621C280002A9FFF7C4FE47
:103260000298002826D0287A012804D0697A0229F9
:1032700001D0062805D10022310028000AF027FAE3
:1032800003E0310028000AF089FE010002982200C4
:103290000DF364FE207AC321084001990907890EC5
:1032A00008432072D848E1790170029803F096F83B
:1032B000401C01D1380013E0D4480E22210019F33C
:1032C0004EECD2480561183817F352FACF48642201
:1032D0000092CF4ACD4B0121183817F388FA01200C
:1032E000411C16D1617B227B09021143E181E17A05
:1032F000A27A090211432173090A6173217AA1722A
:10330000617AE17201210022217262722170BE494C
:103310000A70FEBD7CB50400401C21F08DFFB84E44
:10332000050012D0E8684006C00F0ED0621C2800CD
:1033300001A9FFF759FE0198002806D021000DF3DE
:103340004FFE019803F04AF80600701C02D10120DC
:1033500020700CE0607A217A0002084307D1AD4A60
:103360000092AD4A00212B0020000DF384FF3000B5
:103370007CBDFEB50400401C21F05EFFA04E0500A0
:1033800003D0E8684006C00F01D13000FEBD687A66
:10339000032801D001280AD1207A0109280021F050
:1033A000C5FF217A0907090F000101432172E07965
:1033B0006B461872207A587202980190A07A617A4E
:1033C00007020F43621C28006946FFF70DFE0098B4
:1033D000002801D1300006E001993A000DF359FCB4
:1033E000009802F0FBFF411C02D101212170FEBDBB
:1033F0000028FCD185480B2221002C3019F3AEEBBC
:1034000082482C30C560183817F3B2F97F4864221F
:10341000143003000092814A0121183317F3E7F9B1
:103420000120FEBD70B50B004A780D7811020B2209
:10343000920180184069002429438030012902D17B
:103440000422991C02E001000422981C19F386EB67
:10345000200070BD10B5FFF7E5FD002800D1012068
:1034600010BDF7B582B005000E004F6B8C6BFFF7F7
:1034700081FCE9684906C90F0BD0297A012909D1D5
:10348000674A2B0000926748049A7E3331000DF39F
:10349000EDFDEDE5697A032901D00129F9D1002C70
:1034A000F7D0002FF5D001794A07D30F22795207C0
:1034B000D20F934204D0FB231940920011430171B3
:1034C0000179CA06D30F2279D206D20F62F4982965
:1034D00001000000CC330000000400008611AE1A89
:1034E000934204D0EF231940120111430171C178B6
:1034F0000A07D30FE2781207D20F934204D0F723C2
:103500001940D2001143C170017922798B079207CB
:103510009B0F920F934203D08908890011430171D8
:103520002800FFF7AFFC02000021280015F037FA51
:10353000A8E510B50400C8798A7903020B20800140
:103540002018406913438A786030012B02D0022B87
:103550001BD107E00270CA7842700A79027149797A
:10356000417106E08270CA78C2700A798271497925
:10357000C171200014F047FE2000FFF783FC020019
:103580000021200015F00BFA10BD0270CA784270BD
:103590000A7902714A7942718A78E3E7CA798B79AC
:1035A00012021A436030022A08D182788A70C278E7
:1035B000CA7082790A71C0794871704702788A703E
:1035C0004278CA7002790A714079F5E7F8B50500CA
:1035D0000E000024154B310020006A460CF378FDE4
:1035E000012808D121003000FEF7A2FE00222100B0
:1035F00030000DF310FB084A310020000CF397FD5A
:1036000001281ED1220031002800FEF72FFE0122E2
:10361000210013E0FFFFFFFF9C800200882401C00F
:10362000286402C06F300000C72E0000FC8002003A
:1036300035300000404B4C003E5C000430000DF380
:10364000EAFA641C2406240E082CC3D3F8BD38B54E
:103650000400FFF799FB0500E068C02188430022C1
:103660001100E060FF48130000920DF346FD207A40
:1036700001280AD100220B20800120180092006A44
:103680001100353013000DF338FDF74A2000009289
:10369000F64A2900613000230DF32FFD2100FF3190
:1036A0004A312000FFF792FF00221100200015F0A0
:1036B00076F938BD02004032002110B511849184A2
:1036C000030051846033D18419782022114319708A
:1036D000997868301143422211439970182119F3E7
:1036E000E4EA10BDF8B50E00018945690918CC6DF2
:1036F0002700203738000DF360FD002813D0D94A89
:10370000A31D483200921C002A00390030000DF33E
:1037100017FD0006000E05D02300320039002800F6
:1037200024F09CE8F8BD38000DF351FD0028F9D0D5
:10373000287A0228F6D032003900280024F092E8D6
:10374000F8BDFFB583B01400039821F0FFFC8F2172
:1037500089004018029000200190607821780002D2
:103760000843052864D9401F04060498240E401D10
:1037700000900398C17A007A08F0E6FB21F00DFD75
:10378000092686570700007A083780063500800F23
:103790000B2101280BD1F21E012A00DDF01E0506C7
:1037A00008002D16F11D0B290FDAF01D0DE003287E
:1037B00039D10120F21F012A00DDF01F05060800A3
:1037C0002D16F11C0B2900DAF01C060636162AE02D
:1037D0000098220049210CF0F1FB010028D04A7822
:1037E000901C0006000E84460020521E96460EE0F5
:1037F0000B18DA78AA4207DBB24205DC7B789342E9
:1038000002D00120019004E0401C0006000E864515
:10381000EED80098081A221A6046101A0406240EE0
:10382000604608180090002C02D001980028CFD0E4
:1038300002982030807C80070BD5049800794007DF
:10384000800F02D10198012803D10398002124F0B0
:103850000EE804980921007908420BD048206B46F5
:103860001870012058700020987003980322694650
:10387000FFF7E2FB012007B0F0BDFEB50500160022
:1038800048780C0001270C3600280CD001282FD0D6
:10389000022842D1E868C00440D522003100280047
:1038A0000DF377FA3AE0E8684006C00F0BD020F03D
:1038B0003FFD002816D00B20800128184069803079
:1038C0000078C0070ED0320028006946FFF796FB4B
:1038D0000098002822D021000DF3FAF986E54F095F
:1038E00001000000C837000000040000D5CB7D7641
:1038F000009802F087FD1BE02A00210030000DF344
:103900000EFA15E01EF020FA01905D48A178401EE5
:103910000278914207D10021017023003200280073
:103920000091FFF7BEFB01981EF012FA00E000279D
:103930003800FEBDF8B501250700524E00242D03C6
:10394000FF374A37182060438119305C0A000A3279
:1039500000280BD01088A84208D0091D0622380084
:103960001DF016FF002801D10120F8BD641C042CB5
:10397000E8D30020F8BDFEB504000D00407A02280F
:103980000CD1200003F0DBFE002807D0FF205130CF
:10399000015B0122200023F078EFFEBD182169436E
:1039A000384802AA0D1868892F000D370190781E3B
:1039B00000900821200002F099FC0600EDD002984A
:1039C0000421C06D017000214170203004210400E9
:1039D00019F39EE9207804210843207060780107DC
:1039E0006878090F000101436170E078A178000256
:1039F000084301990007000F09010843A070000A5D
:103A0000E070214930000FF08BFF0028C5D03878D6
:103A1000401C3870009801210170FEBDF8B505000A
:103A20001EF092F9174E07000024182060438119F8
:103A30000A00305C0C32931E002815D01078002844
:103A400012D118880122120390420DD02800FF30B5
:103A5000091D06224A301DF09BFE002804D12106D4
:103A6000090E2800FFF787FF641C042CDDD3380003
:103A70001EF06EF9F8BD0000F46302C0446102C09C
:103A8000892401C09C8002000210000010B5FB4C8C
:103A9000606B002805D123F0FCEE002801D0012046
:103AA0006063606B10BD10B523F0F6EEF3490020A3
:103AB000486310BD30B50020F14D0D210400030016
:103AC0008901691814E0E868401CE8601000526B36
:103AD0008A62002A00D1CB620279052A0BD12A69B9
:103AE000521C2A618362036003710020002C02D102
:103AF0008A6A002AE7D130BD10B50A68E04B002A77
:103B000003D11868401C186010BD8A6A824203D035
:103B10005868401C586010BDD8480024026A002A2A
:103B20000FD08A4210D09A68521C9A6004220A71FF
:103B3000C26A002A01D0516300E08162C1624C6315
:103B400010BD012201620A71006A07228462CD4819
:103B5000402100681EF0A4FF10BD10B50A68002ABD
:103B600010D0C64A936B83420CD1106A002809D04A
:103B7000884207D100209063C24807220068802154
:103B80001EF08EFF10BDF0B5050085B000F0CCFB37
:103B9000002000F0D7FB04007ED0286B2063B748DC
:103BA0000490416A491C4162216000F0C5FB0EF39C
:103BB000B5F803910290206800272E0039002036C6
:103BC000002803D1049A0120506220600023237151
:103BD000307A6071A079717A800889078000890F36
:103BE0000843F321A0710840B17A8907090F0843FF
:103BF000CF21A0710840F17A8907890E0843A0718E
:103C000069692869594008430DD02A6902986B698F
:103C10000399121A8B410AD3029A2869039B696996
:103C2000801A994102E0A869002800D00700029A92
:103C3000039B0021B8185941E160A060E869206148
:103C4000286A6061686AA0612868E061686820622B
:103C5000A868606220002030417B327B49089207CF
:103C60004900D20F1143FD2241731140327B5207AC
:103C7000D20F52001143FB2241731140327BD20616
:103C8000D20F92001143F72241731140327B92060A
:103C9000D20FD200114300E01AE041730221817378
:103CA000317B090701D506218173327B0121D207BF
:103CB00000D102210173827B2300009272482833D5
:103CC0003A00210007F3F2FF002806D1206001E04E
:103CD00000F032FB002005B0F0BD2068FBE7F8B52E
:103CE00005250E0000F02EFB04006448AF08CD9EB1
:103CF00001000000C43B00000004000021A408C231
:103D0000016AA14216D1A06A002803D008F33BF84B
:103D10000020A062002E66610CD0002223000092D9
:103D20005E4828333200210007F3CAFF032500282C
:103D300000D104252800F8BD70B5052500F00CFB66
:103D400004005348016AA14207D1A06A002804D0A8
:103D500008F319F800200325A062280070BDF8B50B
:103D60000F00052600F0F8FA494C0500216A81424F
:103D700015D1A06B002803D008F305F80020A0633C
:103D8000002F0CD0424B00220092454838333A00B5
:103D9000290007F395FF0326002800D104263000F0
:103DA000F8BD70B5052500F0D7FA394C216A81427B
:103DB00007D1A06B002803D007F3E5FF0020A06324
:103DC0000325280070BD38B50120FDF7CFFB304C2E
:103DD0002C20236AC15C5A6A1868DB699847206AFC
:103DE000006B02F0CEF800F0A9FA1DF0B7FF216ACF
:103DF00005000020086000F0A9FAFFF765FE2062C8
:103E000028001DF0AFFF216A002909D02E20425C56
:103E10000B000092234A2148283307F351FF01E0A9
:103E2000FFF74BFE032038BDF8B50600072021F050
:103E3000B1F9174F05004BE0386A006BA84204D077
:103E4000280023F038ED00283DD13400162E10D183
:103E5000280023F034ED002830D0687A02282DD1D4
:103E6000386A2030407B400701D52A2426E02824E8
:103E700024E0192E03D01A2E01D0182E1ED10B20AB
:103E8000800128184069817B00290DD02C2415E081
:103E9000283C01C0E83801C00CFC00C0D13900004A
:103EA000333A0000A0860100C07B002801D02924FD
:103EB00004E0386A006BA84200D0182422000021D8
:103EC000280002F0FDFA0721280007F0FBFF05009B
:103ED000002DB1D1F8BDF8B505250F0000F03CFA72
:103EE000040064D0A06A0026002802D007F34BFF2C
:103EF000A662FB4D286AA04257D100F01FFA207934
:103F0000022801D003281ED1267100F01FFA286A6A
:103F10002030072F077308D0082F0BD11A20FFF786
:103F200083FF272006F037FD40E01920FFF77CFFD4
:103F30002620F7E7286A006B23F0C4EC1820FFF76F
:103F400073FF2520EEE7012801D004282AD100F0D4
:103F5000FDF9E369626A20680B219847286A006BC3
:103F600002F00FF800F0EAF91DF0F8FE26600700F5
:103F7000267100F0EBF9FFF7A7FD286238001DF06D
:103F8000F1FE296A002909D02E20425C0B00009224
:103F9000D44AD548283307F393FE01E0FFF78DFD9F
:103FA0000320F8BD00F0D2F900E0266003252800C8
:103FB000F8BD70B5040004251DF0D0FE0600C84809
:103FC000006AA04219D0217920680325042906D16E
:103FD00005212171E369626A0B2198470DE0A06A0F
:103FE00007F3D1FE012808D1E369626A20680B213A
:103FF00098470021A1622160217130001DF0B2FEBE
:10400000280070BD70B50500042400F097F9280061
:1040100000F0A2F9002802D0FFF7CBFF040000F067
:1040200095F9200070BDF8B505000E0000F086F986
:10403000AE4F002438206043C019816900290ED09A
:10404000002D03D04521095C890705D4002E06D038
:104050004521095CC90702D01830FFF7AAFF641C8C
:104060000F2CE7D300F072F9F8BD01210020DAE748
:1040700010B523F02CEC002801D1012010BD002048
:1040800010BD38B523F026EC1620FFF7CDFE152025
:10409000FFF7CAFE924C206A4179002906D0817947
:1040A0000091417900980022FFF7E2FF216A032086
:1040B0000871206A8069002808D00DF339FE256A4E
:1040C000AA68EB68801A9941A9690860216ACB69DE
:1040D0004A6A086803219847216A4869002809D07C
:1040E0008A6A002A06D100920B0002007E4828331B
:1040F00007F3E6FD032038BDF8B50700CEC90F7001
:1041000001000000C03F000000040000727EDBAE32
:104110007C4E784D306800281ED12C6A23F0E8EBE5
:104120002C20015DE369626A20689847022824D048
:10413000002F05D01620FFF781FE0120306005E03A
:104140001720FFF77BFE242006F02FFC296A0220AF
:1041500008713068002817D0286A2030407B40075B
:104160000DD5042009F0E7F8002808D107F0FAFE81
:10417000040007F004FF844201D00220F8BD0020B3
:104180003060232006F011FC0320F8BDF7B586B09F
:1041900004001600002513002F0003AA04A905A897
:1041A0001FF07CFF059B002B14D06069002802D112
:1041B000306801256061039A0799019200912200FD
:1041C00000211E0004980B00B0470700002D01D00D
:1041D00000206061380009B0F0BD70B586B00600FF
:1041E000002503AA04A905A802AB1FF057FF059CF0
:1041F000002C09D0039A002101920A00009131009D
:1042000004980023A0470500280006B070BD394877
:104210002030017F491C01773649096A00290AD0FC
:104220000A79032A07D1427F521C4277CB694A6A36
:1042300008680921184770472E4810B5006A002801
:104240000BD02030017B032907D1012101732E48B7
:104250000722006840211EF037FC10BD70B5042015
:10426000244C236A002B24D02C21C95C1868032518
:10427000012909D1FFF71EFC002810D001200AE017
:10428000206A2030057313E0022913D1FFF712FCD6
:10429000002804D00020FFF739FF0328F0D00120C8
:1042A000FCF7BAFF18480722006840211EF00CFCFA
:1042B000032070BD03290ED1186B0B218901401812
:1042C0004069022101F066FE206A0421203001735A
:1042D000FFF7E1FEECE7062901D1062006E00729F9
:1042E00014D100210120FFF7A8FE0720FFF775FD7C
:1042F000DEE70000283C01C0A0860100D1390000A3
:10430000E83801C0E4F500C00CFC00C0082901D168
:104310000820EBE75A6ADB699847C9E71D49042082
:10432000096A002907D00A79032A04D1CB694A6AAD
:1043300008680521184770471648006A002800D011
:10434000012070471348006A002800D00120704700
:104350001048002110B5006BC9431EF0B9FB10BD19
:104360000C4810B5006B1EF0BAFB10BD30B5040050
:10437000094D0020010038224A4352199369A34293
:1043800001D110001830491C002801D10F29F2D3A7
:1043900030BD0000283C01C0E83801C010B5002441
:1043A00020290FD065290BD1084819F319FA0028E4
:1043B00005D10648143019F313FA002800D001245F
:1043C000200010BD02488260FAE700003046000479
:1043D000E8F500C0012210B5FF48072142700170C6
:1043E000FE480168930519430160FD4801681143C7
:1043F0000160FC480FF330FE012010BD002010B515
:104400000FF304FEF449491F487010BD012010B598
:104410000FF3FCFDF049491F887010BD0020704764
:104420004042022900D90221EB4A8900233289182F
:10443000ED4A1268012A01D18A5601E000228A560B
:10444000101802228A56824203DB03228A568242D5
:1044500000DD1000000600167047E349DE4A0968D7
:104460004042921C012901D1515601E000215156D0
:10447000081802215156814203DB03215156814223
:1044800000DD0800000600167047D3490278891C39
:104490000A7002794A70827821310A7082794A70F2
:1044A00042780A7142794A71C2780A72C0794872B8
:1044B0007047C9490220C043891C087048702131E7
:1044C0000870487008714871087248727047002877
:1044D00001DD002004E06421C943884200DA0800BD
:1044E0004042000600167047002070477CB56B46BE
:1044F0000024B94E1970F61D5870009801A910F0EB
:10450000EBFC00280BD0A5006B4659795D4BFF8969
:1045100001000000BC43000000040000708703B8E5
:10452000705B0FF39AFDA8196B46197940880FF359
:1045300094FD641C012CEADB7CBD7CB56B46002439
:10454000AA4E19700B365870009801A910F0B9FCEA
:1045500000280BD0A5006B465979705B0FF37DFDE9
:10456000A8196B46197940880FF377FD641C012C5C
:10457000EADB7CBD7CB56B4600249C4E19700F367F
:104580005870009801A910F0C5FC00280BD0A500B8
:104590006B465979705B0FF360FDA8196B4619796A
:1045A00040880FF35AFD641C012CEADB7CBD3EB54C
:1045B0006B460C0019705870009801A910F0D4FCDB
:1045C000002803D001A8FFF76AFF3EBD2000FFF7D7
:1045D0007AFF3EBD002800B511D1022A05D1092974
:1045E00001D8481C00BD082000BD032A05D10529BB
:1045F00001D3C81E00BD022000BD481E00BD022A16
:1046000001D0032A40D1702938D011DC8807800FEF
:1046100038D18B10093B18F3F0EC132727292935E3
:10462000352B2B35353535353535352F2F31350093
:1046300088290DD00EDC7C2922D005DC742901D01C
:1046400078291FD1762000BD802919D0842919D15D
:10465000862000BD95290DD099290BD09D2901D028
:10466000A1290FD19F2000BD262000BD2E2000BD16
:104670003E2000BD972000BD662000BD6E2000BD1D
:104680007E2000BD362000BD080000BD10B504002E
:10469000FFF7A0FF002C00D1401C0006000E10BD4B
:1046A000002804D0012802D0554A904205D14F4A33
:1046B000921E10700020517070470120704710B595
:1046C0004A4CA41E2078FF281ED0012804D10421C2
:1046D00070200FF3E1FC03E0042170200FF3E9FCEC
:1046E0005F200FF39DFC617840180106090E5F20E2
:1046F0000FF3B3FC60200FF393FC617840180106C0
:10470000090E60200FF3A9FC10BDF7B582B00400BC
:104710000D003C4E01200490B06A3B490840B06255
:10472000706A3A49084370620FF032FE01908021AE
:1047300002200FF3B1FC01200AF052FE802102207A
:104740000FF3B7FC01200AF04BFE290020000FF008
:10475000E5FC29480FF38AFC2F063F0E04993A0026
:1047600020000FF057FC002C0CD10E2D01D1284851
:1047700006E010F042F9012801D1264800E0264861
:104780000FF374FCFFF79BFF01980FF008FE049AEB
:1047900021002800FFF7EEFE049A21002800FFF711
:1047A000CCFE049A21002800FFF7AAFE049A2100FB
:1047B0002800FFF7FCFE706A1449C9430840706284
:1047C0000AF062FE04992A0020000EF091FC0AF023
:1047D00096FE20000BF042F90AF056FE049A3900CA
:1047E0002000FFF753FF0700200017E0FDF500C091
:1047F00080210080002D00809C2601C03804000428
:10480000FFFF000000A80080FCFDFFFFC00000804B
:10481000B42701C0AC2701C0B02701C00AF0A9FC31
:104820000600010020000FF02FFC310020000EF0E8
:1048300083FC022107200CF3D5FF0FF03BFC002E78
:1048400004D0102107200CF3CDFF03E01021072036
:104850000CF3BDFF390020000EF076FC04992A000D
:1048600020000EF0BDFB0EF097FB0FF035FC854DE0
:10487000002E1FD084480068002817DB07200CF3A7
:104880006DFF8009012803D1E869401CE8610AE056
:10489000022803D1286A401C286204E0032802D1C0
:1048A000686A401C6862A869401CA8610221072050
:1048B0000CF38DFF0AF023FE744E002C01D17448D6
:1048C00000E0744830612878A0420BD020002C70A2
:1048D0000AF0F4FC20000FF0F1F820000FF0FBF8D4
:1048E0006B4618703069082108433061012005B01B
:1048F000F0BD6449FF2008707047F8B580011700CB
:10490000604B050C0022DB1D9856002800DC42425B
:104910001006000E1F261F2800D206003AA642BE2F
:1049200001000000B847000000040000235DD0D45F
:10493000202905D0402905D0802905D0002404E095
:10494000102402E0202400E030242906090ECD20A6
:104950000FF38DFB290ACE200FF389FBD2200FF332
:1049600069FB410949013143002F02D14020014335
:1049700001E0BF200140D2200FF379FB210080200D
:104980000143CC200FF373FBF8BDF3B5D2208FB0F9
:104990000FF350FB4021084203D044480926019000
:1049A00003E0424809300B2601900F98310018F3BC
:1049B000D8E9002503950295CC200FF33BFB400678
:1049C000FAD5002428E0CC200FF334FB00090001C5
:1049D0004006400E20430106090ECC200FF347FB92
:1049E000D1200FF327FB0004A70004A9C851D02051
:1049F0000FF320FB04A9C9590002084304A9C851B8
:104A0000CF200FF317FB04A9C959084304A9C851C3
:104A100003994018641C0390B442D4DB0398002827
:104A20001AD0002404AF14E0A00038580102081A7C
:104A3000039918F320EE0F990006000E085541194E
:104A40000D0601992D0E0957414302980818641C60
:104A50000290B442E8DB09E00F99701EFF220A546D
:104A60000199150008560302181A02900F980F9A20
:104A70000178FF20401B09181170019A002151563E
:104A80004143029808181099002902D01099001289
:104A90000880300011B0F0BDF8F500C0002B008098
:104AA000C0A2008008A8000008680000E47A0200A4
:104AB00070B5FF4D6969FF484165FF490968816527
:104AC000FE4800248461FCF7D6FA1020FCF7B9FAFE
:104AD000680DFCF7B6FA2C6070BD10B5F54C0200FD
:104AE000616B206B18F38EEA7D22D20018F38AEAFC
:104AF000E36AA26A17F34CEE10BDF8B57D220700F9
:104B0000EC4CD200616B206B18F37CEA05000E00C0
:104B1000E16AA06A3A0018F376EA33002A0017F334
:104B200038EEF8BD10B5E34C0200616B206B18F352
:104B30006AEA7D22D20418F366EAE36AA26A17F3EE
:104B400028EE10BD10B5040009F0E3FA21001CF0B6
:104B50000EEFDB4A002317F31CEE10BD70B5040006
:104B6000D44D01206872D7480168820C114301605E
:104B70000AF091FDD4494000085A64235843A861C3
:104B80006043FCF73BFA70BD10B50124FCF72BFA2B
:104B9000200010BDC7480079704770B5FCF738FA9F
:104BA0000600FCF744FAC34C002526636563A1693F
:104BB000E5624143C348A1620168820C91430160F0
:104BC0002079002804D10120FFF7ACFFFCF724FA7C
:104BD000657270BD70B5B74C2069FFF77EFF6189C3
:104BE00018F348EDE0610500B848A16918F342EDFB
:104BF0000100A84201D8E06901E00800E1617D21DF
:104C0000C90018F338ED206270BD0A2010B5FFF717
:104C1000A5FFFFF7B9FF040010D0FFF7BEFFFFF7B5
:104C2000D9FFA448016A08000A2907D9FFF796FFAF
:104C3000FCF7D9F9FFF7B1FFFFF7CCFF200010BD5B
:104C400070B504009B4D012068729E480168820C7B
:104C5000114301600AF01FFD9B494000085A64217E
:104C60004143002CA96102D00800604305E0E869D7
:104C700048437D21C90018F3FEECFCF7BFF970BD75
:104C80008C490A6A824206D84A7A002A03D14979B5
:104C9000002900D1D4E77047F3B583B000278549D8
:104CA0000D006B6B2A6B390018F3A0EA02900C0020
:104CB000E96AA86A049A18F3A6E905000E0006221C
:104CC00018F3A0E93B00052217F362ED0191AA0F4A
:104CD000B10011430090A8003B00052217F358EDE6
:104CE000029A2300121A8B411AD3684607C8801A09
:104CF000A14115D307223100280018F384E9029A54
:104D0000801861416B4C4A07C0081043636B226BEB
:104D1000C90817F33EEDE162A0620498676320635F
:104D200005B0F0BD70B5634C607900284E8BD0148F
:104D300001000000B44B000000040000D732A56061
:104D400011D1FCF75AF9FCF76DF90500FCF779F978
:104D5000614A01001068930C98431060A0694843B1
:104D60002900FFF7A3FF2079002804D10120FFF7D5
:104D7000E3FEFCF75BF90020607270BD70B5FF24A4
:104D8000514D5A342B68C31A1B1BFF3BFF3B1B1FA3
:104D9000002B04DC5349886A401C886203E081428E
:104DA00001D8824201D2002070BD1800FFF7AFFE8B
:104DB00006002000FFF7D0FE04002868FFF7A7FEDA
:104DC0008219230000213000FCF798F92879002887
:104DD00006D12868FFF79BFE0004000CFCF705F9DC
:104DE000012070BDF8B505006846FCF742FA3E4860
:104DF00000990068814201D0FCF720FA3B480099F5
:104E00000068814201D0FCF719FA394C394E2078FC
:104E1000FF280AD105F011FD002806D0002D04D08E
:104E2000306822000D21FCF71BFA0099306881429E
:104E300001D0FCF703FA304800990068814201D0A4
:104E4000FCF7FCF9F8BD284838B50068FCF7FCF918
:104E500026480068FCF7F8F9264D2868FCF7F4F9B5
:104E600025480068FCF7F0F9214C2178FF2905D08E
:104E700028686A46FCF7F4F9FF20207038BD1C480A
:104E800010B560380078C00705D00AF011FB0DF0AE
:104E90004BFF0AF048FB10BDF8B50AF002FE114EB8
:104EA00000257560FFF7CFFF08498031086B0822A5
:104EB000104308630E48114F60380078044CC00757
:104EC0003DD01DE000A50080683C01C0802200802C
:104ED00040A6008040420F0000210080407B02007D
:104EE000002D310130F600C0E0030004647D0200B3
:104EF0009A5C000408FC00C004F800C0EFFFFFFF4C
:104F00001CF054FF009020690B2188432061206928
:104F1000F16808432061A561FCF7B7F8FCF729F9AF
:104F2000F948C760F9490868082210430860F84842
:104F300001681143016000981CF03CFF06E0A56188
:104F4000FCF7A3F8FCF715F9EF48C7600DF33FF83D
:104F5000F048F149406D4861206910218843206183
:104F600006F399FFF8BDE94810B5C03801690B2276
:104F7000914301610169E94A92681143016100218D
:104F800081610AF095FA0DF0CFFE0AF0CCFADF4A03
:104F90001068082108431060DD4A1068084310605B
:104FA00010BDFFB583B004000027DD4D05F040FCC7
:104FB000002800D0022020F055F9060002D0F06849
:104FC000C004C00FFFF70EFF1CF0F0FE002202909D
:104FD000D448009200680822012101AB1DF086FD33
:104FE0000198002817D1D048002200684A2106F312
:104FF000E0FA002802D00C9800280CD0C549CB4B11
:10500000086E496EFF221840F932002311405940C2
:10501000584008430AD0BF48C44C016E426EFF237B
:10502000F93321401A404266016620E0002C2AD064
:105030000CF3A6FE00900498226863680F00101A13
:1050400000218B41009A19003B00121A8B410AD2B1
:10505000009A20686168801AB941069A0599FFF79D
:105060008DFE002806D1AD488169491C8161FFF79A
:1050700013FFE7E0A748626821688030C260816062
:1050800000F05FF90700A24A106808218843106009
:105090009E4A1068884310609C48C03801699F4A46
:1050A00004231940D1600169994301610169032218
:1050B0001143016143E09948416A491C6D1E4162F8
:1050C0003AD10500006A401C286205F0BBFB0028AD
:1050D000974812D08169816901690B22914301616E
:1050E0008B4A116808231943116001698B4AD26801
:1050F0001143016106F3CFFEA4E080698006800FB2
:10510000012802D12869401C2861FFF72CFF06F016
:10511000B5FD7F4A10680821884310607B4A1068FB
:10512000884310608248016904229143016101694A
:105130000322114301617A4D01200AF0E54F2B490A
:1051400001000000B04F00000004000084E8760C6D
:1051500065F97C4880698006800F0328B5D1002C52
:105160000DD000F0F8F806990700884202D805989B
:10517000874204D26E48C169491CC16168E06B482E
:105180004169694A5165022141616F48FBF7EAFEB6
:105190000CF32FFF61498031086B082290430863AC
:1051A00068480169102211430161614800780228B2
:1051B00001D1022500E04025002C02D000F0CBF800
:1051C0000700002F01D001200543002E04D00B2042
:1051D00080013018406900E00020012100F002FF4A
:1051E0000AF0C9FBE807C00F01D0FBF750FF4220CF
:1051F00005401BD068060AD51020FBF730FF1020B1
:10520000FBF739FF0420FBF7C5FFFBF7D4FFA80726
:105210000CD50125AD022800FBF721FF2800FBF784
:1052200030FF0A20FBF7B6FFFBF7C5FF404D01201A
:105230006860002C16D000F08EF80699884202D8DB
:10524000059988420ED2E869012109044018E861F5
:10525000FFF72CFEFFF71DFE02981CF0B5FD0020A5
:1052600007B0F0BD0AF035FCC02008F033FF02980B
:105270001CF0AAFD0022D2432F48009200680822A9
:10528000012101AB1DF03CFC0120E9E710B505F060
:10529000E3FA002803D026484068002801D0FFF731
:1052A00005FE10BDF8B51F4A224811680826B14313
:1052B00011601B4A1168B1431160224C21691C4DD9
:1052C00004273940A9602169B943216121690B2272
:1052D00011432161401E1AD1FFF74FFE06F0D8FCA2
:1052E00020693840A8602069B84320610D490868EA
:1052F000B04308600A490868B0430860A0698006A6
:10530000800F012802D16869401C68610948A169C1
:105310008906890F0329D9D1F8BD000080220080B9
:1053200000A7008000A30080683C01C000A50080A9
:1053300030F600C088130000302601C0B0F500C070
:105340001800040040A600801000100001207047E3
:105350000948407A704710B5FBF709FF0400FBF7D6
:10536000D2FE201A05D50549C86A401CC862002033
:1053700010BDFFF7C6FB10BD683C01C030F600C091
:10538000704710B5012403200CF37DFFFF49096B22
:105390000205090C0B05120D1B0D9A4204D12203C4
:1053A00010401140884200D10024200010BD24216B
:1053B0004143F74A10B58C180CF365FFE269010010
:1053C000D204C9040120D20CC90C8A4200D10020A9
:1053D00010BD10B502E00120FBF746FF0420FFF7E7
:1053E000E6FF0028F7D102E00120FBF73DFF052092
:1053F000FFF7DDFF0028F7D102E00120FBF734FFC3
:105400000620FFF7D4FF0028F7D1E24C0BE022F092
:105410009CEA002804D020680022622106F3D3F819
:105420000120FBF721FF0320FFF7C1FF0028EED189
:1054300010BDD948402110B517F37CEC10BDF8B56C
:105440000D00070024205043D14940224418390060
:10545000280017F3D4EB28001EF01AFF2800403074
:1054600017F30EED3900403120220D00009017F3A4
:10547000C6EB29882269A0690D00603D0026521EF6
:10548000904207D1E0680A1D824203D90500643DBD
:105490000E1A361D0098390020302A006431009021
:1054A00017F3ACEB002E06D00098616940194968EB
:1054B000320017F3A4EBF8BDFFB581B0002405005E
:1054C0000E001700052018F383FC4188B34A91426F
:1054D0001BD101004031286031600988403909043E
:1054E000090C0AD00F229201914206D8643038602C
:1054F000049820390124018007E005200EF3C8FC40
:105500000004000C05210CF3D1FE200005B0F0BD15
:1055100038B504001CF054FC05009C4840308069FC
:105520009B49000CC03148610520694618F367FCAF
:1055300000280BD04188994A914207D1984941806F
:1055400005222100FFF77BFF012400E0F2ED4496E5
:1055500001000000AC530000000400003B2D53BFCD
:10556000002428001CF03AFC200038BD38B50500A6
:105570008B48403000698B4C000C80342063042041
:10558000694618F346FC6B4619880905C90D0028C1
:10559000A16212D04021095A874A6039914207D945
:1055A0002800403017F376EC0021C943018003E066
:1055B00004222900FFF74DFF012038BD38B5040053
:1055C00077484030006A7749000CC0318863062074
:1055D000694618F31EFC00280BD0010040310A88F0
:1055E000682A01D968220A8006222100FFF731FFCC
:1055F000012038BD6B49F0B56C310A0068486C3247
:10560000006B040C08001430C46065484030006A28
:105610002705030C080054308363CE69012031054F
:105620000500090D3F0DB94200D1002501273F03B8
:1056300001003E403C40A64200D00021D2692943EF
:1056400015051E0504002D0D360DB54200D10024B0
:105650000C433A403B409A4200D000202043F0BD2A
:10566000F8B500210026554A4E481060544A4F486C
:105670001060544A37201060534AFF20401C1060CD
:10568000524A102010604748042280300261504A7C
:10569000426102225302836102624E4D052206637B
:1056A00012024562C2619A00C262494A4A4FCB0067
:1056B0005C1962600124A4021219491C0129EF50EF
:1056C000F5D3444BC900CC186260444A5A5035495E
:1056D0000622C0318A61424ACA6102221D008A62E2
:1056E000D20120350A62CD624A6200228A63012219
:1056F00012033B4B4A630022D40066197360FF33E8
:10570000384E5B1C521C012A2E51F5D3314CD2006D
:10571000203415196B603300A35005224263220028
:1057200028328263022253024A609E00C363103C07
:105730000E618C6000220B604A6122003832002129
:10574000CB001D196A600125AD025219491C0129BF
:10575000E750F5D3C9000B195A606750114903226D
:10576000CA66214A0A673722CA67AA104A67120125
:105770008A671E4E002106601B4F82600D00C160CB
:105780000421380017F30AEBE80081194F60FF3756
:1057900014497F1C6D1C362D3150F1D3042127E0B4
:1057A000C0A30080B0460004B0F500C0604800040B
:1057B000EFBE0000BAAB0000DC08000048BB0200EE
:1057C0004CBB020050BB020054BB020058BB02009D
:1057D000007B01C0B87201C0004000800050008012
:1057E000008401C000100080001B02C0007101C0D5
:1057F000380017F3D4EAE80081194F600F49104BC5
:10580000002531501D600E484030C461022484617F
:105810000B4AC10C403A51620A4F47610461116260
:1058200020374762046291625E633720186311611A
:105830000CF304F904488560F8BD00000000018005
:10584000C0A30080B87201C0C0A400809948142190
:1058500010B517F37AEA10BD70B505000E0001D13E
:10586000012070BD30898419607A217A00020843D2
:1058700001280DD1607B217B00020843032807D15A
:10588000002D11D0280022F06EE8002813D001E08E
:10589000002D03D0E87AA073A87AE073607A217AA9
:1058A0000002084301280AD100223100042000F040
:1058B000A6F9002803D1300017F308FFD0E7002035
:1058C00070BDF8B50D000400110000267A481F00D5
:1058D000320017F325FF0028206014D00221017345
:1058E0002168202008812068012120302860017271
:1058F000002141722868390A077341732968002022
:1059000088720126C8723000F8BD1CB50C00030077
:105910006422694601A8FFF7D4FF00280FD0009841
:1059200000210174002C417405D0019901234A7BA8
:105930001A434A738C61022181720021C17201985D
:105940001CBD10B5040008001100FFF7DEFF0028A1
:1059500003D001002000FFF77FFF10BD2D8C4A917E
:1059600001000000A85700000004000068F780D381
:105970000022F0E77CB5140005000B0064226946A4
:1059800001A8FFF7A8FF00280BD00098210A047493
:105990004174022181720021C17201992800FFF730
:1059A00065FF7CBD7CB5040015000B00FF22913221
:1059B000694601A8FFF78FFF002811D00098002149
:1059C0000174417406222900123017F32CE9009962
:1059D000082088720020C87201992000FFF746FF56
:1059E0007CBD7CB51C00160005000B00FF22913227
:1059F000694601A8FFF76FFF00280DD0009822002C
:105A00003100103017F30EE90098210A8472C17238
:105A100001992800FFF72AFF7CBD7CB514001E0009
:105A200005000B006422694601A8FFF754FF002817
:105A300011D00098210A04744174062231001230FA
:105A400017F3F0E80099082088720020C8720199C5
:105A50002800FFF70BFF7CBD70B50600108915000C
:105A6000841800222274200062740622123017F378
:105A7000DAE8E07AA17A000208430830A072000A4E
:105A8000E07229003000FFF7F1FE70BDFEB51D0089
:105A900006000F0014000B006422694601A8FFF7FE
:105AA0001AFF00280ED0742F0CD10098E521017444
:105AB00044740321857481720021C1720199300000
:105AC000FFF7D4FEFEBD0000003D01C0EC04000461
:105AD00070B50500008944191EF0CFFE00280AD0D9
:105AE000607B217B000208430B2804D00A2802D0E7
:105AF000052004F096FFFC4BFA481C6800222900A0
:105B000000680223A04770BDF848011F0860F848EC
:105B100001214170002101707047F4490020091FE4
:105B20000860F349487008707047F14841780029CF
:105B300001D001210170704770B51CF055F90500C6
:105B4000EC4817F360FE040028001CF051F9022510
:105B50000DE020002573FFF7BBFF1CF045F90600A0
:105B6000E44817F350FE040030001CF041F9002C0B
:105B7000EFD170BD70B51CF037F9DD4C05006078D1
:105B8000002809D0D94904200856411C04D0811CA2
:105B900002D0002104F3D3FFD7480078012802D1B6
:105BA000142004F02AFF002020720420FBF724FDBB
:105BB000D248002200680C2105F319FDFFF7BCFF55
:105BC00028001CF015F970BD10B5FFF7D3FFC849C8
:105BD000002008704870CA49086010BDC448017AA6
:105BE000032901D0032101727047FF2800D008402B
:105BF0007047C44910B509681BF0E0EE7D22D20061
:105C000017F328EA8905800A084301D021F0FEED48
:105C100010BDF8B50024160005000F002200002971
:105C200001D03889C2191EF0DDFB00287DD0B049B3
:105C3000087A03287AD00228FCD0680726D5002FDE
:105C400024D0507B117B04020C430B2C08D010DCB9
:105C5000032C0BD0082C09D0092C07D00A2C13D107
:105C6000A948AA490088097808430BD0FF250526D2
:105C700015E0102CFAD0122CF8D04F2C04D1FF25AF
:105C800007260CE004208543042608E0062E06D1F2
:105C90009648001F006817F308E9C0055CD49348D4
:105CA000001F006817F300E901002800FFF79DFFBF
:105CB000002851D08E484030818A002900D1868248
:105CC000934E0025002C1AD0308800280DD087492B
:105CD00004200856401C08D1081F00684079FFF7CF
:105CE00088FFFFF771FF35804DE01CF07DF8040060
:105CF0008048390017F3DFFD20001CF079F87B4F56
:105D000004243F1F38680221045779480172601C3F
:105D10000FD0A01C0DD00121200004F310FFC820DB
:105D200009F090FB0021200001E026E016E004F3DA
:105D300006FF38684079FF2828D0FFF75AFF3088DF
:105D4000002823D01EF04EFB002803D0FFF73CFFB5
:105D500035801BE0308819E00020F8BD680715D5B4
:105D6000002F13D01CF040F804006248416F4BAF85
:105D700001000000A45B0000000400009C98F5678F
:105D8000390017F3A2FD20001CF03CF808E068077A
:105D900006D5002F04D0FFF7D9FE3800FFF7A2FE8A
:105DA0000120F8BD5748582110B516F3E2EF10BD99
:105DB000F8B500200D00534F1600B88232E0687825
:105DC000297800020843FF38163821D1E978AA78EB
:105DD00009021143CC082800E200914218D1121D9B
:105DE00011040914B14213DC0821082C00D221004F
:105DF000CA00011D4348143016F31EEF06E0E00010
:105E0000C019002114300A0006C0641C082CF6DBFF
:105E1000E978AA7808021043311A091F0E043614D3
:105E20002D1D4519042ECADCF8BDFFB50A208BB024
:105E300000251F0005900B98099540692E000790DA
:105E40001FF0E8F906900B980B990089441824314B
:105E500040188446E078C00701D1A01D01E0200071
:105E60001230A1780A07930F012B04D108090828E2
:105E70001FD13880CAE0910F02D14025092017E0D8
:105E8000028829498A4209D142888A4206D18288F9
:105E90008A4203D101252E00280009E00078C007BE
:105EA00003D008250326022002E002252E0003204D
:105EB0003880A0780007800F022864D10D98002751
:105EC00007706046801D09900798407A02285AD1D1
:105ED0000C98002840D00C9820300A90007DC00615
:105EE000800F012822D90C98183016F3E8EF00072C
:105EF0001CD501201BE00000B4F500C0F0F500C087
:105F000064F600C0143D01C0003D01C000FC00C0AB
:105F1000B0F500C048F800C09C2401C01C3E01C080
:105F2000C4F700C0C8F700C0FFFF00000020A17840
:105F30000A07920F022A03D10909090700D5012790
:105F4000384309D00A98324A007E41072000490FA1
:105F50000C3017F3D9FD059004A903AA0091019212
:105F600006981121490140180378059A07982100E5
:105F70001CF027F90398002802D00D980121017028
:105F8000049800283FD02348006816F398EF284271
:105F900039D0A0780007800F022837D11E4FB88A69
:105FA000002833D0C120C0000025089026E0B04270
:105FB00002D01A4988421ED1E08A1849884207D087
:105FC00021000998163102221BF03CFC002812D156
:105FD000A069401C1AD00998022208A91BF032FCC3
:105FE000002808D1099821001A30183104221BF02A
:105FF00029FC00280AD06D1C082D04DAE800C41919
:10600000A08A0028D3D100200FB0F0BD0120FBE70B
:10601000FC80020060F600C0143D01C0FFFF0000DC
:106020007047704738B505000C000021684621F024
:10603000B2EC6B46187880070ED101200DF039FDC7
:10604000012C01D1092400E014240DF038FD2000BA
:106050000CF313F8002403E002200DF02AFDF1E711
:106060002100280007F0DFFF010020000DF0B9FF3C
:10607000641C2406240E082CF2D338BDFE4A106B93
:10608000FE494863506B8863704770B5040059201F
:106090000D00C000211820007E300FF3F3FBFFF746
:1060A000EDFF0BF3FDFF0B2080012018406920302D
:1060B000C17A28000FF3E2FB28000FF328FC70BD23
:1060C000EF49486A0422904348627047002010B5A7
:1060D0000FF38FFC0021062007F0ADFA0CF306F851
:1060E0000121062007F07AFA0CF308F8E34840385B
:1060F0000168820C114301600CF39EFC10BD10B5C9
:106100000EF0A8FC10BDF8B505000E00DD4C170020
:106110002078A84202D16078B04206D03100280031
:106120000EF086FC206125706670D748406A806951
:1061300000280DD03A003100280011F0A9FC216997
:10614000884213DA3A003100280011F0A1FC0EE079
:106150003A003100280011F072FC2169884205DA0A
:106160003A003100280011F06AFC00E00800616884
:10617000884200DB0800A168884200DBC9DBDD043F
:1061800001000000A05F000000040000CF42260BC9
:106190000800F8BD10B50CF0F0FD0006000E10BDB3
:1061A00010B50CF0EDFD10BD10B504000CF0EBFDCA
:1061B000CF22F321002806D0022811D0032820780E
:1061C00013D0084002E020780840001D10402070E5
:1061D0000CF0D6FD012820780BD0800880000BE061
:1061E0002078084010401030F1E708403021084383
:1061F000EDE780088000401C207010BD00210800E1
:1062000010B511F0D1FA10BDA34A5368834203D0F0
:106210000029506000D0F1E770479F4A936883429D
:1062200003D00029906000D0E8E770479A48806862
:106230000006000E704710B5140002688A4201D1B2
:10624000FF2909D1016007F0D9FB93498968884289
:1062500002D02100FFF7E1FF10BDF8B505000800EE
:1062600000210091E9681600FF24C9050AD5694696
:106270000BF0F0FA012805D16B46894819784018CF
:10628000403004790B208001320021002818FFF7EC
:10629000D2FFF8BD080010B504781900A407A40FB8
:1062A00014700FF3C1FB10BD7B48C06870477A497A
:1062B000C8607047FFB50800002183B01700794D12
:1062C00000912A881E000C00002A01D00124298098
:1062D00001788907890F029101A90FF3A5FB6B468D
:1062E0001A79197A03980CF0EAFA0CF0B5FA0BF364
:1062F000A7FC3800684F19D06B4869460DF0CDFBFC
:10630000002813D17869401C78610098800602D477
:10631000002005F0C5FC0098C00601D405F0E0FCA3
:106320000BF38EFC002069460DF0B7FBFE606B4658
:106330001A79187A03990CF0FEFCFFF75FFF0DF055
:10634000B7FB0BF377FC002E05D16B461A79197A4F
:1063500003980CF0D9FA002C01D00120288007B056
:10636000F0BD10B50CF36CFB10BD10B50CF005FDC5
:106370000006000E10BD70B50E040500360C4B482B
:106380000022310017F3EAF9040006D14848002240
:10639000310017F3E3F904000AD0022020731C2017
:1063A000656120812018702116F316EDAC20208144
:1063B000200070BDF7B5FF212D310700FFF7DBFF8F
:1063C00005002BD01C202E18288102982C00AC34FC
:1063D00006602021200016F300EDA078F32180084C
:1063E00080000840001D01070198090F00010143CA
:1063F0005920C000A1703918200006220C3016F375
:1064000026EC3900FF3106224A31A01D16F31EEC9E
:1064100003216820F46581550520B0702800FEBD79
:10642000FFB583B01400018945690E181C21471877
:1064300001817021380016F3A6EC1E480699006809
:106440000C9B0279019200910499220030000FF315
:10645000FFFA218818480022814206D161888142D2
:1064600003D1A188814200D101220699280012F0AF
:1064700009FAB870287A032826D10698052104283D
:1064800021D005281AD00D281ED11CE000A50080BF
:1064900040A3008000A80080E4F600C0F05800048B
:1064A000304401C04CFD00C0204E0000A804000490
:1064B00038050004F4FB00C0FFFF0000687A0228E2
:1064C00001D0012800D1B970380048E710B50400A8
:1064D000FBF780FD012805D1200017F315F90020F6
:1064E000C04310BD002010BDFFB5FF2181B00600E4
:1064F0005D310B9FFFF73FFF040002D1401E05B046
:10650000F0BD2089039A05190A23002F009200D1BB
:106510000C235920C0003118029A2000FFF780FF99
:106520000220287000206870049820352870000A26
:106530006870218921810A99852001552000FFF783
:10654000C5FFDCE77CB50C0015000699002201921E
:1065500000912A002100FFF7C7FF7CBD7CB50C002D
:10656000150006990122019200912A002100FFF7EF
:10657000BBFF7CBDF0B5150007000E000A0085B01A
:106580000024290068460FF3A6FA0028F5906481DC
:10659000010000009C63000000040000E7D3A3B6E4
:1065A00013D12B001D3B16F378ED11100A101010BB
:1065B000100E0E0E0E0E1010100E10100E00307871
:1065C0006B4618730CE00024E443072D06D1002E1F
:1065D00004D00822310003A816F342EB002C03D1AB
:1065E0003800694621F0EEE9200092E7F0B513008B
:1065F00087B006AA00921A00002505AB07F0F9FB48
:106600000699059888422AD00CF03CFF0DF08FFBCC
:10661000FD4E3068B10C88433060059800281ED0CC
:10662000002401AF01200599A04008420BD0A00032
:1066300078556D1C042C06D101200BF3FFFA30684D
:10664000E10208433060641C0D2CEBDD002D06DDFB
:10665000FF20785501A80BF363FA0BF319FB88E6CA
:106660000A00012110B5FFF7C1FF012010BD10B5D0
:106670008A781407A30F022B07D101282AD1C878E2
:10668000C10727D1800725D422E0A40F15D1130913
:1066900016F302ED0E080808081E1E20201E1E0814
:1066A0001E1E0A20022010BD012811D0032811D17E
:1066B0002031087804280DD10AE0012B0AD11309F2
:1066C000083B16F3EAEC080707070505050505076B
:1066D000012010BD032010BD010070B50A008C78A8
:1066E000123225070020AE0F931F022E0CD1CC785A
:1066F000E50705D1A00701D4100070BD180070BDDA
:10670000A207FCD4881D70BDAD0FF5D0012EFAD1C3
:1067100022090A2AF6D00E2AF0D00F2AEED070BD38
:1067200010B504001EF0B1FD617A022904D1603079
:106730000078022807D203E0032904D0012902D0FF
:10674000207A012801D1012010BD002010BD0028B1
:1067500010B509D01EF072FD002805D0192149019D
:106760004018007A012800D0002010BD70B5040048
:106770001BF058FB0500E17AA07A1EF096FD0FE0B1
:10678000E068C00407D52000FCF7F4FB02000121FB
:10679000200012F07CF9E27AA17A200005F081FE57
:1067A0000400EDD128001BF041FB70BD10B50400C2
:1067B0001EF044FD416C002909D09B21890042183C
:1067C000924903004118643320000FF3C9FA10BD49
:1067D00010B504008D4820180FF30FFB1320400163
:1067E00000212018017281720520C00120188160EB
:1067F00010BD70B505001EF021FD040028001EF03C
:1068000044FD8F218900007A61180C008207203432
:106810002079920F002817D0002A15D1227A25312D
:106820001207D60F0FF39BF9207A0007C00FB04272
:1068300001D0FBF766FF280010F054FB207A000718
:10684000C10F287A0CF0DCFD70BD10B504001EF0FD
:10685000F5FC8F218900401800222D210A54253093
:106860000FF394F92000FFF7C4FF10BDF8B5050041
:106870001EF0E4FC1321490141180C780923DF22A2
:10688000EF269B01022C07D10F79C01837400F71FA
:10689000017E0024114019E05C4C443C245CE40778
:1068A00002D18C78002C00D001240F793740E60704
:1068B000F60E3743002C0F7104D1C118097E202237
:1068C000114302E0C118097E1140C018017628006A
:1068D00010F008FB280010F08DFB20000BF37EFF6A
:1068E000F8BD10B504001EF0A9FC132252010021CE
:1068F000801881702000FFF7B9FF10BD10B50400AB
:1069000020001EF0C2FC60300078012802D920006F
:106910001DF051FEE27AA17A200005F0C2FD0400CC
:10692000EED110BD70B504001EF088FC13214901A2
:1069300043181A780921FB258901022A01D1002276
:1069400002E0002A05D101224018417E294041760B
:106950000FE0DA78002A00D00122002A04D143187F
:106960005B7E04252B4302E043185B7E2B404018DE
:1069700043760121002A00D000212000FFF766FBAA
:10698000200010F037FB70BD10B504001EF056FC5F
:106990001322520100218018C17020003E343C17A0
:1069A000010000009867000000040000B40970DADC
:1069B000FFF7C2FF10BD1B4A831A90420ED005DCC0
:1069C000194A801A0AD007280ED107E0174818186C
:1069D00008D07D22D200801A06D101E00020704745
:1069E00001207047022070470E29F9D8F6E70029E8
:1069F00003D00E2901D10B4870470A48C01F7047C9
:106A000010B5040008001100FFF7F1FF2070000A24
:106A10006070012BE2700BD10A200EE000A3008011
:106A2000610200006E09000060090000CEF9FFFF5E
:106A3000022B01D1282000E01420A07010BD10B559
:106A4000040007F022F8012801DD012000E0002009
:106A5000002C06D0012C07D0022C01D10BF364FBD3
:106A600010BD0DF075FA10BD0DF080FA10BDFEB529
:106A700004002120405C0E00210000257E312F0003
:106A80000028019125D00B218901611849692B2229
:106A9000525C90423BD130002C3122301AF0F0FE93
:106AA000002834D1207A012502281FD130000C3073
:106AB0001EF04EFC00280AD0C168C90416D4A17A81
:106AC000827A914212D1E17AC07A81420ED10127B5
:106AD0000CE0207A022836D120001EF0B9FBFF30EE
:106AE000FF30801C407F800711D501253000123017
:106AF0000199062200901AF0C3FE002807D03448FE
:106B0000009906221AF0BCFE002800D00025207A49
:106B1000022816D1012D07D101980622B11D1AF0C5
:106B2000AFFE002800D101271DF0CFFE002808D0BD
:106B3000012F06D1012D04D102201EF0D9FB01F056
:106B40001EF82800FEBD0128FBD1CEE7FFB583B0BB
:106B50001C000622070001200190380080300290BE
:106B600086697761707B4008400070730298806985
:106B70000500AC35B23016F37EE80598002805D044
:106B80002800059906220C3016F374E8E87897215E
:106B90000840E870387A022804D1029881693800E8
:106BA00020F01EEF002C03D0207801210843207034
:106BB0003000FFF79FFC002801D1019005E0002C78
:106BC00003D02078400840002070019891E4000034
:106BD00060EB31008168002907D17121095CC9434C
:106BE000090704D1C06D002801D0012070470020A2
:106BF0007047FF4AFE4B11544A00521892085B1C22
:106C000089081A545A1C1154704770B50C00487802
:106C10000978F74E000200250843B61E012816D158
:106C20000221072006F009FA002801D0012070BDDA
:106C3000E078082803D908207070E07000E07070D8
:106C4000A078307071780020FFF7D3FF03E07078F0
:106C5000E0703078A070280070BD0322002112027D
:106C60008018C16201634163816370470100E1489C
:106C700010B504F351FF0100DE480C3804F30EFF99
:106C800010BD4169496815E0814212D108690028A8
:106C900002D0CA68C26002E04A69C8685060C86829
:106CA000002802D00969016106E008694969886025
:106CB00002E0C9680029E7D10020704770B50500DF
:106CC0000C001EF0ECFA0C30C26D81686030521876
:106CD000FF2195312170090A61700821A1700021FE
:106CE000E170807CA0722900FF31E27206224A31F5
:106CF000201D15F3C0EF0C2070BDFEB50400002070
:106D0000050002900E00200000941EF0A1FA07007A
:106D100035E020001EF0C3FAE1680C30C90428D524
:106D2000010060318A7CB24223D0002E02D0007D67
:106D300001281ED18E74029800280BD12020C05D3E
:106D40000C2242435523643201A902A8FEF7EBFD51
:106D5000019D103529002000FFF7B0FF01002D181C
:106D60000198C27A837A12021A4351188172090A71
:106D7000C172E27AA17A200005F09DFB0400002C8C
:106D8000C7D10299002902D00098FEF797FDFEBDF9
:106D900070B5050002201EF06BFA0CE02000FFF732
:106DA000E0FC002803D029002000FFF778D45447E6
:106DB00001000000946B0000000400004066056EB6
:106DC000A6FF217A200005F0F5F80400F0D102209A
:106DD00015F063F90DE02000FFF7CDFC002804D08A
:106DE00029002000FFF793FF70BD0221200015F05D
:106DF00063F90400EFD170BD70B50125002104F0E6
:106E000004FF8048801E007800280FD07D4CE41CD1
:106E1000207800280AD0280004F0ABFE611E097813
:106E2000884203D800202070FFF7BCFF70BD10B56A
:106E3000040010D060690168491E0160A068FFF776
:106E4000DBFFA06800211AF0F1FF2000FFF723FF0D
:106E50002000FFF715FF10BD10B51EF003FA8F21BB
:106E600089004418C03401E0FFF7E1FFA06B00285F
:106E7000FAD110BD010010B54A7A0020022A03D1D0
:106E800008001EF016FA0C3010BD10B5FFF7F2FF27
:106E90000021C1650166416606216C3015F390EF53
:106EA00010BD10B50400FFF7E5FF002101758160FA
:106EB000C16001612000FFF7E8FF10BD524870B5C6
:106EC0000C3804F3C4FD504804F3C1FD4F4E0024B8
:106ED000250018206043811935504B484D600C380F
:106EE00004F3E6FD641C0C2CF3D308210020FFF70B
:106EF0008AFE002070BD70B505001EF0DAF90400AE
:106F00000C342000FFF770FE00281BD1A07FC007C3
:106F100018D10121280020F022ED002812D10B20E9
:106F200080012818406940308189394816F3FCEB0C
:106F30002168884206D22800FCF77EFD002801D196
:106F4000012070BD002070BD10B5FFF793FF040055
:106F500001E0FFF76CFF206E0028FAD110BDF3B5F9
:106F600081B00E0001981EF0A4F9040001981EF0F3
:106F700079F907000C341AF069FF0500002E11D0D2
:106F8000617D0020002900D06075217D012909D193
:106F90002075032000023818C16A491EC16201E051
:106FA000FFF745FFE0680028FAD10198FFF7CCFF12
:106FB0000198FFF7A0FF002807D001980022FF30BA
:106FC0004130018A019820F0E2EC28001AF042FFDB
:106FD000FEBDF7B584B005000E0048680390280098
:106FE000FFF748FF009003980024002871D0039811
:106FF0008068029001890F18380014300190FC6DF0
:10700000306807E0A2F500C0443401C0183301C065
:1070100088130000401E3060029804F0C6FD01286D
:1070200002D10298FFF7E8FE01984078002803D1CA
:10703000E078F7210840E070687A02281DD1287AAC
:1070400006281AD1A079C0070CD1306800280CD1CD
:1070500000986030807C002807D10221280020F0B1
:107060007EEC00E00698002803D0E0782021084359
:1070700002E0E078DF210840E070287A032809D197
:107080006820C05D001F042804D3019A390028003D
:1070900016F000FC6820C05D0C28A07812D1000713
:1070A000800F029802D10CF007FC01E00CF02EFCDE
:1070B0000400687A02282DD1306800282AD10022E5
:1070C000110024E00107890F04D102980CF036FC6E
:1070D00010E02BE000090C2801D0042805D101980C
:1070E000C16902980CF09EFC04E002993A00280065
:1070F0001CF02DF80400687A02280BD12800FFF755
:10710000FAFE002806D0FF205130415B0022280003
:1071100020F03CEC002C03D1029800211AF086FEEE
:107120000398FFF7B8FD0398FFF7AAFD200007B00A
:10713000F0BD70B505000C0004E00022210028001D
:10714000FFF747FF20680028F7D170BD3EB56946BC
:107150000400FFF7BDFD0300552120006A46FEF73D
:1071600072FC3EBDF3B5002483B00E0003982700E7
:10717000019400F0A9FB009003981EF073F83321EE
:1071800009014518002E36D0039800F09FFB04003B
:107190001DF0A5FB002813D002201EF0B3F80399C0
:1071A00088420DD1208802280AD10098C030007E84
:1071B000002805D1FAF785FF002801D0FF5A2916CB
:1071C00001000000906F00000004000013BCD60214
:1071D000012000E0002000280ED06068C00709D020
:1071E0000398007A04F012FF002800D0012760689D
:1071F000C00701D10120019003988030007A0CF083
:1072000019FB04000C2002902EE0002016F365FF0D
:10721000F9E7686880680189401860300299002E9B
:10722000017213D02968012901D0012C04D10199E0
:10723000002901D01421417228680022012801D8B8
:10724000002F08D0012C06D9012204E02868012271
:10725000012800D8002203982900FFF7C4FE012866
:1072600002D1002E00D0641E2868002803D0002E12
:10727000CFD0002CCDD1002F0AD0002C08D0009800
:1072800014228030C06B01040398090C00F027FE23
:1072900005B0F0BDF8B505000E001AF0E1FD0700DD
:1072A000287A032804D1280016F0DAFA00284FD0F3
:1072B000687A022841D128001DF0DEFF032109026F
:1072C0004018C06A002803D100212800FFF754FFAE
:1072D0002800FCF72FFC002E04D00B20800128187A
:1072E000406985682800FFF7CFFD0400E868C00406
:1072F00019D5207D002816D121005C312800FFF728
:1073000022FF210008312800FFF71DFFF94800780F
:10731000002808D06034A07C002804D00020A0748D
:107320002800FFF71DFF002E12D0EA7AA97A280064
:1073300005F0D5F80500D5D10AE0297A032907D14F
:10734000032805D17120C00029182800FFF7FBFE93
:1073500038001AF089FDF8BDF3B581B00D00019831
:107360001DF0B1FF040001981DF086FF06000C34EB
:107370001AF076FD070003200002002D25750AD1C2
:107380003018C16A002901D0491EC162019800214C
:10739000FFF780FF1FE0012D1DD1627D0123002139
:1073A0001D00002A00D165753018C26A521CC262E5
:1073B000D048007800280ED000221800130004F0F6
:1073C00003FC012807D16034A07C002803D1A574F8
:1073D0000198FFF7C5FE38001AF046FDFEBDF8B56E
:1073E0000D000600088901234718487BC00730D1EB
:1073F000C14800220188C1481DF013FB04002AD1B6
:10740000BD4800220188BD4803231DF00AFB04008B
:1074100021D1B849C868401CC860707A022818D1C8
:10742000F86D8179C90714D180780107890F10D1CF
:1074300000090C280DD130001DF045FF0B218901FA
:10744000711849690C304031897B0160022140305C
:1074500001750020F8BD287B20736661A8881C2672
:10746000A080A519702239002800268115F380EC30
:10747000AC2020812018E865F96D0A88203215F3C8
:107480000EEC20002681F8BDF3B585B00120002464
:107490000290059801941DF016FF0598FFF7F4FC83
:1074A000070005005C371AF0DBFC03900598007AB2
:1074B000032804D1059816F0D3F9002875D060355B
:1074C0000495E87B4006810F12D03968800F400098
:1074D000884200D308000499897B401A05062D0EC6
:1074E00067D078688068018940186030067A1BE0B0
:1074F0003868F3E77868002813D08068641C018935
:1075000024064018322160304172007A240EB042C5
:1075100001D0002102910600059800223900FFF7F2
:1075200062FD6D1E2D062D0E012DE3D87868806852
:10753000018940180299012922D1010060310A7A9B
:10754000B2421DD1C26D641C92782406240E12072B
:10755000920F06D10121019100784007400F06905B
:1075600009E031224A7202780100143110231A43D3
:10757000027000880884059800223900FFF733FD67
:10758000049844730498C07B4006800F04D004988C
:107590000499807B001988730198012805D1396806
:1075A000069A0598330016F084FE03981AF05CFCE6
:1075B000C7E506980006000E16F37EFD16F38DFD56
:1075C0000600ECE7FEB5040004F0F9FA4A0D8D6CF4
:1075D000010000008C73000000040000AC79F3B1DE
:1075E00007006069029020890025061902981DF0A5
:1075F00074FE0C3001900120012F009010D00099F2
:10760000200004F016FB01280AD141492069884274
:1076100001D1032F04D03C498868401C01258860B3
:1076200039480078002821D0374F01247F1D387851
:1076300000280ED1009804F0B0FAB91E09788842EB
:1076400004D301203C70FFF7C1FB0FE0387800281D
:107650000CD0F06D8079C00708D101986030817C32
:10766000002903D184740298FFF784FD2800FEBD31
:1076700042695368002B03D15060416988607047AC
:10768000002907D1186141694A68C260002202617D
:1076900048607047CA68002A01D0106101E04A6959
:1076A0009060CA68C2600161C860704701004969A2
:1076B0000020496800290BD003E00800C9680029B0
:1076C00006D08A681389D218D26DD2781207F4D402
:1076D000704702000020002A08D0012A06D0022AA2
:1076E00001D0032A07D18A4205D303E08A4201D0A0
:1076F000012900D10120704770B50E0040690025B6
:107700004468002C16D009E0A0F500C0E6F700C0E0
:10771000640400042500E468002C0BD0A0680189F3
:10772000405C4007400F16F3D1FC3100FFF7D1FF5A
:107730000128EFD0280070BD03B50820C8406B4673
:107740001978084000D001200CBD70B500241AF053
:1077500091FB0500654804F395F9002805D0040065
:10776000010062480C3004F3B7F928001AF086FBD8
:10777000200070BDF7B584B005000F00FFF7E5FFEE
:10778000040001D10120E6E41AF074FB0026029007
:10779000E660A76026613889C719287A03280AD1CC
:1077A000687A032807D17120C000281860618068BA
:1077B000002101913FE0F86D8079C0070BD02800CF
:1077C0001DF064FD332109014018002160618068CB
:1077D000012601912FE02800FFF760FB0390FF20B6
:1077E0005130405B019038784007400F16F36EFC33
:1077F00006000B20800128184068012816D1039F3D
:1078000031006037787C0090FFF796FF00280DD09C
:10781000039831005C3060612000FFF76DFF797CD8
:107820000126C943090706D0002604E00398012673
:107830000830606180680699002902D02000FFF7B7
:1078400035FF01002000FFF713FF60690168491C44
:10785000012E016004D101990122280020F0AAE83C
:1078600002981AF00BFB002075E4002810B507D031
:107870001DF033FD002803D00C30007D012800D01E
:10788000002010BDFEB505001DF027FD04001AF014
:10789000F1FA0600287A032809D1280015F0EAFF3A
:1078A000002804D130001AF0E9FA0120FEBD606919
:1078B000002806D02100002214312800FFF79DFB8C
:1078C0000FE000206B460290597A02221143597250
:1078D0000122009202000190029928000023FAF789
:1078E000DFFA30001AF0CAFA0020FEBD383401C0B9
:1078F000FC487047007A022803D0032804D1FA48D4
:107900007047F9481C38704700207047FEB50400E6
:1079100000200D0002901DF0C9FC06002868270019
:1079200025002837C035102852D025DC2100E83149
:107930000D2849D006DC801C71D001286FD12100B0
:1079400010313DE0260080360E2826D00F2866D163
:10795000012068622068B84261D1A87F00285ED10A
:107960002000743000F36AF8706A002801D1012009
:1079700030622100403123E0112829D0122809D09B
:10798000212801D022284AD10100D848002203F33F
:10799000D7FF44E00120287741E0080000F34EF8CB
:1079A0002068B8423BD10120D149286200200860FC
:1079B000F06A012833D1B06A012830D12100343176
:1079C000200003F3DCFF2AE0080000F337F826E08C
:1079D0002068B84201D101200290687FF82CE9911B
:1079E000010000008877000000040000FFA320DDF4
:1079F00002281ED2686A00281BD1A87F002818D14F
:107A0000FAF77DFB002814D0002E12D0F068C004D5
:107A10000FD5300016F008FC15220021019202005B
:107A20000091029930000023FAF749F9687F401C61
:107A300068770020FEBD70B50400080009682200C8
:107A400023001032803323294AD015DC891C1FD033
:107A50002500C03501291DD0032934D0142918D19F
:107A60000120A87700201DF02BFC002810D0012158
:107A700049021FF0E2EF0BE024292AD0252903D088
:107A8000262901D0272904D19D48002203F362FF53
:107A9000002070BDF9F70CFF012003F0CCFA0120A3
:107AA00003F0CCFA9748002404602000FAF7DFFACC
:107AB000287F002803D0122003F003F82C77002041
:107AC00003F01EFAE4E7206F1FF0BAEF21001C312B
:107AD00002E0210064319A63200003F35AFFD7E7E4
:107AE000210058319A63F7E710B5086FFFF70CFFD4
:107AF0000020C0310861132002F0E3FF10BDF8B58B
:107B00007D4DFFF701FF87691AF0BEF92C000600D2
:107B1000C0342069002803D004F3CBF90020206191
:107B200000222B0000927848D0333A00290004F359
:107B30005DF930001AF0ACF9F8BDF0B50800C030BE
:107B400087B00690086F0E0080360C000590FFF796
:107B5000DBFE05000AF382F90490326C736C0F00AF
:107B6000121A8B4106D2326C0498736C3900801A59
:107B7000994106E0306C716C049AC043C943801887
:107B8000794102902869029A0E0000273300121AE8
:107B9000BB4112D22869029A3900801A0022B141F1
:107BA0000092230002005948D433210004F31EF947
:107BB00006990120087607B0F0BD06984761077660
:107BC00028880128F7D10598FFF799FFF3E7FEB55C
:107BD000494EFFF799FE370004008037386B0128C3
:107BE00026D020883500C035012806D12869002814
:107BF00003D004F35EF9002129611AF045F90190E0
:107C00000AF32CF9796438646869002808D10022E5
:107C1000330000923D482269D433310004F3E6F882
:107C20000120287601981AF033F9082002F049FF64
:107C3000FEBD70B504007430FFF20AFF2000E8308A
:107C4000FFF206FFC034206904F333F900252561F3
:107C5000606904F32EF9656170BDF3B587B0060065
:107C6000006F0390FFF750FE029000201DF028FBEC
:107C70000700089831000368300028314030059132
:107C80003500C0313400069034308035C034092BC3
:107C900004917ED009DC9B1C15F330EA0B2B488045
:107CA0008064C9D4A1A4B7FE800031001C31232B0D
:107CB00070D02DDC0A2B6ED00B2B6DD0122B6CD01C
:107CC0001C2B6BD1606904F3F4F8002767612776F9
:107CD000206904F3EEF82761E86A012807D13168CA
:107CE0000698814203D10599300003F352FE01202A
:107CF0002863002009B0F0BDA0480004EC4900044E
:107D0000084A000418F700C081780000D37800000A
:107D1000242B76D0252B03D0262B01D0272BD0D196
:107D200000221900FF4803F315FEE2E7002003F0EC
:107D300085F9002003F07FF9FB4901200027086046
:107D4000A777207F002803D0122002F0BAFE277701
:107D500001202862F549FF20F13048630398FFF7BE
:107D600036FFCCE0FDF756F8FDF7F4FA686A002814
:107D700001D101202862300000F086FD3000FFF7BD
:107D800058FF03981FF05CEE002F22D0F868C00463
:107D900005E071E06CE082E092E059E0B1E018D5D6
:107DA000380016F041FA1522002101920200380035
:107DB0000B000091F9F783FF002060620498FFF246
:107DC00047FE049800226421FFF2F4FD0498FFF2BC
:107DD000E1FD31001031300003F3DBFD89E70120C4
:107DE00068628CE00298807800280BD0849EB74BA4
:107DF00001000000847B0000000400000BCC5569EA
:107E00000298008801289AD1207E002897D10398F3
:107E1000FFF77FFE77E731E00020607673E701200F
:107E2000002F60760DD05920039BC0003918062220
:107E3000181819F057FD002803D1C0490868401CE4
:107E4000086002980088012863D1207E002860D154
:107E50000398FFF75EFE5CE001202862300000F02E
:107E60001DFD56E00120A07700201DF033FA002808
:107E7000BED0012149021FF0EAED44E7A9633100B9
:107E80006431B2E7A96331005831AEE70121E962FC
:107E9000FFF2E8FDA86A0128AAD13168059881425D
:107EA000A6D1206A0128A3D1310000E003E03431DB
:107EB0009BE700212963E96A002907D1089909682D
:107EC000082901D1FFF2CEFD01202862012003F034
:107ED00021F81EE0002F1CD0F868C00419D50398C3
:107EE000FFF77FFE380016F0A9F915220021019254
:107EF000020038000B000091F9F7EBFE0498FFF246
:107F0000B1FD049800226421FFF25EFD0498FFF2A7
:107F10004BFD069969E70898F6E6F7B586B006982E
:107F2000FFF7FCFC059006981DF0C4F9FF210490B2
:107F3000069800242D31FEF764FA050059D02889EF
:107F4000702146191C202C182881200014F360EFA2
:107F500006980BF02CFEA070E068A1784009400163
:107F6000084310210843E060152000020390270019
:107F7000E66508986037787206995920C00009189C
:107F8000009101916F4B04220221300008F348FC5C
:107F9000F07802210843F07007983071000A707180
:107FA0000898142827D10598008802280AD10C20A7
:107FB0003872039A069821000BF015FD28000BF08B
:107FC000CDFC10E00498406A012804D006981DF00A
:107FD0005FFA002802D0002016F39DF8387203994A
:107FE00028000BF047FD040003D10021280019F000
:107FF00045FF200088E60720F0E7F0B51FB48CB0FD
:10800000040000202600BC360A901DF063F9002809
:108010007ED0C168FF34CA040B218901641C002A88
:1080200076DA40180B9040690F99403080898002C1
:108030000290C517A2690E98E369801A994108D386
:10804000A2690E98E3690F99801A99410F00069072
:1080500008E00E9AA0690F9B801AE169C04399411C
:10806000CF430690069A206A616A8018794105918B
:108070000490029A06982B00390014F30CEC0B992B
:1080800049694031897B0F0015F376EBA06A441AE9
:10809000002C00DC3C19029A059904982B0014F37B
:1080A000FAEB1F000092029A2000E1172B0015F353
:1080B00020E9009A801A08902348B94100780C0002
:1080C000002814D0870205208002874200D90700CB
:1080D000089A0021B81AA14107D2089A0021D01BA2
:1080E00023008B411C00089001E0002408940B98A9
:1080F0007D2740693F014030827B0298290015F3BB
:1081000004E8089A05000021B81AA1412CD200E029
:108110002CE0089AE81B00252300121AAB4123D259
:10812000089A2300D01B040002003068AB41121AE9
:10813000AB411BD2290009E0084A000418F700C02F
:1081400000A60080F87A0200DDF700C034600E9AC5
:108150000F9BA018169A594103C2FF49FF4A0968AC
:1081600030688918884201D801200A900A9811B015
:10817000CBE5F0B507001FB482B0006FF84E019058
:10818000B06900258402059904982B00220014F39D
:1081900082EB2900766BA51A99413C00FA368034AF
:1081A000B54205D9E06B8019A84201D9A81BE0634C
:1081B000E06B049A059B80180C9A0021594103C278
:1081C000206B01283FD0E06B8119A9423DD83C00CB
:1081D000C034617E012938D1DF49E04A0968891835
:1081E000884232D30198007A05F0C6FB00282CD1D2
:1081F000207E002829D12069002826D18B3852B949
:1082000001000000807F0000000400005816860571
:108210001AF00AFD002822D11AF006FD00281ED10E
:10822000D54800220068462103F345FA002816D1FC
:10823000FDF71FF9002812D00C9A0092059B049AB2
:108240003800FFF7E4FE002809D1F9F76CFF002899
:1082500005D01FF00EEC002801D10120BFE4002062
:10826000BDE4F3B58DB00600006F07901DF02CF84B
:108270000798FFF75DFB070000201DF035F806901A
:108280000E983100006834310B910C310A91343171
:108290000991743135003400C035803412280891BA
:1082A0007ED047DC801C7CD001287BD109F3EAFD1D
:1082B00004900020059102900390A062A064E06405
:1082C000286268626877A8770120F9F7E4FEF86809
:1082D000E0631CF036FB002838D002AA0092059B10
:1082E000049A3000FFF74FFF00282FD0069800288F
:1082F0002ED00698C068C0042AD5A048006800287F
:1083000026D0069815F0A4FF152200210192020044
:108310000091069801210023F9F7E5FC0898FFF287
:10832000ABFB089800226421FFF258FB0898FFF28B
:1083300045FB0FE01E2856D01F2874D10998FFF284
:108340009BFB606A002801D1012020620A9946E067
:1083500001202862606A012813D100206062012197
:10836000E062306F49031FF07CEB0998FFF284FB59
:108370007D21099800220901FFF230FB0998FFF2E4
:108380001DFB206B00281BD13888022818D0786884
:10839000C00715D07A49E06B884211D8079802E0EF
:1083A00028E01FE03FE0007A03F058FE002807D0E5
:1083B000E06B14220104306F090CFFF7B8FD01E0F7
:1083C0000120A062E06A01282AD1A06A012827D1F1
:1083D000286A012824D10998FFF24EFB1EE03000E4
:1083E00003F3EBFA1CE00120A062E06A012817D138
:1083F000286A11E001270020AF771CF075FF0028E4
:1084000002D079021FF02CEB2F620898FFF234FBA8
:10841000E06A012804D1A06A012801D10B99DEE7A6
:1084200000200FB07BE40E98FBE7F0B50D000600CE
:108430004E49006F096887B0FF315A310904090CB1
:108440000591FFF775FA09F31DFD0F000021029158
:10845000039104902868801C58D03400803401288F
:1084600056D1E16CA06C002359405840084325D0F8
:10847000A26C0498E36C3900801A994108D3A26C6D
:108480000498E36C801A390099410D00009007E0D0
:10849000049AA06CE16C801AC043B941CD430090AE
:1084A000E06B009A00212B00121A8B4104D2E06B82
:1084B000009A801AA94100E00020E063FCF7BEFCAE
:1084C00003F342FD1CF03DFA002816D0206B002873
:1084D00013D102AA0092049A3B003000FFF753FE2A
:1084E00000280AD0012200927D22E36B0599D20078
:1084F00002A8FCF7D8FD002808D103F34EFD0020A8
:10850000310020634031300003F357FA0020A5E624
:108510002800A3E6F8B504000F00066F3000FFF74F
:1085200007FA050000201CF0DFFE3868801C3FD0F1
:10853000012805D0152836D016283BD101202FE080
:108540000020F9F7A8FD200000F0B2F9F9F7C4F90E
:10855000C034207F0027002803D0122002F0C5FA83
:10856000277705480022006869210BE0683C01C0BC
:108570002F08000000A60080B0F500C018F700C06A
:10858000F07F000003F397F8676267772888012877
:1085900005D1207E002802D13000FFF7C4FA052063
:1085A000F9F78EF804E021002831200003F305FAE2
:1085B0000020F8BD3800F8BD10B50B68046F9B1C97
:1085C0001AD0012B13D002008032032B11D0042BC0
:1085D00017D1010010319163516A002901D10121A5
:1085E000116200F065F920001FF03EEA07E001206B
:1085F00003E01C309063F6E7002002F036FD002017
:1086000010BD080010BDF3B585B00700B8397297EA
:10861000010000007C830000000400000E3FE545DF
:10862000002003901CF06AFE050006983A000068DE
:10863000B4323E003C0003218036C0342528049229
:108640006AD008DC801C15D0012814D0232852D011
:1086500024287ED105E0262851D027284FD029286C
:10866000F7D1A07E01282DD1E07E421C0228E276BF
:1086700019D9A17686E03800FFF7F9FA0020A07634
:10868000E076F9F735F9002D70637BD0E868C00417
:1086900078D51BF0A6FD002874D10120F9F705FD5F
:1086A0000120A07604E0002D72D0E868C0046FD5E8
:1086B000280015F0D7FD132200210192020000913D
:1086C000012113E0022863D1E07E421C0228E276F9
:1086D000CFD8002D5CD0E868C00459D5280015F02B
:1086E000C1FD132200210192020000912800002305
:1086F000F9F703FB4CE0A07E0128BAD048E0012046
:1087000002F01CFC00252800A576F9F7CEFC0498A1
:10871000F9F719F925772CE0B16B38001030814258
:1087200021D1A07E03281ED10020F9F7BEFC8C4980
:10873000002008608B490860E0760220002DA076BA
:1087400011D0E868C0040ED5280015F08BFD132267
:1087500000E014E0012101920091020000212800B4
:108760000B00F9F7CAFA0498F9F7EDF8012002F0C6
:10877000E5FBB16B380003F32AF909E002E0069843
:10878000039005E078480722006840211AF046FA75
:1087900003986DE5F8B505000020009008682E00EC
:1087A0002C0000278036C034252820D012DC801C05
:1087B00008D0012822D12800FFF759FA0020F9F744
:1087C00074FCE77668480722006840211AF026FA10
:1087D0000098F8BD26280FD027280FD10020A776B3
:1087E000F9F763FCFCF734FBFCF7D2FD2777B16B9C
:1087F000280003F3ECF8EBE7A776F7E70091E7E74B
:10880000F0B504000E0097B019F05CFB05002000E5
:10881000FFF72DFA210074312C220BA8169114F3C6
:10882000DAEA2100E8312C220F00684614F3D2EA7C
:10883000FF213131200014F300EB2C22380069466F
:1088400014F3C8EA16982C220BA914F3C4EA2000EA
:1088500000F04BF8210010310F00200003F3A7F8BF
:1088600020000121803001623E4A416200211160F6
:10887000DA22876311553D49C1632800266719F044
:1088800025FB17B0F0BD0121018041603749C1606F
:108890008160374901617D21090181614161704732
:1088A000344800B5FFF7EFFF32481C30FFF7EBFF0D
:1088B00000BD0200927800201209042A01D1002292
:1088C0000A70704710B504000120FCF76FFA200011
:1088D0008030016A012907D1002101620121416232
:1088E000206F09031FF0C6E810BD70B50400224ACE
:1088F0000021001D03F35FF82000204A211D1030E5
:1089000003F359F820001C301D4A211D050003F314
:1089100052F820004C301B4A211D060003F34BF88F
:108920002000194A2900283003F345F82000174A8F
:108930002900343003F33FF82000154A2900403065
:1089400003F339F82000134A3100583003F333F8A9
:108950002000114A3100643003F32DF870BD00008F
:1089600014F700C018F700C00CFC00C068420000FB
:10897000400D0300D0490004B9760000CF77000015
:10898000F379000029830000D37F00009B81000061
:108990008582000077830000F1840000FF48808B0F
:1089A0004007800F012800D00020704738B5040030
:1089B000FB480D00406B03F39AFAF9490022343169
:1089C0000092220028000B0003F32EFA38BD10B5E8
:1089D000F34C606B03F38BFA0020606310BDF04929
:1089E000002010B50200C860EE484921006802F37B
:1089F0006CFE10BD70B50400EB4D6888002807D0F0
:108A0000200001F04BFF688821007C31288026E09F
:108A10002000FF304130066BFCF71AFAD0AC1A8BFD
:108A20000100000078870000000400005DE53629A1
:108A3000FCF7B8FCDF490120886100200866F021BE
:108A4000085309F333FAE21DF9325165106501202C
:108A500002F07EFA02F0D0F803200DF0A7FC01210D
:108A600000220903300001F002FF6888210058311C
:108A70002880200002F3B5FF70BD202010B502F061
:108A800048F810BD10B5F9F762FB002822D000208D
:108A90001AF0DEF800281DD11AF0DAF8002819D1F2
:108AA000FBF7FEFC002815D11EF0FAEF002811D1CB
:108AB000C14800220068462102F311FE002809D1B6
:108AC00005F077FA002805D116F07FF8002801D1CB
:108AD000012010BD002010BDB84810B52038408AD4
:108AE000002805D0B248B349406B0969884227D1B4
:108AF000AF4880308069002822D1AF4C0022206826
:108B00001B2102F3ECFD00281AD120680022462127
:108B100002F3E5FD002813D1FBF7C2FC00280FD1BA
:108B20001EF0BEEF00280BD11AF092F8002807D1F2
:108B30001AF08EF8002803D116F047F8002800D06C
:108B40000120002804D1F9F702FB002801D10120FF
:108B500010BD002010BDF8B500252C00954E944F97
:108B6000708997494037884219D2796D386D6140D4
:108B7000084314D009F39AF93A6D7B6D801A994134
:108B80007D27FF0023003A0013F3A2EE768923002D
:108B90003A0013F39EEE801BA14100D3012528006B
:108BA000F8BD30B587B003A904A810F0DFFD0500BB
:108BB00001220221684603F332FA040009D0AC42D4
:108BC00007D2042002F0C4F900980199059104909D
:108BD00003E0052002F0BCF92C006B4698892018B0
:108BE00003F363FA002805D0042002F0B1F9012054
:108BF00007B030BD002200926B4699897D22D200D9
:108C0000230004A8FCF763FAF2E7FEB50D00694EF5
:108C10000968B1660100FF3141312B680C000F6B10
:108C20002034222B49D012DC022B38D008DC9B1CCC
:108C300064D0012B13D0032B60D16148163029E09A
:108C40000120032B2ED0122B58D1207156E0233B4C
:108C500014F37CEA070A0D10101054305400010080
:108C6000343102F3BEFE49E05548133012E0544857
:108C700014300FE03800FEF76DFE01684A6801000D
:108C80004C318A4204D12968002202F38BFE35E080
:108C90004B481530F7F794FB1EF09AEE2EE048484B
:108CA0001730F7E76071022002F052F9F06A401CB9
:108CB000F06223E0306A401C30622078022801D044
:108CC00001281BD16078411C0228617010D2380045
:108CD00015F0D2FA13220021019200912178012986
:108CE00000D00021020038000023F9F710F805E059
:108CF000344807220068402119F09AFF0020FEBD89
:108D000070B50400FF3441340A682500236B012646
:108D10002035012A0ED005DC921C12D0012A15D173
:108D200001200FE0022A03D0282A0FD1AE710BE0F8
:108D3000343001E05830AE71E06118001EF0A8EE4A
:108D400002E0002002F0A5F9002070BD080070BD0F
:108D500070B50400FF304130056BFCF783F8FCF779
:108D600021FB1BF048FA012811D10021280001F055
:108D70008BFD2000FF3025300400FEF291FE002222
:108D800064212000FEF23EFE2000FEF22BFE70BDAC
:108D9000F0B506003500FF350020413585B0039061
:108DA000286B029008682C0020340A2874D00BE04D
:108DB000C84A000400F700C0B0F500C0E83C01C09C
:108DC000FFFF00000CFC00C00DDC801C2FD0012830
:108DD0002BD00B2863D1E9693000643081422CD15B
:108DE0005836EE6129E037003437252828D0262868
:108DF00001D0272853D13000FF302530FEF250FE3D
:108E0000E869B84205D0012102980022090301F067
:108E10002EFDEF61002738002770F9F750F9FCF7B5
:108E200021F8FCF7BFFA27712EE000204B6AC82614
:108E300001000000748B000000040000A98A439D1B
:108E40006070F74807220068402119F0FBFE039884
:108E500005B0F0BDE869B84203D13000FFF782FFEA
:108E60001CE01BF0D2F9002811D1607001202070A5
:108E7000F9F72FF9029815F009FA1322002101924F
:108E800002000091029801210023F8F74AFFD9203F
:108E9000805D002802D0092001F045FE0120A0706D
:108EA000E969300002F3A7FDD1E7FFE70120E07098
:108EB000CDE70391CBE7F3B585B006003500FF356C
:108EC000413500200390286B2A0002900698283232
:108ED0000068140003210127083C222804923DD099
:108EE00030DC09286FD025DC801C40D001286BD1F4
:108EF000002020706070F8F70FFDA8620298C0682B
:108F0000C00434D50298407A032801D001282ED11C
:108F10001BF07BF900282AD10120F9F7DAF8C149C2
:108F200088694969084303D11BF01EFD00281ED043
:108F3000277025E00A2877D02128D8D12078012869
:108F40003ED113E0252871D026283ED027283CD0DA
:108F50002928CCD1B348C269521CC26120780128AB
:108F600018D16078421C0228627009D92170AC487F
:108F700007220068402119F065FE039807B0F0BD94
:108F8000029815F083F9132200210192020000914A
:108F9000012110E00228F0D16078421C02286270A2
:108FA00001D9217059E0029815F070F913220021BF
:108FB00001920200009102980023F8F7B2FEDCE76C
:108FC0000228DAD149E051E05AE03000FF30253084
:108FD000FEF270FD012001F0C5FF01F017FE300028
:108FE0003430E8610020F9F774F806980068262804
:108FF00009D02078032806D1029808F07DFC0028CB
:1090000001D1207125E000202070FBF735FFFCF72F
:10901000D3F90498F8F7ABFC00202071A770E96938
:10902000300002F3E8FCA8E728E0FFE77D490020D4
:1090300048618861207803280FD10020F9F749F8AA
:10904000F9F78FF8002803D104F079FD012804DD39
:109050000020607002202070A5E70498F8F787FCD4
:10906000012001F07FFF01F0D1FDD7E7E969300071
:109070006430814281D15836EE617EE7E7707CE74B
:109080000698039079E710B5664CE41D01F075FC75
:1090900000280CD064480088002808D020780007F9
:1090A00005D1E01FC078002801D1012010BD0020AB
:1090B00010BD10B55B4C5D48E41D006B1CF010FA50
:1090C000002802D02078000703D15648C078002835
:1090D00005D055480088002801D0012010BD00208F
:1090E00010BDF8B50A0001000400FF3110684131DD
:1090F00026000D6BE036102825D02FDC022874D016
:109100001BDC801C40D0E71DF93701283ED0032826
:109110006CD128001EF0C6ECFFF7CBFF002803D16E
:10912000FFF7B1FF002862D0200001F0F5FB04201A
:109130000DF046F921007C316AE00D287ED00F2821
:10914000E6D101203082E868C00479D5308A002851
:1091500076D10021280001F0A1FB15E02300343373
:10916000232877D009DC1128EDD0122876D10121EF
:10917000490228001EF092EC06E0242866D0282838
:109180006CD12948418801800020F8BD2000FF30C3
:109190006130002500908570F8F7BCFB012001F0DC
:1091A0007CFF35823D6500207D65F8F792FF204801
:1091B00005602048C0340580207E002802D0257636
:1091C000FBF7F8F800980079002804D0122001F08D
:1091D000AAFC0098057106200DF0F2F8164800224E
:1091E0000068692102F385FACEE715E036E00D4903
:1091F00001208861022001F0B5FE03200DF0E0F8A7
:109200000020308208F35CFE796521005831386512
:10921000200002F3F0FBB7E728001EF044ECB3E7B0
:109220000CFC00C000F700C0E83C01C0484B000443
:1092300048F800C0D8F700C0B0F500C056DA483290
:1092400001000000708F000000040000FA5090F14F
:1092500000E009E02000FF302530FEF235FCE5E7B4
:10926000CB6121002831DDE7CB6121001C31D9E73A
:109270001000F8BDF8B50400FF3041302500006B48
:10928000FF3561350090086826002F0034363C3FDA
:10929000022839D015DC801C5BD001285DD100206C
:1092A00001F008FF002001F002FF2879002804D017
:1092B000122001F042FC00202871002001F05CFE29
:1092C00045E0122804D0282847D10120A8713EE0AB
:1092D000FBF7DCFDFCF77AF80020F8F704FF380014
:1092E000FEF2F2FB2000F830FEF2EEFBFC4900201B
:1092F0000863FFF78AFB00981EF0DEEB012100985F
:1093000049021EF0D6EB1EE0FBF7C0FDFCF75EF84D
:109310001AF085FF012803D0F148806900280FD199
:109320000098002101F0C4FA3800FEF2CDFB0022C3
:1093300064213800FEF27AFB3800FEF267FB02E09F
:1093400000981EF0BAEB3100200002F35EFB002013
:10935000F8BD012001F0AEFEF9E70800F8BDF8B550
:109360000400080021000268FF3126004131583610
:109370000F2A67D01EDC0B2A64D016DC921C61D049
:10938000012A28D0052A25D1D64D2878FF2807D0D4
:109390000100D5486A460068F8F70CF8FF202870ED
:1093A000E820005D022847D144E00C2A4AD00E2A6A
:1093B00010D147E0232A4BD004DC152A42D01A2AC8
:1093C00008D13FE0242A3FD0292A03D1C44A516A58
:1093D000491C5162F8BD2500FF35C14800276135A1
:1093E000AF708761076147610120F8F77CFEFBF7EA
:1093F0004DFDDA2007532879002803D0122001F010
:109400009CFB2F716879002803D0022001F0B4FD85
:1094100010E0FFF7DAFB002814D1B4480822006EF0
:1094200039001040794008430CD1012001F0A4FD1F
:1094300001F0F6FB310012E00428FBD1A849C86E08
:10944000401CC8660020F8BDCE612100283106E02E
:10945000A34A106F401C1067CE6121001C31200010
:1094600002F3D3FAEEE710B5F9F7F2FC002801D0C9
:10947000F9F716FB10BDFEB50200FF3206004132BF
:10948000106B00900B683400FF34253430000194D9
:109490006430643C3500270002900020E035A0379E
:1094A000142B7ED00FDC924A9B1C127A13F362EECF
:1094B00014CF4A969696D296969696969696E8FEEB
:1094C000FDFCFBFAFA961C2B6CD02CDC152B1AD069
:1094D0008348162B006966D01A2B7ED01B2B7DD1BA
:1094E0007F4D00282DD0FCF71BF9002829D1606A98
:1094F00069698842FAD1608B012822D8E06A002885
:10950000F4D101F04BFB01F0A0FB0028EED1FFF7F6
:10951000CDFA00287ED07648017A00297AD10069F8
:109520000028FBD116E11D2B75D034005834232BB5
:1095300072D0242B71D0282BD1D1B8713000FFF715
:1095400077FA77E10020B870F8F7EEF9787900281B
:1095500004D0022001F010FD002078713879002835
:1095600004D0122001F0E9FA00203871B8790028FF
:1095700009D00020B8713000FFF75AFA5B488030FC
:1095800000880028DDD10120FBF72EFC0026A683F1
:109590002662666256486E822E8286705548066044
:1095A00002E067E0BDE020E15348068053480660D2
:1095B0005348012700683200462102F3A4F800282E
:1095C00002D1287A022811D14D482E72006800225B
:1095D000692102F398F8002801E018E12CE105D197
:1095E000012100980022090301F055F9FFF73BFF24
:1095F000002800D0092700981EF06AEA002804D04D
:1096000001210098C9061EF054EA3E48016801296C
:109610000BD103E0FFE07CE006E101E106603A489F
:1096200007220068022119F017FB0020F8F75BFD04
:109630003800F8F76DF8608B002801D001F0EAFAE5
:10964000207E002802D02676FAF7BEFE10AEAD26A8
:10965000010000006C930000000400004595B54235
:10966000F2E001F0A5FAEFE0297A0229F8D104002E
:10967000287200980022C90201F017F90120F8F7BA
:1096800051F823480460DFE001F0CEFA0120F8F73A
:1096900049F8D9E01B4D002AE2D1E06A00281BD02E
:1096A0001AF036FF002802D0E868002814D000988D
:1096B000002101F007F904E064E061E056E08FE08A
:1096C00040E00198FEF20AFA019800226421FEF2BD
:1096D000B7F90198FEF2A4F90520F8F723F8054838
:1096E0000169216240696062E06A002818D001F0D7
:1096F0009BFAA9E000F700C09A5C000408FC00C0D7
:10970000683C01C0143D01C048F800C0D8F700C053
:1097100050F800C0B0F500C04CF800C00CFC00C010
:1097200001F099FA90E001212872009800220903C3
:1097300001F0BBF888E00198FEF2D0F9FF48012162
:10974000C16211E0002A7FD10520F7F7EBFFFC484A
:10975000016921624069606201F081FA002873D1D9
:10976000FFF7AEF90028C2D002996AE00198FEF234
:10977000B5F908F3B9FBF21DF9325165106563E0E4
:1097800001202882086811285ED00F2813D1F8F72D
:10979000FCFC002803D00098002101F093F8019808
:1097A000FEF29CF9019800226421FEF249F9019829
:1097B000FEF236F948E0102812D1688A401C0004F5
:1097C000000C6882298A00290AD1032808D2F8F7F8
:1097D000DCFC002804D00098002101F073F833E08D
:1097E000D848C068002802D00120F7F79BFFA08B63
:1097F00001210843A0830198FEF270F924E0D049CA
:109800004A69002A20D000281ED0487901281BD19F
:10981000FFF756F9002817D0FBF78CFF0128A3D1DA
:1098200012E0C749012048710EE004F0E0FB002877
:1098300099D009E031002831D46102E031001C31B7
:10984000D461300002F3EBF80020FEBD0800FEBD3D
:10985000F0B5050000208DB002902800FF304130A7
:109860000C90006B039028000B6858300B900C385C
:109870000A90B430099060300890B34807902800EF
:10988000FF30253006902E002C382C00AB4F0A00FC
:10989000E036C034102B059023D00EDCA8489B1C6A
:1098A000006913F372EC12FC35323232FB32323281
:1098B0003232FAF91E1E1EF8F732A048202BC06A79
:1098C0007ED014DC152BE7D00CDC112B79D0122BB9
:1098D0001BD1A08B4007800F012816D108980121C9
:1098E0000171C7E1162BFCD01A2B0ED1C2E1290061
:1098F0006431232B66D0242B71D0282B70D0292BD8
:1099000003D18F48816A491C816210000DB0F0BDFF
:1099100008998978002930D00898C078002806D0A6
:1099200008990020C8700A2001F011F9A2E1A08B6B
:1099300001210843A0830598FEF2D0F8834D0598D5
:1099400000222900FEF27CF80598FEF269F80899D9
:1099500000208870A18B8907C3D4F862A08B0221F4
:109960000843A08303980022090300F09EFF059896
:10997000FEF2B4F800222900FFE00C9A0021916168
:109980003182718260636E4AA183D16801204003F5
:10999000814202D100201100C8601AF04AFC0490F4
:1099A0000120F8F7AAFB664841698069014318D095
:1099B000049800281DD10398012100F083FF02E0E4
:1099C000F3E088E06CE10698FEF288F80698002241
:1099D0006421FEF235F80698FEF222F80DE04FE120
:1099E0004AE1FFF7D6F8002803D00C9801218161E5
:1099F000E1E7A08B01210843A0831AF089FD00282C
:109A000002D00120029033E0307A022801D10B9974
:109A100055E14F48002200684A2101F37EFE0028EC
:109A200005D147480121C0680903884220D1A08B95
:109A3000C00706D10798408A00281DD1F86A00287F
:109A40001AD10020F862A08B02210843A08303985A
:109A50000022090300F029FF0598FEF21128C51223
:109A6000010000006897000000040000164F662EF9
:109A70003FF83B4905980022FDF2ECFF0598FDF206
:109A8000D9FF03E0A08B06210843A083A08B072801
:109A900020D118F049FA0400029800280AD0F8F7FB
:109AA0007EFB00280FD10AE0A1E03FE0C5E0B2E074
:109AB00013E110E00398FFF737F8002803D02000E7
:109AC00018F036FADCE00A99280001F3B2FF200012
:109AD00018F02EFAD8E00020F8620598FEF208F897
:109AE0001C48406E02F335FACEE0A18BCA07F1D1D3
:109AF0004907890F01290AD0002808D10398FFF7E8
:109B000013F8002803D00698FDF2F2FFB8E0708A3F
:109B1000401C0004000C7082318A002906D1032801
:109B200004D20398012100F0D7FEADE00698FDF2C3
:109B3000DFFF08F3E3F9099A51651065A08BC107AF
:109B4000C8D1012108430728A0836DD0F86A0BE033
:109B5000484B000400F700C0143D01C0C83C01C0E0
:109B6000B80B0000B0F500C0002817D0F948416BD1
:109B7000F9480069814229D000220092F74A17E093
:109B8000200018F0D5F9F4490020886178E00598A4
:109B9000FDF260FF0598FDF24DFF75E00798408AE1
:109BA000002871D0079900220092098948430200D9
:109BB000E94BEB480021643302F368F964E00028C4
:109BC00004D10398FEF7B0FF002859D10020F862B5
:109BD000A08B02210843A08303980022090300F010
:109BE0006EFE0598FDF284FFDE490022CFE70120DA
:109BF0003082F8F7D4FA002803D00398012100F04E
:109C00006BFE0698FDF274FF069800226421FDF2B7
:109C100021FF0698BFE70598FDF26AFFA08B062199
:109C200008430728A0832FD118F07EF90400039879
:109C3000FEF77AFF0028A3D145E71AF073FC00284D
:109C40000FD0C94800220068462101F370FD0028AA
:109C500007D0C24805F096FC05220021FF20FCF742
:109C600078F80398002100F037FE0698FDF240FFD7
:109C7000069800226421FDF2EDFE0698FDF2DAFE60
:109C8000052001F08DF9CCE6002049E60899012075
:109C90008871C6E6A28B5207920F012A01D00028D4
:109CA00002D00C98C16102E00C990B98C8612900A0
:109CB00028310EE0A28B5207920F012A01D0002812
:109CC00002D00C98C16102E00C990B98C861290080
:109CD0001C31280001F3ADFED6E7317A022900D00D
:109CE0001DE6A18B4907890F0329F9D19A4E00245B
:109CF000B4617169084304D008F300F9099A516509
:109D00001065346174610698FDF2F2FE89E610B5C3
:109D1000FFF7BDFB040008D11AF047FE002804D06D
:109D2000FEF741FF002800D00124200010BD894823
:109D300010B5894C8030006BE41D1BF0EFFB002850
:109D400002D02078000703D18348C078002805D0CE
:109D500086480088002801D0012010BD002010BDD9
:109D600010B57D4CE41D00F026FE00280CD02078B4
:109D7000000709D1E01FC078002805D17B48008882
:109D8000002801D0012010BD002010BD10B5724C7C
:109D9000E41DFFF7ACF9012805D12078C043000786
:109DA00001D0012010BD002010BD70B505006A4C27
:109DB000E41DFFF7EBFF012807D1280012F35DFA3D
:109DC000012181402078014201D0002070BD012096
:109DD00070BD03B56B4660481978C171197901727D
:109DE0000CBD5D4910B54A6B824204D10020486326
:109DF000172000F0B6FE10BD574910B54A6B8242DD
:109E000005D1002008634863032000F0AAFE10BDBE
:109E1000F8B59402002506000F002B00220012F373
:109E200080ED3B00B01AAB41190000196941F8BD43
:109E30007CB504000D0068460FF0FAFB009A019B08
:109E4000121BAB4102D2019900987CBD0020010099
:109E50007CBD10B5F8F79AF900281ED04448016976
:109E60004069814219D1404800220068FD0F0780F7
:109E700001000000649B000000040000E220139A2F
:109E8000082101F35EFC002811D107F0A9FC00288D
:109E90000DD118F00FFF002809D118F00BFF002892
:109EA00005D139480078002801D1012010BD0020DB
:109EB00010BD2E4910B54A6B824203D10020486381
:109EC00000F001F810BD70B5FFF7CDFF01283FD1BC
:109ED0002E48FEF2F2FE04002C480821FEF27CFE21
:109EE00005002A481021FEF277FE281884422FD15F
:109EF0002748FEF2E2FE040025480821FEF26CFE2F
:109F0000050023481021FEF267FE281884421FD165
:109F10002048FEF2D2FE04001E480821FEF25CFE3C
:109F200005001C481021FEF257FE281884420FD16C
:109F30001948FEF2C2FE040017480821FEF24CFE4A
:109F4000050015481021FEF247FE2818844206D06D
:109F5000064C206E002802D1A07900281ED11920BD
:109F600000F009FE70BD0000C84A000400F700C000
:109F700088130000C3870000B80B0000B0F500C0D4
:109F8000E83C01C000A000806004000464040004F8
:109F9000A804000488050004380500040120F7F730
:109FA000D5FBA079401EA071FF49FF20F530FEF7D8
:109FB00039FDD7E710B5FFF7DDFE002808D0F8F728
:109FC000BEF8002804D107F3A3FFF84AD1609060DF
:109FD00010BDF6490120803948717047002210B544
:109FE000F7F770FE012804D107F392FFEF4A5161A1
:109FF000106110BD70B50600EC4C0D006169206960
:10A000000023594058400843ACD008340FCC121AF2
:10A010008B41A7D2F8F793F80028A3D1FFF7AAFE47
:10A0200000289FD000F0D1FF00289BD0E048983C4A
:10A030000088002802D0206E002893D1FBF78EFB09
:10A0400001288FD0002D04D000213000FFF7C6FF7B
:10A0500088E717F073FF0500D64800220068462104
:10A0600001F36FFB002802D00120607002E01B208A
:10A0700000F081FD280017F065FF73E7F0B50500DB
:10A080002E00FF360020413685B00390306B0290E1
:10A0900008682A00340000273432203425281CD0D8
:10A0A0000ADC801CC035002839D0012813D00B28C9
:10A0B0003FD10120687639E0262801D0272838D101
:10A0C000F26100202770F8F72CF8FAF7FDFEFBF795
:10A0D0009BF927711EE0677022E0F069904203D17E
:10A0E0002800FEF767FE15E01AF0B7F8002811D136
:10A0F000012067702070F8F714F8029814F0EEF859
:10A1000013220021019202000091029801210023F4
:10A11000F7F72FFEF169280001F395FC06E06F7652
:10A12000A54807220068402118F0B4FD039805B047
:10A13000F0BD0391FAE7FEB5040025000020FF35CD
:10A1400041350190286B009008682600C03622280F
:10A150006FD008DC801C64D0012818D00B2843D0B5
:10A16000232866D067E02200FF32693227003437A7
:10A17000252802923BD026280DD027280BD029284D
:10A1800059D18A488038C169491CC16151E0F7F74B
:10A19000EBFBA86247E0FAF797FEFBF735F92000E2
:10A1A000FF302530FDF2AEFC062000F003FF20005A
:10A1B000FF3061300021060001700800F7F7B1FFA1
:10A1C0000298F7F7FCFBE869B84205D00121009836
:10A1D0000022090300F07DFB0020307139002000CF
:10A1E000EF6101F330FC1EE00120707621E00020D9
:10A1F00030760298F7F7E3FBE869B84206D1012010
:10A20000F7F78FFF2000FEF7D5FD05E0707E0028F0
:10A2100002D0092000F0AFFCE969200001F313FC33
:10A2200007E000207076644807220068402118F09B
:10A2300031FD0198FEBD0191FBE7F0B50500080076
:10A240002900FF3141310C6B584F0A002B00016887
:10A250007C33803F89B0172907931BD01BDC03296F
:10A2600073D011DC891C37D001292BD004296DD182
:10A270002800FEF79FFD012100220903CCCC24C653
:10A2800001000000609F000000040000B1FAC0F669
:10A29000200000F028FB290034315CE00B29E6D0D7
:10A2A0000C29E4D016295BD1F9E001231B29FBD04E
:10A2B00009DC2C000026803418297DD0192918D0FB
:10A2C0001A294DD1EBE0232977D0242948D10798CA
:10A2D0002900A031D0613EE0FEF7C7FBFEF7BDFBD1
:10A2E000F86D401CF8650A20B871D3E0FBF796F8CA
:10A2F000D5E03548002200681B2101F32CFA002824
:10A3000002D0FAF7EBFD25E0206B012810D1E06ABE
:10A310002B4901280CD10800C3698269A06CE16C4B
:10A32000801A994103D326488661C6612663E66296
:10A33000F86B012802D1FAF7D1FDFE6307F3F2FDB5
:10A34000F967B867A26BE36B801A994102D2386E45
:10A35000002806D00799280001F37FFB9FE085E0E5
:10A360009EE0BA6FA06BFB6FE16B801A9941B865F4
:10A3700017F0EEFD0490206B012832D01449B86D1F
:10A3800088422ED30F4906910988C902814228D3F9
:10A39000FEF7C1FE012803D17969786C884220D18B
:10A3A000FFF708FD002802D03879002819D1B879C4
:10A3B000002816D000220DE065E06EE0979B0000BB
:10A3C00080F700C0E83C01C0B0F500C00CFC00C044
:10A3D0007C150000FC484621006801F3BCF9002808
:10A3E0000DD0049817F0B8FD0F203863B86DF74909
:10A3F0000004000CFEF720FB7E617E644FE0F44811
:10A400000088002809D0F3480221FEF2EFFB002863
:10A4100003D0049817F0A0FD9CE7EF48A26B806B77
:10A42000E36B101AB341029003937E6106207E64B1
:10A4300000F0CAFD01F3D8FD0698002200920088C2
:10A440007D228302E448D20000681E300104090C1A
:10A4500002A8FAF778FE0028049804D117F07CFDD2
:10A4600001F3EBFD76E717F077FD18E0DB4C207881
:10A47000FF28D1D00100DA4805AA0068F6F7C2FF2C
:10A48000FF20207066E7E362386B0F2807D13E6338
:10A49000FEF7E3FAFFF721FD01E0C0352B7600203F
:10A4A00009B0F0BDF0B5050008002900FF314131C9
:10A4B0000A00096B87B0019101682E002C008836D4
:10A4C000803418297ED07EDCC64A022952697BD0AE
:10A4D0007BDC891C7AD0012979D1F7F74DFA280065
:10A4E000FF30BD4E6130817900278036002906D0CB
:10A4F00087712800FEF7C4FA3088002868D0B94870
:10A500000027076147618761476401004771803117
:10A5100087708F60CF600F614F614770077007666B
:10A5200007F300FDAF4A803203C23288FFF784FC94
:10A53000A0630690E163A8480591806F7D23A94937
:10A54000DB00584380310CC939008018069A594104
:10A55000059B801A994108D33088A26B8002E36B77
:10A56000C11780185941E163A0639B487D27806F24
:10A57000FF0047439B48E16B80300CC80491A06BFF
:10A580000390801A9941C01B0023964F9941964928
:10A59000B865884202900DD23088039A8002049BED
:10A5A000C11780185941E163A06330888102029885
:10A5B0000818B8658B488D49806D0004000CFEF7C3
:10A5C0003BFA06E0C7E06FE0CEE060E08CE0C9E077
:10A5D0008EE081487D23C06FDB005843226D636DA0
:10A5E000804F00218018594180373A687B68801A73
:10A5F00099410CD279683868616520650220FAF7C4
:10A600001BFC7848816B491C81630121C16332883E
:10A61000E16BA06BFFF720FCF961B8610026E36BEA
:10A62000A26B714070406364084322640FD0012024
:10A630002063E06A01280AD1BA69A06CFB69E16C69
:10A64000801A994102D3BE61FE612663E66201224F
:10A650000198110300F047F9E035287A022800D16B
:10A660002E7201981DF05CEA002804D001210198A7
:10A67000C9061DF046EAFEF738FD002803D0019810
:10A680000021FFF7B5FC0120F7F76AF8258BE516E6
:10A69000010000005CA3000000040000996B454B22
:10A6A00069E016292FD0172966D1FEF7E0F9524844
:10A6B000016E491C0166416941643FE01B2942D09B
:10A6C00012DC192957D01A2956D14B4CE0780028B2
:10A6D00051D1F7F750F901284DD16071FEF70FFD08
:10A6E000002848D0A0783DE0232941D0242943D137
:10A6F00028007C302900A031D06120E03E4842642F
:10A70000FEF7B5F937E03C4C002A34D02069002828
:10A7100031D0607901282ED1FFF7B9FB01282AD169
:10A72000FBF730F8012826D0E078002823D1FEF787
:10A730009EF9606D401C60656069606431002800AE
:10A7400001F395F917E0FEF7DAFC002813D0FBF7C8
:10A7500019F800280FD12848016900290BD00121E0
:10A76000817040790028E9D105E00120E06202E033
:10A770000120C0352876002007B0F0BD2800FEF784
:10A780002DFB012101980022090300F0B6F82900F1
:10A790003431D4E710B50400080022000968FF3204
:10A7A0004132891C33D0012932D1D820005D0028E4
:10A7B00005D02000883021009431D06124E00E497A
:10A7C000012048720548002200681B2100F3CDFFDC
:10A7D000002817D021007C3116E00000B0F500C041
:10A7E000F19A00001C3E01C0EC040004683C01C06A
:10A7F0009A5C000408FC00C000F700C08813000049
:10A80000DB9A000021007031200001F330F90020B4
:10A8100010BDFEB505000E006A481400418B491CAE
:10A8200041831AF0E0F8002812D0310028000FF020
:10A83000ADFF0921014002221040002C02D0002867
:10A8400005D0002102002800002300F036FAFEBDEA
:10A85000310028000FF09AFF8007F8D500206B46E2
:10A860000290597A0122114359720092020001901C
:10A87000029928000723F7F78BFBFEBD524810B55D
:10A88000006818F026FA4F498C390800343801F373
:10A89000DEF84E4800210161416181611E21418144
:10A8A00010BD48498031086370474948C1788278B3
:10A8B0000902114306D0052902D9464A914201D323
:10A8C000454A1160417802780902114301D03F4A9C
:10A8D0005181417902790902114301D03F4A118027
:10A8E000C17983790A023E491A430A82417B027B7D
:10A8F00008023C4910430880704770B50C00334D86
:10A90000E9688C4201D1002A02D021001DF002E941
:10A91000EC6070BD7CB505000E000800F7F715FC73
:10A920000124280013F0EEFC1022019202003100F5
:10A93000280000230094F7F730FA7CBD70B50400BE
:10A94000FF304130056B052000F048FB1F49002017
:10A950000864086688638864C8640865487119F0EB
:10A9600090FC002803D101212800FFF7D3FF07F353
:10A97000E3FA8034206461646165206504200BF093
:10A980005BFD0121002209032800FFF7B6FF70BD1F
:10A9900010B50E49040000200864086688638864C6
:10A9A000C864086548712000FF304130006B012108
:10A9B000FFF7B0FF07F3C0FA80342064616461657B
:10A9C000206510BDC84A0004B8F700C000F700C0F9
:10A9D0001E3E01C0FDFF0000ACF700C0C0F700C084
:10A9E000E83C01C0CAF700C0032010B502F076FFB2
:10A9F00010BD012010B502F071FF10BD022010B58E
:10AA000002F06CFF10BD10B5FF480088002807D089
:10AA1000FEF78BFB002803D1FEF771FB002801D065
:10AA2000002010BD012010BDF8B50125F74CF84EEF
:10AA30002079F84F00281CD0F06940004008F061F0
:10AA4000380004F0BDFDFAF7C6F9F3490028486163
:10AA50000CD100252571C821E760216105216181A4
:10AA6000C420657160610A20E08002E0207900283E
:10AA70000ED1EA488168020D91438160380004F0EC
:10AA80009FFDF0690121C9070843F061FAF7A3F9B6
:10AA90002800F8BD70B5FF21E14DDB4895A465F5B0
:10AAA0000100000058A7000000040000CAB196276A
:10AAB000F5312980002101800A21841C01821E2099
:10AAC0002070002060700120A0700020E0702171D3
:10AAD00060711DF03EE8A071000AE0710420207250
:10AAE000002060720320A0720020E072288820738A
:10AAF000000A607370BDF8B5FAF7CAF8CE480025B1
:10AB00000580CE48C64C0570CD480580CD4805600F
:10AB1000FF205A30A06304F0AEFECB494000085A33
:10AB200020600126657226627D276563FF00A562AD
:10AB3000E7612663E56205F03EF820713222E68087
:10AB4000C248E2602061C248608166712566C148E2
:10AB500021006566803160610800B34B20384D608C
:10AB6000C38142818581458205810A2205828282D4
:10AB70000D80E767A667FFF78BFEFDF7EBFEFFF79B
:10AB800093FFFFF75BFF0020F8BD10B50400FFF74F
:10AB900035FF002807D002201AF04AFCFCF72AFFF4
:10ABA0000022210002E0AC480022210000F34AFF0D
:10ABB00010BDF1B517F0E0F9994E0700756E346ECF
:10ABC000009A0021012011F3C0EE29432043716651
:10ABD0003066380017F0D4F90023290020005940CE
:10ABE000584008430AD1FFF709FF002800D002208F
:10ABF0001AF01EFC012189061CF096EFF8BD0F200B
:10AC0000D7E78A49CA69904203D10020C86115205C
:10AC1000CFE7704710B5854CE06901F3C2F9002019
:10AC2000E06110BDF8B505007D26F60017F0A4F927
:10AC30000700FFF7EFFF884901200A6858318A4270
:10AC400000D0002000281DD0754C6034002D02D0AB
:10AC5000A589002D00D1658919F08CFC002803D04E
:10AC6000A08A002800D005002089002800D0060016
:10AC7000002200926D4B2A007243784800211C3359
:10AC800001F32CF9380017F07BF9F8BD6448002176
:10AC9000603081750800C5E7644808B5C0690028C0
:10ACA0000AD15F480022614B60300092C2896B4834
:10ACB00000211C3301F312F908BD59486030807D32
:10ACC000B0E75A48C069002800D001207047FFB59E
:10ACD00085B00E0017000025FFF790FE0400FFF777
:10ACE00092FE5D49002806D00A680800583082426A
:10ACF00001D1012000E0002002900020002C0190F2
:10AD000004D155480968343081422AD0FEF717FA39
:10AD1000012803D0FEF7FDF9012824D1002C22D10F
:10AD200017F02AF90400002E08D107F30FF94A4A58
:10AD30008032D16490641820FFF73BFFFFF74EF894
:10AD400001280BD1464D002F01D1002005E0002243
:10AD500005981100F6F7D4FF01202870200017F0A5
:10AD60000FF909B0F0BD02983E49204304914AD042
:10AD70000120002C05D13849E031097A052900D09D
:10AD800000203549029AC031002A039103D003996B
:10AD9000CF6204998E753900314301D10C2532E020
:10ADA0000B2500282FD0002E01D0092000E0002024
:10ADB000002F01D0022100E000210143019119F090
:10ADC000D9FB00281AD02848006812F336E902217E
:10ADD00001430198FAF7D1FF00280FD101981CF028
:10ADE000BCEE00280AD101000500002C019000D122
:10ADF0000C25002C07D10398C16204E0002C02D17D
:10AE00001A490120C8600298002804D0002C02D101
:10AE1000049901980882002DA3D029E01C3E01C0AE
:10AE2000683C01C00021008088130000A0F700C02A
:10AE300080280080CAF700C0D8F700C0C4F700C05F
:10AE4000C8F700C0CCF700C0567B0200204E0000BF
:10AE5000830600000A1A0000084A0004ABA800009C
:10AE600004F700C0C83C01C060F600C0143D01C03A
:10AE70002800FFF79EFE74E770B50500AE48AF49A5
:10AE8000006809680843AE49096808432FD1FEF7F6
:10AE900056F900282BD1FEF73CF9002827D1FEF700
:10AEA0005EFFFFF7B0FDA74C002821D06431471E9C
:10AEB0000100000054AB0000000400003EDEE393FC
:10AEC00019F0A5FD00281DD019F05EFB002803D164
:10AED000FFF7ADFD002815D0A0480068012807D075
:10AEE0009F48008800280DD09E480088002809D07F
:10AEF00004F01FFE608B0121401C608328001CF0C1
:10AF00001EEE70BD608B0022401C60831100280083
:10AF10000123FFF7E6FE70BD0A2054E670B5F9F78D
:10AF20001FFB00280CD019F072FD00284FD0FFF74E
:10AF300074FD00284BD0FDF795FD002847D044E074
:10AF400089488A49C06888423FD019F060FD0028CE
:10AF500035D00025FFF75CFD012400280CD002202D
:10AF60001AF070FAFCF750FD02682100403082426E
:10AF700000D00021080070BDFFF74FFD00281CD055
:10AF80007549754AC03909682000683A914200D075
:10AF9000002000280AD1704A8032D26A002A05D0E7
:10AFA0006D4A20005C3A914200D000206A4A443A3F
:10AFB000914200D0002404432500280070BD6C4855
:10AFC000007A032801D0022801D1002070BD0120A1
:10AFD00070BD654910B50968002909D16049654A05
:10AFE00009881278114303D00A2801D00B2801D117
:10AFF000012010BD022019F02CFD10BD5648203054
:10B00000007A7047544920310A7A022A03D1564AFD
:10B010005268002A00D00872704770B5FFF7FDFC37
:10B020000124002816D0FEF794F84B4DC03D0028AF
:10B0300003D1FEF778F8002804D0474920002A6899
:10B04000443903E044492A68200068398A4200D024
:10B05000002070BDFFF7DCFC00280CD002201AF0A5
:10B06000F1F9FCF7D1FC026821004030824200D0A7
:10B070000021080070BD012070BD1FB500201AF02E
:10B08000E1F900280AD0C068C00407D5FFF7C5FC65
:10B09000002803D0FDF7DFFD04B010BD012202211E
:10B0A00002A801F316F8030008D00420FFF7AAFF56
:10B0B00000220092304A002102A807E00220FFF798
:10B0C000A1FF00221100100013000092FAF759F8B6
:10B0D000E2E725480169C1607047F8B50024070020
:10B0E0000E001AF05FF91E4DF00608D528881021D1
:10B0F00088432880FFF78CFC002800D10124B0058C
:10B10000800F002600280DD03800FCF77FFC29882E
:10B110000322120291432980068019F080FC002846
:10B1200000D00124288831210901084203D10D48AB
:10B130000680124806602000F8BD0B490860704781
:10B1400009494860704708498860704718F700C08F
:10B1500014F700C010F700C0C84A000448F800C047
:10B160001C3E01C0D8F700C0A0F700C0FFFF0000E0
:10B17000143D01C0C4F700C088130000CCF700C024
:10B18000FD480088002802D0FC490120886000208A
:10B190007047F9480188F948002901D001218160F0
:10B1A0000178042901D10521017000207047F3487E
:10B1B0008068704710B50C00022011F00EF80028CE
:10B1C00003D10221080001F0E2FF617A032902D0D5
:10B1D000227A012A0CD1E268D2042ED5002804D0AC
:10B1E000FF304130007A072827D0207A012824D068
:10B1F000022908D1FFF70CFC00281ED0FF2049309F
:10B20000005D072819D1E068C00409D5607A0328D9
:10B2100002D0207A012803D1D7480088C0060CD577
:10B2200016F0B4FED6490A78002A07D101220A7026
:10B2300016F0B0FE0120FFF7C6FC10BD16F0AAFE06
:10B2400010BD10B5CD4C2069002803D000F3B3FE2B
:10B250000020206110BD38B50400FFF7D9FB00289D
:10B2600004D0C54800888005800F0ED0FFF7E9FFA5
:10B270000022C2480092C0887D22D200BF4B4243C8
:10B28000C0482100103300F333FE38BD10B502F082
:10B29000D3FB002805D002F056F9002801D1012087
:10B2A00010BD002010BD38B50D00B44CE1688842D7
:10B2B00028D10020E060FFF7E9FF0028A95BD45EF9
:10B2C0000100000050AF0000000400006D0430FFDA
:10B2D00020782AD002281FD11CF056EC00280FD16C
:10B2E000F9F742F900280BD1AC480022006846214A
:10B2F00000F359FA002803D11CF036EC00280CD0DA
:10B300000022009260887D22D200A14B4243A448D3
:10B3100029000C3300F3F6FD38BD03200121207015
:10B32000490328001CF014EC38BD0028FCD0062886
:10B330000AD1FFF777FB002800D002201AF08CF822
:10B34000012109031CF004EC0720207038BD10B562
:10B350008F4CE068002803D000F337FE0020E06047
:10B3600010BD70B516F01CFE894C05002078002831
:10B3700005D0072803D0FFF7EAFF07202070280038
:10B3800016F012FE70BDF8B5060016F009FE804CEE
:10B3900005002178002919D0012917D0072915D0D7
:10B3A000032913D0042911D005290FD006290DD067
:10B3B000FFF7CDFF0022009260887D22D200424339
:10B3C0002300774831000C3300F39CFD280016F071
:10B3D000EBFDF8BD70B5050016F0E2FD6C4C060003
:10B3E0002078072808D1FFF75BFF002804D002204F
:10B3F00020702800FFF7C7FF300016F0D5FD70BDA4
:10B4000010B516F0CDFD0400FFF7A1FF60490878E4
:10B41000052803D0042801D0032801D1012000E031
:10B4200000200870200016F0BFFD10BD10B5FFF71A
:10B43000FEFA002801D05B4809E0FFF7F3FA002884
:10B4400007D002201AF008F8FCF7E8FA7430FCF292
:10B450008BFB0A20FFF7C1FB10BDF8B5040045695E
:10B460004B4E0020B060FDF728FB484F388800287D
:10B4700003D019F0D3FA002804D03078012801D085
:10B48000052857D1454800220068462100F38BF972
:10B49000002834D1FAF765F8002830D03888012721
:10B4A000002821D0687A032802D0287A012803D105
:10B4B00019F0B4FA002806D0687A022814D119F0DD
:10B4C000B8FA002810D01020F5F7B9FE1020F5F7D3
:10B4D000C2FE0420F5F74EFFF5F75DFF0920FFF7E8
:10B4E0007CFB314807703DE03078052820D12E489C
:10B4F00001210770062089053070280030E0388867
:10B5000000280DD00020FFF791FF1020F5F797FEDF
:10B510001020F5F7A0FE0420F5F72CFFF5F73BFF10
:10B520003078052802D10220307016E0012819D1A8
:10B530000020F9E7002810D007280ED0FFF7B0FE52
:10B5400000280AD0307802280CD1FFF7A9FE002885
:10B5500008D019F063FA002804D0012160690903BA
:10B560001CF0F6EA0020F8BD10B519F062FA0028C8
:10B5700029D1064806490088002819D00B480088C0
:10B58000002815D0012048701DE000001C3E01C0BD
:10B59000C4F700C000FC00C049AE0000B0F500C018
:10B5A0003BAF0000004B0004817D0200E83C01C07D
:10B5B0000878002801D0072805D119F047FA00289B
:10B5C00001D1FFF77DFB002010BD70B501894469F2
:10B5D0000D1828000FF347FF00281DD019F01EFAA0
:10B5E00000280AD01B480078002801D0072804D181
:10B5F0000121890420001CF0ACEAFFF718FA0028AA
:10B6000003D1FFF70FFA002806D019F00AFA002834
:10B6100002D01C20FFF7E1FA28000FF33EFF0028BC
:10B6200005D00D48002200681E2100F3BCF870BD53
:10B630000A480088002805D006484178012901D130
:10B6400002214170704703484178022901D103214A
:10B6500041707047C4F700C0B0F500C01C3E01C087
:10B66000142359430918D031097C0120032900D241
:10B670000020704710B50400007C032801D2401C54
:10B68000207462682260A2686260A16022686068BB
:10B69000131ADB1C062B0DD8431ADB1C062B09D80A
:10B6A0008B1ADB1C062B05D810184018032111F348
:10B6B000F8EC0BE0884201DA030000E00B00934253
:10B6C00001DD100002E0884200DB080040D229883A
:10B6D000010000004CB3000000040000D2C1154C72
:10B6E000E06010BD03000220032210B5411E1400CB
:10B6F0008C402104090C8B4205D3401C0004000C33
:10B700000A28F3D90A2010BD30B5012544689540B8
:10B710000368AC4203DA5918641C12C030BD1C0027
:10B7200014411A1B5118016030BD0A0010B5416860
:10B73000002909D0012393400068994202DA11F3ED
:10B74000BAEC10BD104110BD6120C04310BDF8B56A
:10B7500004001000069A009202000F001D00200055
:10B760001CF058FB060019D0F87E06982968076877
:10B770002000FF3003220D30FFF7C6FF2000FF300E
:10B78000032239001530FFF7BFFFFF203D30025B79
:10B790002000FF3039002D30FFF7B6FF3000F8BD34
:10B7A0007FB503AA040002AB009201AA1CF032FB91
:10B7B000010020000122C0304260002200290273F3
:10B7C00032D025000398A035E880029803220104B6
:10B7D0000914A9800198288128006C30FFF794FF94
:10B7E00006212800695E03227430FFF78DFFFF20D9
:10B7F0003F30025B06212800695E9430FFF784FF2A
:10B8000018F0D6FE002809D0FF48006811F332EC8A
:10B8100001000420FAF7CFFA002805D020001CF020
:10B82000C2E920001CF0C2E97FBD70B504001DD044
:10B83000072008560B268E572500E4350100280006
:10B84000FFF722FF287C002801D0E96801E0612190
:10B85000C9432000FF3003221D30FFF755FF2000B1
:10B86000FF30032231002530FFF74EFF70BD03216A
:10B87000FF300D3059E70321FF30153055E7FF2128
:10B880003D31095AFF302D304FE7FF213F31095A32
:10B89000FF30353049E770B50500FFF7F6FF0400CB
:10B8A0002800FFF7E4FF201A70BD70B50500FFF710
:10B8B000E2FF04002800FFF7DAFF201A70BD70B520
:10B8C0000500FFF7DCFF04002800FFF7D0FF201A77
:10B8D00070BD10B50400E430142111F326EB2000F4
:10B8E000FF3000211D300A0006C00400080003C418
:10B8F00010BD0100A0310022CA816122D2434A81D9
:10B90000FF308A812D3000210A0006C07047612275
:10B910000100D243A03110B58A80CA8000220A817A
:10B92000943113000CC100F0B5F910BD70B50400DE
:10B9300016F040FB05002000D030142111F3F4EA8A
:10B94000200000F0B2F9280016F038FB70BD70B589
:10B95000050016F02FFB04002800FFF7E7FF280082
:10B96000FFF7D5FF2800FFF7C4FF200016F026FBE5
:10B9700070BD10B50400FF3003212130C1838183E5
:10B980002000FFF7A6FF2000FF3000212D300A0025
:10B9900006C006C0200000F088F910BD0100FF318C
:10B9A000491C89690120012900DA0020704770B51F
:10B9B0000400FF30401C026AC1690261C160826AF2
:10B9C000416A826141612000FF3003212530FFF789
:10B9D000ACFE2500A035E8802800002194300A0044
:10B9E00006C0200000F056F9280003217C30FFF744
:10B9F0009CFEA880E988081A28812000FFF769FFCB
:10BA000070BD002907D0017A002904D00121C0307F
:10BA100041600021017370470121C0304160002165
:10BA20000173704703000A000800C03210B51168A6
:10BA3000994204D1002111600AF01CF810BD73482E
:10BA40004168491C416010BD704800787047F0B5EE
:10BA500004000B2080012018476989B0002004A948
:10BA600006901CF074E8607A032831D1E068C004C5
:10BA70002ED53D00FF354135A868002828D0FAF7BB
:10BA800046FD0499884223D118F0D2FF002802D144
:10BA9000A87B00281CD05E4EA86846430AF31EF916
:10BAA000FD1DF9352A6C6B6C801A99410023321AFE
:10BAB0008B410DD201210022009100210192072229
:10BAC00020000B00F6F791F90AF308F9696428647D
:10BAD0000DF0CFFD2500C03505906868F806DFCD74
:10BAE0000100000048B7000000040000811BC620D0
:10BAF000002805D000204A496860A860487059E0D5
:10BB0000A86826008036002809D10120A8600AF321
:10BB1000EFF8F1634249B0630020487048E020002C
:10BB20001CF002E800283BD0FAF7FBFC049988429D
:10BB300036D10AF3DDF8B26BF36B801A994105999F
:10BB400011F3B0EE0006000E35490690012848704A
:10BB50002ED906A80DF0D1FE6B461A7E00210A20D0
:10BB60000EF082FD6020005D00280BD06B46197E30
:10BB7000884207D82C490122087810430870200019
:10BB80001CF022E85F206B46005D197E88420FD8CA
:10BB900000200100287307222000FAF7C7FD07E004
:10BBA0000598B26BF36B002180185941F163B063C3
:10BBB0000120A8601A486B46197EFF374137017093
:10BBC000B87B002853D0FAF7ACFC049988424ED1D8
:10BBD0000AF38EF802900391E17A062000F0FEFA53
:10BBE00043E0F868C0043BD5032000023E18F08B08
:10BBF000002835D0306A00282FD1F16AB06A0023BE
:10BC000059405840084328D0F08B064B58430890C1
:10BC1000C3170793F36AB26A039907E060F600C09E
:10BC2000DCF700C040420F0070F600C00298801A96
:10BC3000089A9941079B121A8B4111D20121412286
:10BC4000009100210192072238000B00F6F7D7F887
:10BC500003990298F162B06202E000203062F7E7D7
:10BC6000E27A0621380001F056FC0700B9D1002223
:10BC700000921848059A2B00210000F357F909B0EB
:10BC8000F0BD10B50400007A01280CD02000C030AF
:10BC9000006800F3AEF920001821B83011F34EE926
:10BCA0002000FFF7DEFE10BDFF213F3100B50A5A2C
:10BCB000A623195EFF303530FFF730FD00BD0100CF
:10BCC000FF3100220D3113000CC10800110006C025
:10BCD0007047000091B60000914200D91100484B16
:10BCE00080001A501A00103A11500120704745493F
:10BCF000800008587047444810B5FDF237F84049B5
:10BD00001439086000200A1D8300D3580C68401CB9
:10BD1000E31A0006000E04280B60F5D3086800281B
:10BD200000DAFEE710BD3749C07B1031085C704770
:10BD3000F0B5060096469C46324A314BB6009759FC
:10BD40009B590024012025009F4213D28B00D1581B
:10BD50001A002B4B0020103B9A58914200D9012425
:10BD600099598F4206D32649012514390968214380
:10BD700000D101207146002900D00C6061460029E5
:10BD800000D00D60F0BDFEB5050000200E00019052
:10BD900000901D492869884201D00120FEBD194844
:10BDA000E97B1030475CB74201D10020FEBD16F0A0
:10BDB0000BF902903900300001AA6B46FFF7B8FF7B
:10BDC000040017D10F4AB8001158002900D1FEE72E
:10BDD000491E115000990198411A09481438036806
:10BDE000C91801600748E97B10304654B00011586B
:10BDF000491C1150029816F0EBF82000FEBD00001F
:10BE0000C0050004705000046404000470B50024F0
:10BE1000B34D04E040194068F4F7A2FB641CE00055
:10BE200029580029F6D170BDAE4821214901816011
:10BE300081680122920511438160704770B500242A
:10BE4000A74D04E040194068F4F796FB641CE0003D
:10BE500029580029F6D170BD70B5040005F3CCFF58
:10BE600006F365FC142003F0DDFB002C01D1F9F78B
:10BE7000B4FB16F0A9F8050007F018FDF9F7DDFB93
:10BE800006F346FC002C01D105F3B0FF06F349FC94
:10BE9000280016F09DF870BD914810B53C38826BB3
:10BEA000521C8263416812200EF0DEFB16F08CF803
:10BEB000040000F0C4F8200016F08AF810BD042039
:10BEC00010B5FFF29EF8012010BD70B50220FFF7FB
:10BED000B7F8F9F7EFF8FEF7BEFD002401260028B9
:10BEE00019D018F0B2FD002815D018F0A2914925FC
:10BEF0000100000044BB0000000400007574B3940E
:10BF00006BFB002803D1FEF7BAFD00280DD018F016
:10BF1000AEFD002809D118F05FFB76493C390028B6
:10BF200000D08C62754804800E6307F004FB7448EF
:10BF3000002200681921FFF254FC18F04DFB002884
:10BF40000CD0704D2E72F9F739FF6F480188002927
:10BF500002D004802C7201E0F9F73AFF6B486C497B
:10BF6000006888420BD1FEF77BFD002800D002203C
:10BF700019F090FA012109031BF008EE08E0FEF722
:10BF80006FFD002801D0042000E00320FEF743FEEF
:10BF900000F0A5F870BDF8B5002019F07BFA002874
:10BFA00002D001200DF06BFAF9F78EF8002019F09D
:10BFB00071FA002802D002200DF061FAFEF755FD5B
:10BFC0004C4C544E00253C3C00282FD018F047FD27
:10BFD00000282BD018F000FB002803D1FEF74FFDFE
:10BFE000002823D018F043FD00281FD1206B434FB9
:10BFF00000280DD119F04EFA1BF0D8ED002807D11A
:10C000003F48002200681B21FFF2EBFB002802D012
:10C01000A5623D8015E030880125002800D03D80D4
:10C0200018F0DAFA002811D0A5620FE018F01FFD11
:10C03000002806D0206B002803D025633088002814
:10C0400001D0032000E00420FEF7E5FD00F047F8F2
:10C05000F8BDFEB5304C60693025284360612F4E35
:10C06000706A02273843706206F0CEFD01902C49B9
:10C070002A4A0020C03A0870D068D10D8843D060A9
:10C0800028480078C00701D1F9F785F802A8FAF727
:10C0900071F906F0B0FFFAF7EDF90090FAF760F9E0
:10C0A000009B002202A9FAF7EBF911F0EBFF06F36F
:10C0B0003FFF019806F0C1FD05F0EFFBF6F781FBAD
:10C0C000F5F7FCFD17480078C00701D1F9F7F8F93A
:10C0D0006069A8436061706AB8437062FEBD10B5C4
:10C0E000F8F7E5FF104807220068012116F022FE4C
:10C0F00010BD00005CF800C000300080D8F700C020
:10C10000B0F500C0143D01C0C8F700C0ACF700C0D6
:10C11000FFFF00001C3E01C0C0A20080C0A800803C
:10C12000D00300043A5C0004302601C0F84B10B57F
:10C130005C68002C02D1586002604160002800D188
:10C14000586010BD70B504000E00002515F046FFC4
:10C15000EF4903E0A14201D14C680DE04968002994
:10C16000F8D10DE0E168490505D5072E02D0217A06
:10C17000B14200D125006468002C01D0002DF1D01F
:10C1800015F030FF280070BDF8B50025070015F048
:10C1900025FF0090380019F03DF904000926B6018A
:10C1A0000FE0200019F026F9002805D08019C06999
:10C1B000002801D0012506E039002000FFF7C2FF6A
:10C1C0000400002CEDD1009815F00CFF2800F8BDFC
:10C1D000D04880687047CF498868401C88607047A5
:10C1E000CC498868401E88607047CA48C06870475C
:10C1F00070B505000E0015F0F1FEC5494C680AE067
:10C20000217AA94206D1E17AB14203D115F0EAFEC2
:10C21000200070BD6468002CF2D115F0E3FE002010
:10C2200070BD70B504000500803420690026002828
:10C2300034D1A069002831D1287A03280FD1E87AB7
:10C2400001280CD100210320FFF7D2FF8030816943
:10C25000A161416961610069206145611FE0AE48EB
:10C260000022642111F360FB0028A06107D01C218B
:10C270000181A06901003031616101218173A7480A
:10C280000022642111F350FB0028206106D0456193
:10C290002069002802D0A069002800D101263000C2
:10C2A00070BD70B505002C008034A1690120002903
:10C2B00014D02269002A11D000268E73A06911F3D0
:10C2C00009FBA6616661287A032802D1E87A012871
:10C2D00002D0206911F3FEFA0020266170BDFEB580
:10C2E0000400012615F07AFE250080350190287A99
:10C2F000FF282BD1874F002039780123EF0D272805
:10C300000100000040BF00000004000026AE60F8FD
:10C310001A0082400A4225D183401943287239709D
:10C320008100C9194C61810182480E1840213000FA
:10C3300010F318EEEE60207A012811D0B8680128B9
:10C3400001D107F049FE0B208001201841694031DE
:10C350008A7B0092817B1300287A012207F066FE17
:10C36000002604E0401C0006000E0328D0D30198EC
:10C3700015F042FE3000FEBDFEB505000020029023
:10C3800015F036FE002D019004D08820405D040099
:10C39000FF2800D1FEE7297A634F012929D00B211C
:10C3A000890169184A694032927B00921300897BA7
:10C3B000002207F03BFEB868A04215D011E0A000B3
:10C3C000C019856945615B48A201803516182C7239
:10C3D000E9684022300010F394ED641C2406240E1A
:10C3E000EE60B868A042EAD8B868002801D107F02A
:10C3F0000CFE01213878A1408843A100387000204C
:10C40000C9194861019815F0F7FD0298FEBD0200B8
:10C41000117A0020012905D0022903D0032901D077
:10C42000042901D1100064E7704710B50400007AB8
:10C43000012805D0022803D0032801D0042807D101
:10C440002000FFF799FF00208034E060FF20207279
:10C45000002010BD030010B501D1012010BD18004F
:10C4600018F0F9FF0400D868400507D56068002877
:10C4700004D00EF033FC002060602060002010BD6E
:10C4800070B50400C0680025400523D5207A032834
:10C4900001D0042803D12000FFF70DFF050059202B
:10C4A000C0002118801D241822780120FF2A0ED0F8
:10C4B0000020030007F03AFD002808D11A4B267827
:10C4C00001225968B24091435960FF21217001282F
:10C4D00000D10125280070BD70B50500C068400579
:10C4E00030D5280018F0B7FF04004068002839D183
:10C4F000287A03280FD1E87A01280CD100210320E3
:10C50000FFF780FE0B2189014018C16A6160806AD3
:10C510002060606802E00EF0D9FB606000280BD15B
:10C52000012070BDD0050004905000047405000483
:10C53000600500042C1902C00830206028001BF0A0
:10C540005CEB0FE0E97AA87A18F095FF0400280068
:10C5500018F081FF0300200018F07DFF416859604A
:10C56000006818600020DCE770B50500C068002492
:10C57000400511D5280001F0BBFD0400287A0328EE
:10C5800001D0042806D12800FFF755FE012801D16B
:10C5900001240AE0002C08D1287A022801D00328BF
:10C5A00003D12800FFF798FF04002000B9E710B579
:10C5B000040040213E3010F300ED200006217E30C3
:10C5C00010F3FAECE068012109038843E060FF20E2
:10C5D000002149300155FE2138200155200008F086
:10C5E000C4F910BD01000020002905D00A7A012AF3
:10C5F00002D1172040010818704770B50400FFF7FA
:10C60000F1FF05000920800120180EF389FA2000AF
:10C6100008F04BFA2000FF3006214A3010F3CCEC32
:10C62000002068757DE73F2210B5125CD2070ED05E
:10C630000B229201841800290AD0007A012806D121
:10C640001BF0DEEA012201002000F9F7E4FE10BD34
:10C650000122FF21F8E710B504000021FFF7E3FFF6
:10C660002000FFF7CAFF2000FFF7A1FF10BD70B543
:10C6700004000D00160015F0BBFCFF4903E0A142C9
:10C6800001D14C680EE049680029F8D10CE0A17A8C
:10C69000A94206D1E17AB14203D115F0ADFC2000E8
:10C6A0003FE76468002CF2D115F0A6FC002038E7C3
:10C6B000F8B504000025C17A807A18F0DCFEE27A31
:10C6C000A17AFFF7D4FF002800D101252000FF3018
:10C6D00006214A3010F370EC0922207A210027004D
:10C6E0009201C031B837A618002808D0012811D00F
:10C6F000022819D0032822D1607A032818D10868AB
:10C70000FFF28BFC1821380010F32CEC99A6DF43C4
:10C71000010000003CC30000000400002457B8EEF4
:10C7200030000EF307FA0FE02000FFF79EFF002D08
:10C7300002D02000FFF7AEFE00250AE02000FFF740
:10C7400093FE01E00228F9D0002D02D02000FFF76F
:10C75000A1FE2800F8BD002802D0017A032901D0EB
:10C76000002070470B2189014018406A704770B55E
:10C77000040018F07AFE200018F050FE0500E06872
:10C78000400503D50920800128184461C048206372
:10C79000C0486063A87F20342076E86F002818D155
:10C7A00003F0A0FD0028E86700D1FEE7040008348C
:10C7B0005421200010F3E0EB0321A171E07901097D
:10C7C0000901E171042148200155A07A410849007E
:10C7D000A172B0E6F8B5040010D0AC4D287803285B
:10C7E00002D1E868A04209D0FEF74EF9002807D030
:10C7F000E868FF304130007A072801D10120F8BDF8
:10C80000237A0126032710F338ED0604171E1B0FA9
:10C81000170F03200FF01DFD23E0002F02D0F86852
:10C82000C00401D4AC602E702878012802D1A86819
:10C83000FEF787F80020F8BD0220AC602870F3E70F
:10C84000607A022808D12000FBF71AF92100FCF7D2
:10C8500077F8EC602F70E7E70328E5D1002018F0A7
:10C86000EDFD0700FEF715F90028DBD0D5E770B520
:10C87000040002206072200018F0F7FD200018F07C
:10C88000CDFD0500E068400511D50920800128187C
:10C890004461E06840050AD57F488068002806D1D9
:10C8A000FEF7F7F8002802D12000FFF793FF784841
:10C8B000206378486063A87F20342076E86F0028E2
:10C8C00018D103F00FFD0028E86700D1FEE704004F
:10C8D00008345421200010F350EB0321A171E079BA
:10C8E00001090901E171042148200155A07A41089C
:10C8F0004900A1721FE610B5040015F083FB0B215F
:10C900008901611849690122CA73617A02290FD12C
:10C91000614BD968491CD960604B8034217A9C6A8C
:10C92000A14205D15C6B8A409443D90D0C435C63F2
:10C9300015F06CFB10BD10B5040015F063FB0B2265
:10C940009201A21852690021D173617A022905D19E
:10C95000514AD168002901D0491ED16015F056FB1B
:10C9600010BD02000B208001101841690020002A30
:10C9700005D0127A002A03D10800FF3051307047E9
:10C98000032AFCD10800FF305530704700210028F1
:10C990000AD0027A002A02D11721490103E0032AB2
:10C9A00002D1DD218900411808007047002800B538
:10C9B0000BD0017A032908D1FFF7CDFE00212922EF
:10C9C000C94352018018C175017600BD70B50400DD
:10C9D0001FD0207A03281CD12000FFF7D7FF0500C5
:10C9E00017D02000E4621BF01AE92000FFF7F2FEE6
:10C9F0002B4820632B4860630B208001201840697E
:10CA000068302860284868602848E86020001BF0EB
:10CA10000AE990E570B50400FFF7B8FF05001BD0E8
:10CA2000032060722000E462FFF7D4FE1C482063FC
:10CA30001C4860630B2080012618706968302860EC
:10CA4000194868601948E86020001BF0ECE870693C
:10CA50000021FF30413081736DE510B504000420E2
:10CA60006072E068400502D52000FFF7B3FE0B219D
:10CA700089010F486118086220001BF0D4E81721D3
:10CA8000002049016118487510BD0000D005000460
:10CA9000316700C0F76600C090500004C0A200805B
:10CAA000F96300C0B36600C0892401C0446102C0BC
:10CAB000604B01C030B5042141720021F94A016385
:10CAC000416313680B22920182185469DD88403457
:10CAD000258254695D894034658254691D7A4034E9
:10CAE000257552695B7A4032537503221202801811
:10CAF00041830A22C183828301628162C16230BDA7
:10CB0000E94A002138B508001170516011618300B5
:10CB1000401C9B180006000E03285961B00C8D675D
:10CB20000100000038C7000000040000778D6B8210
:10CB3000F7D30EF04BF8E24CE34922680092E14A49
:10CB4000E248E34BFCF2D8F8002804D0E148F3F7C0
:10CB5000D7FC1AF0DEEF22680092DF4ADF49E04896
:10CB6000E04BFCF2C9F8002805D0DA48401CF3F786
:10CB7000C7FC1AF0CEEF0EF0ABF80EF081F8DB49EF
:10CB8000D948486008001BF05CE8002038BDFFB5BC
:10CB900081B00D0000260399280018F080FC0700E2
:10CBA00000D101260EF026F8040002D1002005B0C5
:10CBB000F0BD01982072A5720398E0720C98206174
:10CBC000E068012189028843F107490D08430B21E0
:10CBD00089016518E0600020A86161212000C94337
:10CBE000A03001824182FF2028600198052875D07D
:10CBF000002E75D06869002806D120000EF053F889
:10CC00000028686100D1FEE76E690B9830730F2031
:10CC10008002306101212920815505213000C901A0
:10CC20008830611808603000F6F7B6FE69690020A8
:10CC3000FF316131FF36761C48767061B0619E48E5
:10CC4000062201685920C000201810F36EE9FF2069
:10CC500088210855A8732000FFF79AFC012873D09B
:10CC60000A98002806D02000FF300A9906224A3090
:10CC700010F3F0E80520C001002120180181954A39
:10CC80002000FF301B3A4130028042800F22818019
:10CC900082710172FE2238200255E26831200003C1
:10CCA00082430920800120184162C1610162C16292
:10CCB0008162016341630120C0038243200040215F
:10CCC0003E30E26010F38CE9049800280DD020007B
:10CCD000049906227E3010F3BEE80BE014E0FFE773
:10CCE00059200622C0003918AEE7200006217E3008
:10CCF00010F376E9E068C0218843E0602000FEF789
:10CD00006AFE20000BF0F1FBFF200026483006559C
:10CD1000019B10F3BCEA070532111635350D3500BD
:10CD20002000E4621AF084EF2000FFF77DFE27E088
:10CD30002000FFF7C9FE23E02000FFF7A2FD1FE05F
:10CD400002E00398022803D320000DF06AFF2DE7CC
:10CD50000398AF23DB005843654940186862200000
:10CD6000FFF72EFE2000FFF73BFE2000FFF709FD36
:10CD7000604820636048606302E02000FFF777FEB0
:10CD8000686900282ED0E16849052BD505002021CF
:10CD90002C3010F3FCE82B2046552800403064214D
:10CDA0008673818144490968CA8802824A8942821D
:10CDB0000A7A0275497A41750520C0012018006879
:10CDC0008C2110F3E4E828008030C6800179FD2230
:10CDD00049084900114001717821803081631E218A
:10CDE000403081602000E2E6F8B504001700007AC8
:10CDF0000025032801D0217200E00D00002B06D091
:10CE00002000FF30062219004A3010F324E80520E4
:10CE1000C00126182F4A20000021FF301B3A413064
:10CE20003181028042800F22818082710172FE2155
:10CE300038200155E068012109038843E0602000A3
:10CE400040213E3010F3CCE8002F05D02000062210
:10CE500039007E300FF3FEEF2000FEF7BCFD20000E
:10CE60000BF043FB207A00281DD001281FD0032897
:10CE70004DD1002D46D10B208001201841690D2095
:10CE800080016831201841631C4981630721C90171
:10CE90001B4861180860174820631748606320002A
:10CEA0001AF0CAEE33E02000FFF7BEFD2FE02000AD
:10CEB000FFF7DDFD2BE00000F0FB00C09050000408
:10CEC000A8F800C0385000046C0500046005000498
:10CED00080EC01C01A0001004450000480050004E9
:10CEE00074050004E0F801C05DA80100942401C0AD
:10CEF000D85801C0F96300C0B36600C0892401C0DE
:10CF0000446102C0022D02D12000FFF73AFCE06824
:10CF1000400505D53068002802D08C2110F336E892
:10CF20000020F8BD3EB500230C000A6903198355A3
:10CF30000100000034CB00000004000083E21E3634
:10CF40000021009102920191E27AA17A207AFFF702
:10CF500028FE617A4172172149016218127841183E
:10CF60000A70FB490163FB4941633EBD3EB50023A6
:10CF70000C000A690021009102920191E27AA17AE3
:10CF8000207AFFF70EFE617A41723EBDFEB50023A6
:10CF90000D0006000A690021009102920191EA7ACF
:10CFA000A97A0520FFF7FDFD04007ED0687A607243
:10CFB000287A2072200014301AF050EEA069E46242
:10CFC000243060612900200040223E313E300FF3C2
:10CFD0004CEF2900200006227E317E300FF344EF13
:10CFE0002000FF30062231004A300FF33EEF592077
:10CFF000C0002918062220180FF3A0EF2000FF30F0
:10D00000E82159300FF3CCEF286B20632900203141
:10D010008E7E20002030827EF606EF23F60F1A4027
:10D02000360132438276427EF72632404E7E360704
:10D03000F60FF600324342761A404B7EDB06DB0FDA
:10D040001B011A4342762A0080321669130022001F
:10D05000803216619B699361097E0176E068402108
:10D060008843E9684906C90F890108438021E060C7
:10D070008843E9680906C90FC9010843FF21491C13
:10D08000E0608843E968C905C90F09020843042123
:10D09000E0608843E9684907C90F89000843E060F8
:10D0A000E86840070DD4092100E00AE0890168180A
:10D0B000C2696118CA61026A0A62426A4A62C06A47
:10D0C000C8622000FEBD0100FF3170B504004A3186
:10D0D000F6F7F8FB0B20800120184069FF30413043
:10D0E000817B491E0906090E81730CD1E17A00206B
:10D0F000FFF7A6F818F094FA002804D100221100D6
:10D10000200011F085F8092080012518E86A002622
:10D11000002802D003F012F9EE626E62E06804218A
:10D120008843E0600021200005F099F820002E637C
:10D13000FFF781FA2000FFF758FA17204001201866
:10D140000CF06FFF79E4F3B583B00D000B27BF013E
:10D15000CE1970690A69017B00206B4607C32B005A
:10D16000EA7AA97A7E330620FFF71BFD040030D04F
:10D1700020003930017810221143CA064908D20F25
:10D18000490011430170FF300399062211300FF35B
:10D190006CEE7069E11948610920800129184A6A1A
:10D1A00020184262E26801231B039A4302231A43B8
:10D1B000E2604B6A4362096B0163FF200021493042
:10D1C000015504208243E8684007C00F80000243F5
:10D1D000E2602000F5E410B50C00097A020000209E
:10D1E000012910D0022909D003291FD1617A02290F
:10D1F0001CD121001000FFF79FFE08E02100100065
:10D20000FFF7B4FE03E021001000FFF7BFFE002887
:10D210000CD00B229201A118496982180029516192
:10D2200004D005228831D2018218116040E4F8B59B
:10D23000002506000F0014F0F9FE47494C6827E06E
:10D24000E1684A0523D5072E02D0227AB2421ED1C8
:10D25000042F02D0627ABA4219D1627A022A05D129
:10D26000FF214931095D072911D10FE0032A02D1BD
:10D27000C9040CD50AE0217A012905D1FF214931E1
:10D28000095D062903D101E0042900D12500646865
:10D29000002CD5D114F0CEFE2800F8BDF8B505005D
:10D2A00002210320FFF7C3FF070002210800FFF758
:10D2B000BEFF0600A84200D10026AF4200D10027E1
:10D2C000287A01242403002819D0022801D0032839
:10D2D00023D1FDF7EDFB002803D1FDF7EEFB00287D
:10D2E0001BD03000384324D0022018F0FBF8A842AD
:10D2F00013D13C0032D13400002C2FD10DE0E8686E
:10D300000321A043E8600800FFF791FF040004D068
:10D31000002018F0E7F8A04220D10F480178032937
:10D320002ED1002E2CD1002F2AD10021017008000F
:10D33000F8BDE8680321A043E8600800D30E7660DA
:10D340000100000030CF000000040000D038CD5AAA
:10D35000FFF777FF04000BD10321FFF772FF0400F2
:10D36000D4E70000316700C0F76600C0D0050004B4
:10D37000AC420FD02000FFF74BFAFC4C207801287C
:10D3800008D1FB480088C00604D51AF076ECA068E6
:10D39000FDF7BBFFFDF796FB002800D0022018F038
:10D3A000ABF8F8BDF8B504000B22E168920101204A
:10D3B00049050026A518002903DA2000FFF7A0F987
:10D3C0001EE0237A0FF376EF071C05090D151C11DB
:10D3D0001C002000FFF767F914E02000FFF762F857
:10D3E00010E0607A0228F8D00CE02000FFF775FE0C
:10D3F00008E0A86906702000AE6107F0DEFA01E0DF
:10D4000000281FD02000FFF753FF14F019FE07007B
:10D41000002C04D1D748F3F787F81AF08EEBE068B8
:10D42000400504D56869002801D00DF05CFC05209A
:10D43000C00120186E61066020000DF006FC380067
:10D4400014F002FEF8BD10B514F0FAFDC74907E06C
:10D450003922525C120703D514F0F6FD0120EFE6E5
:10D4600049680029F4D114F0EFFD0020E8E610B57A
:10D4700014F0E6FDBD4906E0CA68520703D514F072
:10D48000E3FD0120DCE649680029F5D114F0DCFD5C
:10D490000020D5E610B514F0D3FDB44906E0CA6803
:10D4A000D20603D514F0D0FD0120C9E64968002951
:10D4B000F5D114F0C9FD0020C2E610B514F0C0FD8E
:10D4C000AA490BE0FF224932525C002A06D0CA6802
:10D4D000D20503D514F0B8FD0120B1E64968002952
:10D4E000F0D114F0B1FD0020AAE610B514F0A8FDAB
:10D4F0009E49092349689B0119E00A7A012A15D13E
:10D50000CA68520712D4CA18526A002A0ED00832CA
:10D51000D4792407240F022C08D1002A06D0927A4D
:10D52000D20703D014F090FD012089E64968002954
:10D53000E3D114F089FD002082E610B5FFF783FFE8
:10D5400000280BD1FFF793FF002807D1FFF7A2FFB8
:10D55000002803D1FFF7C9FF002801D0012400E013
:10D5600000248549854802F3CFFD002C07D0002810
:10D5700002D002F063FB63E602F04EFB60E6002897
:10D5800002D002F052FB5BE602F03DFB58E670B5BC
:10D5900004000D00160014F053FD744903E0A1428D
:10D5A00001D14C680EE049680029F8D10CE0217ADD
:10D5B000A94206D1E17AB14203D114F045FD200021
:10D5C000CAE56468002CF2D114F03EFD0020C3E5EA
:10D5D00010B514F035FD654908E0FF224932525C70
:10D5E000002A03D014F030FD002029E64968002904
:10D5F000F3D114F029FD012022E65C4800690028DF
:10D6000000D00120704710B5040014F019FD5749EF
:10D610004968002907D102E04968002903D114F0C4
:10D6200013FD00200CE60A7AA242F5D114F00CFD9D
:10D63000012005E606227E3010B514F025FA0028F8
:10D6400001D10120FCE50020FAE5F8B50500002431
:10D6500014F0F6FC0700002D01D10020F8BD1926BA
:10D660002B7A76010FF326EE07111508051919110B
:10D670001900687A022808D1280017F0EDFE8019F9
:10D68000007A012809D1012407E0E868C004FAD42F
:10D6900003E028001AF0F4EA0400380014F0D4FC87
:10D6A0002000F8BD2030807E4021C2073448002A87
:10D6B000026801D00A4300E08A430260704710B557
:10D6C00017F0B8FF002823D1022017F0D5FE0EE096
:10D6D000200017F0C1FEFF214931095D002902D069
:10D6E000406A002814D102212000FEF75DFD0400ED
:10D6F000EED102200EF0CBFD10E0200017F0ACFEC2
:10D70000FF214931095D002904D0406A002801D079
:10D71000012095E5022120000EF0C8FD0400ECD1A7
:10D720008EE5184800687047F8B5012507000C0021
:10D7300014F086FC06003B000FF3BCED0B2E2643D5
:10D74000073D3D3D2E2E2E2E3D00032071055E7CB3
:10D75000010000002CD30000000400006FFDE8E988
:10D760000EF09FFD002803D117F090FE002834D062
:10D77000C168C90431D50400FF344A342DE00000EB
:10D78000D00500041C3E01C01D000100FC80020009
:10D790009C80020000A30080F0FB00C0002C05D19B
:10D7A00017F0C4FE002801D004007E3404210720B5
:10D7B000FFF751FD002800D0002504210120FFF7CC
:10D7C0004AFD002807D000250CE0F948F2F7B6FE24
:10D7D0001AF0BCE901E0012D04D1200008F35AF948
:10D7E000F8F778FD300014F039FC2800F8BD70B56A
:10D7F0000400012514F02EFC0600002C05D0012C9D
:10D8000003D0032C01D0042C07D104210720FFF7FB
:10D8100022FD002807D0002507E0E548401CF2F76C
:10D820008DFE1AF094E904F345FB300014F016FC69
:10D8300028009BE4F8B505000E00012414F00AFC52
:10D8400007002B000FF340ED11120A19190A0A0AFA
:10D850000A0A0A12121212120A0A120002210720E0
:10D86000FFF7F9FC00280AD000240BE0D048801C08
:10D87000F2F764FE1AF06AE901E0012C02D13000EF
:10D8800004F3B2FC380014F0E9FB2000F8BDF8B551
:10D8900005000E00012414F0DDFB07002B000FF340
:10D8A00014ED071B051B141B05051B000221072097
:10D8B000FFF7D1FC002800D0002404210120FFF74D
:10D8C000CAFC002808D000240BE003210720FFF742
:10D8D000C2FC0028F7D101E0012C02D1300004F392
:10D8E000A4FC380014F0BAFB2000F8BDF0B5050028
:10D8F000012085B00C00049014F0ACFB0027002D33
:10D90000039025D0012D52D0022D10D0032D4ED1E1
:10D91000002017F0BBFD002849D0C068C00446D5E0
:10D9200008F32CFA6160206004F37EFB3DE00320E5
:10D930000EF0B7FC002803D117F0A8FD002836D060
:10D94000C068C00433D508F319FA616020602EE086
:10D9500098488068002802D0002004902AE0E668F9
:10D96000A569A068029004F3B4FB019100900298AD
:10D970003100794008430DD0029A3900A818009A66
:10D98000019B7141801A994104D3684607C8801AE7
:10D99000B1410CD202982A003B0031000FF356E847
:10D9A000401C79412A000FF38CECE160A06020005C
:10D9B00004F3CFFB039814F051FB04981EE47E4956
:10D9C0000861002070477C48006970477A490978EF
:10D9D000884201D1012070470020704710B5040033
:10D9E000FF3059300BF029F8200007F0FFF831E440
:10D9F0000123C268DB02C9079A43090D0A43C260CA
:10DA0000704710B5437A032B07D1002A02D017F0D4
:10DA100053FF1FE417F040FF1CE4490009180520DC
:10DA2000C0010918088B012AF3D1421C1205120DFE
:10DA30000A830FE410B50400C068400503D4200039
:10DA4000FFF7BAFC06E4002903D02000FEF735FEFC
:10DA50000FE501212000FEF718FE2000FEF7FFFD74
:10DA600007E570B5060014F0F5FA05005248406865
:10DA700007E0017A4468012902D13100FFF7DAFF9B
:10DA800020000028F5D1280014F0E8FAA2E5FEB540
:10DA900000210A00684606C0474844680B20800100
:10DAA0002BE0207A012827D12000FF304A300622BF
:10DAB0006946029013F0F2FF00281DD00B20800170
:10DAC00025182F6B04F339FB060020001AF072E8CA
:10DAD000002801D137002E633900300008F313FE0F
:10DAE0003649884208D3029A21212000F8F790F89D
:10DAF00000212000FFF79EFF6468002CD1D1FEBDFD
:10DB000010B514F0A7FA2C494968002907D102E0A2
:10DB10004968002903D114F0A1FA0120A9E4FF22E9
:10DB20004932525C002AF3D014F098FA0020A0E4A5
:10DB300070B50400002514F08DFA0600200017F0DF
:10DB4000A5FC03000DE0187AA04209D1180017F0D7
:10DB5000B4FC002804D04069002801D05FC92DBD65
:10DB60000100000028D70000000400003C273B858E
:10DB7000012502E05B68002BEFD1300014F078FA49
:10DB8000280031E570B504001500002904D02000FC
:10DB900006227E300FF386E9002D06D02000FF30EC
:10DBA000062229004A300FF37EE91DE570B5050015
:10DBB000FF3000244A300DF00FF8002800D1012476
:10DBC000280008E02000010090500004D005000467
:10DBD000808D5B00641CC27A817AFEF784FD002888
:10DBE000F8D1200000E5F8B5FCA10026096802285C
:10DBF000009115D100256F46785D17F051FC0AE0C1
:10DC0000607A022803D12000FFF7D0FF8619217A1D
:10DC10002000FEF7DDFA0400F2D16D1C022DEBD3DB
:10DC20003000F8BD10B5040017F02AFC217A012954
:10DC300002D1E16849070BD5617A022906D1002893
:10DC400006D0FF3061300079002801D001201AE4AD
:10DC5000002018E410B5FF2414F006FAE0490B2365
:10DC600049689B0105E0CA181268A24200DA140054
:10DC700049680029F7D114F0FBF9200003E4010002
:10DC800001200622030010B506F08CF9002804D10B
:10DC9000D44940234A681A434A6007E40100062237
:10DCA0000020012310B506F07DF9002804D1CD4AEB
:10DCB00040235168994351600BE470B514F0D4F9D6
:10DCC000C7494968002903D114F0D2F900208BE438
:10DCD0000022140001260D7A072D06D23300AB4036
:10DCE0001D00154201D1641C1A4349680029F2D174
:10DCF00014F0BEF9200077E4F8B5002507000CF019
:10DD00006BFF002801D00020F8BD14F0ADF906002B
:10DD1000B34844680CE0E068400508D520000622BE
:10DD200039007E3013F0C4FE002800D1250064685D
:10DD3000002C01D0002DEED0300014F099F928000D
:10DD4000F8BDA849800040184069704710B506F03A
:10DD50000CFA002004E4FEB500F035FA06F0D5F91F
:10DD6000441C06F01AF94443A50206F0CEF904005B
:10DD700006F013F944430120A10280020F18281A6B
:10DD80000026019004F35AF92A0033000EF368EEDE
:10DD90001C003100B81A99410292F3D2029A0198FC
:10DDA0002300121AB341EDD206F0B5F90020FEBDF2
:10DDB00070B50D00002805D00521C9014018046880
:10DDC000002C01D100200FE4E06C29000FF3BCE926
:10DDD0002068291D0FF3B8E92900206D08310FF3E1
:10DDE000B4E92900606D0C310FF3AEE929006068D9
:10DDF00010310FF3AAE92900A06814310FF3A4E948
:10DE00002900E06818310FF3A0E92900206E1C31C9
:10DE10000FF39AE92900203120690E000FF394E9ED
:10DE20002900606E24310FF390E920006030018BEF
:10DE30003172090A7172418BB172090AF172818BD8
:10DE40003173090A7173C08BB073000A8034F073A8
:10DE5000208830352870000A68706088A870000A31
:10DE6000E870A0882871000A6871E088A871000A2B
:10DE7000E87120892872000A68726089A872000A15
:10DE8000E8720120DFE4FEB50020009014F0ECF809
:10DE900001905348446861E0E06840055BD50B2081
:10DEA00080012618207A7569012812D002280CD02A
:10DEB000032814D120000CF0BAFF012805D10198E5
:10DEC000012414F0D5F82000FEBD200019F0F0EE7A
:10DED00027E00022110020001300FEF7ADFF424FA3
:10DEE000280039684030CA8802824A8942820A7A08
:10DEF0000275497A417500212B20415528002021C7
:10DF00002C300FF36CE85920C00039682018062225
:10DF100007000FF332E8B27B39000220012306F03C
:10DF200041F8002D19D00520C001201800688C216F
:10DF30000FF354E82800F5F757FDE81D0021F930EC
:10DF40004161862281615153782181631E20FF3512
:10DF50004135A86001E0012000906468002C9BD14D
:10DF6000019814F085F80098FEBDF3B56F164B4686
:10DF70000100000024DB000000040000C8484E310E
:10DF800081B007000CF032FE002801D00020FEBD59
:10DF900014F074F8060017480025446813E02000C8
:10DFA000FF30062239004A3013F08CFD002809D1D9
:10DFB0002000029906227E3013F084FD002801D152
:10DFC000250002E06468002CE9D1300014F05AF812
:10DFD0002800FEBD10B5040003F056FD002804D152
:10DFE0002000F3F7C3FB002800D0012013E5000058
:10DFF00002030000D005000490500004F0FB00C0B4
:10E00000F8B5050014F03AF80090A4480B26B601C4
:10E010004468012713E0E06840050FD5A019406966
:10E02000FF30401C4169A878020938009040014245
:10E0300004D0E52229002000F2F74BFC6468002C94
:10E04000E9D1009814F01EF8F8BDFFB581B01C00AE
:10E0500015000A9E14F012F80021216031608F49EA
:10E060004A6828E0D168490524D50B218901511857
:10E070004969FF31491C8F694B693B4337683B4312
:10E080003360019B93420FD1029B002B236805D084
:10E090008F693B432B4323604D610BE04F693B434A
:10E0A0002B4323608D6105E04B6989690B4321682F
:10E0B0000B4323605268002AD4D113F0E3FF91E4AC
:10E0C00070B5002503212800FFF7D9F804000321CB
:10E0D0000800FFF7D4F8002C01D0002815D121004A
:10E0E000014313D0002C00D10400002C0ED0217A63
:10E0F0002000FEF777F8040008D0607A0328F6D1F4
:10E100002000FFF7C0FA0028F1D001252800D1E453
:10E1100010B5C2680400D00415D5207A002808D0B4
:10E12000012811D003280ED1607A032801D00128DC
:10E1300009D1002904D1200019F0F6FB002802D1F2
:10E14000200019F0C4ED66E49003FCD401204004E3
:10E150000243E2605FE410B513F090FF4F4906E020
:10E160000A7A062A03D113F08DFF012053E449688F
:10E170000029F5D113F086FF00204CE401000B22AA
:10E18000F8B592018A180092927B01200500FF2ABF
:10E190001ED10A7A022A00D1002559220024012723
:10E1A000D2008E183E4A39005268A140114210D167
:10E1B0002206120E2B003100012005F0FDFE002882
:10E1C00007D10099364A8C735168A7403943516092
:10E1D000F8BD641C062CE5D3F8BDFEB500F03DF893
:10E1E0002F4C0290A1680FF3B8EB002501902C484A
:10E1F000A90008184469002C21D00B2080012718A1
:10E200007E6902994036B0890FF3A6EBB075002005
:10E21000F0758034217A019A5143E26889021161D4
:10E22000E16880224861E068C1781143C170B27B27
:10E2300000921300B97B207A012205F03DFF6D1C8E
:10E240002D062D0E032DD2D3019804F34CF814485B
:10E250008068401E05F052FFFEBDF8B500200500A5
:10E260000F4E0B27BF013061A800801940690028BC
:10E270000DD0C019406934694030808904E0210024
:10E280000FF36AEB20000C00002CF8D130616D1CFC
:10E290002D062D0E032DE7D33069F8BDD0050004FF
:10E2A0009050000470477FB503000B2080011818C0
:10E2B00082690D00022404291BD2180017F0D8F936
:10E2C000002805D01420684380180079040910E064
:10E2D0001800FFF712FA00280BD0022168460FF051
:10E2E00053FF280010F021F980006946085C0407FC
:10E2F000240F200004B070BD03000A0000B517F021
:10E30000B7F9002807D00B20800118188169602018
:10E310005043B030085A00BD10B5F2F7BBFF0028DB
:10E3200010D0F2F7AFFF7549012080058860C01159
:10E33000F2F776FF00F038F919F088EB00F044F9B5
:10E34000F2F798FF10BD70B513F098FE06006C4808
:10E350000168080609D5480607D5684CA568E01786
:10E36000E060FFF7D9FFA56001E019F070EB300025
:10E3700013F088FE70BDE6E710B513F0FC32A45C24
:10E380000100000020DF0000000400009B929D5D62
:10E390007FFE040000F0ECF800F0F4F8200013F029
:10E3A0007BFE10BD70B5040013F072FE05005948E5
:10E3B000016821430160600601D4200618D5480693
:10E3C00016D5080614D5F2F7DAFF5149FF20401C94
:10E3D000C8604A68024200D088604F4908686122DC
:10E3E0001205904308604D4988684D4A1040886086
:10E3F000280013F051FE70BD10B5F6F747FD002858
:10E4000001D1484810BD484810BD10B501F0BFFA11
:10E4100046494000085A464B40495843C9680B07D3
:10E420001B0F0EF370EF080507060609090B0B0614
:10E43000400810BD800810BDC00810BD000910BD07
:10E4400010B5FFF7E2FF3B49884201D13A4810BDC1
:10E450003A49884201D13A4810BD3A4A3A49904275
:10E4600019D03A4A904201D1394810BD394A9042F8
:10E4700002D13748D23810BD374A904201D13748CF
:10E4800010BD374A904201D1364810BD364A9042FD
:10E4900001D1364810BD080010BD70B5040013F05E
:10E4A000F7FD05001B480168A1430160600601D427
:10E4B000200618D5480601D5080614D41648016868
:10E4C0006122120511430160016842051143016098
:10E4D0000F49C00D8860F2F76AFF10488168104A42
:10E4E000D24311438160280013F0D6FD70BD094A64
:10E4F000010012680020914300D101207047C00044
:10E5000005D5044818304068002800D000477047FF
:10E510000030008078F800C00021008000280080D2
:10E520007FFFDFFF3F3D00007F841E00407B020035
:10E53000A0860100001BB70054150000405DC60016
:10E54000B013000000F82401540D000000366E01E5
:10E55000AA0A000080BA8C0100F04902AA06000055
:10E5600000751903EB040000007C9200AA1A000059
:10E570003349002010B5086132490420086100F0D9
:10E5800036F810BD002010B5F2F71EFD0120F2F79D
:10E590001BFD0320F2F718FD04000020F2F747FDF1
:10E5A0000120F2F744FD0320F2F741FD02002100B3
:10E5B0000320002300F058F810BD7047234922487B
:10E5C00008602248312180304161B32141611F48F8
:10E5D0004030C16B02229143C16370471B49B12097
:10E5E0008031486118481949083808607047154853
:10E5F00010B50168164A114001608168154A114042
:10E6000081604168144A114041608168052291434C
:10E61000816012494868124A1040486001F07AFA55
:10E620001048C069002803DB40210E2001F099F951
:10E6300008211F2001F095F901F041FA10BD0000FA
:10E640000029008000280080CD0200000023008007
:10E6500000CFFFCFEF7BFBABB5AAAABF00220080A3
:10E6600040F0FFFF002100800A2A10B511D00B2ACC
:10E670000FD00C2A0DD1002B0BD100210420FCF26D
:10E680006BFB0448426910218A43426182698A43D4
:10E69000826110BD00020090F8B5FE48FE4A018874
:10E6A00091421DD002001288012441889440FB4F02
:10E6B000012904D1FD68A5432C43260003E0FE6830
:10E6C000A64334432500F6498088096813F0CAEA56
:10E6D0008905800A0843FD6001D019F0ECE9FE606D
:10E6E000F8BDF8B501210600EA48012558388155E2
:10E6F000E849102057398855EA48B1010F18EA480F
:10E7000000220188E948130016F0A3FAA90000913D
:10E71000002878502FD0AC210181DE48B400503859
:10E720000059403045720098385801894018D9493D
:10E730005039095944310EF31CED0098082138581E
:10E74000D44A01730123083A18001159A840014323
:10E750001151110048390959121D8871000AC871F8
:10E7600010005438805D1159834019431151401CE9
:10E770001100543988556D1C102DC0DB012100207B
:10E7800017F0CEF8F8BDC34910B5C068714C5D41B3
:10E79000010000001CE3000000040000B30318E0C7
:10E7A0005C39095C002908D1C6490A68002A02D1EF
:10E7B000C548086001E0FFF79EFF002010BDF8B5D6
:10E7C00085018400B84EBC4F5C3EB16A002912D16D
:10E7D00030000C300059C17982790802310058317B
:10E7E000095910430840310050310851C0072BD15E
:10E7F0007859002828D17D21B448002209010FF35F
:10E80000F7F8002878511FD00021B162A64EAC2243
:10E81000503E028130594030417278590189401888
:10E82000315944310EF3AEEC01203100483108512A
:10E83000315900228871CA7132004C32115901439A
:10E840001151795908200873F8BDF8B5040000206B
:10E85000E168954E8900503E71588871C871E16831
:10E8600089007158012208714871E1688900715866
:10E8700020310A76E1688900715837002031087626
:10E88000E0680C3F395C002913D1800035586C35A5
:10E8900028000EF368EC03218902084329000EF3D7
:10E8A00072ECE0688000305810226B300178114320
:10E8B00001707D4801255C38056445648564C56444
:10E8C0008562E068395C002908D1FFF778FF764956
:10E8D000E06858390D54E068491C0D542000FFF7DA
:10E8E0005CFFE0680721800030580023203001756C
:10E8F000E068800030586D4920300377E0680028D8
:10E9000003D1694A118051809180674A0D0A921D96
:10E91000117055709170090AD17011005239002898
:10E9200002D10868C37003E0052280000858C27055
:10E93000E068800008588370E06880000858037120
:10E94000E068800008584371E06881007258D5790A
:10E9500096792A02324309D05348083805004258B4
:10E96000183D6A50E16889004350E0680C2116F0B8
:10E97000E1FF0020F8BD70B5040013F093FB4A4A94
:10E98000EF25A100503A53582033002C1D7603D0B8
:10E990005258172320321375434B00223C3B5A50E8
:10E9A00013F084FB70BD70B5040014234249584332
:10E9B0003C3940180FF3AEF83F4B3B4E0121A2010A
:10E9C00040330D00D318573E09E02A00002804D137
:10E9D00088001858002800D100221000491C002887
:10E9E00002D1325D8A42F0D870BD012008B5009096
:10E9F0003748142100686A46FCF257FF08BD3548C5
:10EA0000704770B50C000121C9078A78264B800039
:10EA1000383B1958A14230D0002C1C500DD000209A
:10EA2000012185005D59A54204D0451C0E00AE4071
:10EA3000164222D1401C0128F3D31B4D5C3DA8781F
:10EA4000A0421AD0280019496230002C09D0C2789F
:10EA500083781002184388420FD000F051FE012045
:10EA600008E04278037810021843884205D000F08D
:10EA700047FE0020F2F7FFFBAC7070BDF0B505005B
:10EA80000024094A21008000503A135885B02033F1
:10EA90001C7516580123203633761058AE012030ED
:10EAA00004760548371822E0DC7D0200FFFF0000F5
:10EAB000000200909C2401C090950200E6F700C07F
:10EAC00064040004C8F500C073E20000C40400043C
:10EAD000B0F500C067E50000A00004903858002899
:10EAE00004D00EF35BFF049900207850641C494861
:10EAF000405DA042F0D8484F14203A00143A11006B
:10EB000068437C310B00543BC3188218C01901AF15
:10EB10000DC70024A80147180AE0A000009038584B
:10EB2000002804D013F0FAFA009900207850641CF1
:10EB30003848401C405DA042EFD8374C683405E0AF
:10EB400001980EF3BEFFA05113F0E8FA01980EF3FE
:10EB5000E1FF0028F4D105E002980EF3B2FF7860DF
:10EB600013F0DCFA02980EF3D5FF0028F4D105E08B
:10EB700003980EF3A6FFA05113F0D0FA03980EF3FA
:10EB8000C9FF0028F4D12349A0510120091F0864BE
:10EB90004864C864886405B0F0BDF8B5795FF4B323
:10EBA0000100000018E7000000040000E0D9CB8C51
:10EBB000002425001C48A70034301426C5511B48EA
:10EBC00066431438301814210EF330EA1748142124
:10EBD00030180EF32CEA15481421143030180EF3B7
:10EBE00026EA11483022001DC15910486243A8305E
:10EBF0001018C4608160456185610D49C56101617E
:10EC00000C4901620C4985624162FCF2C1FD641C41
:10EC1000012CCFDB09490820F1F71AFD0849FF2034
:10EC2000401C8860F8BD0000847D020068950200E9
:10EC3000C7E3000053560200235A0200AD5F0200F2
:10EC40000030008031B56B461A78587899780024E6
:10EC5000012A0ED0022A0AD1484A10704848017091
:10EC600000F03AFE10F066FA040000F058FE2000B2
:10EC700038BD444A10704448017000F0F8FD10F0AF
:10EC80009DFA040000F019FEF1E7F8B500263F4FA9
:10EC900034003D1DA00040190068FFF7D3FF002895
:10ECA00006D0A00039684019006888600120F8BDCE
:10ECB000641C052CEEDB002E05D1386801210222F0
:10ECC0008172027241720020F8BD30480022006853
:10ECD000017A01290CD0022929D1284B417A1970D7
:10ECE0002B49C1602B4901612B4941612B4916E039
:10ECF000244B417A1970817A234B02291970284BD1
:10ED0000C360284B0361284B436107D12749097829
:10ED1000BF2901D01F2901D1254900E02549C26141
:10ED2000426081610121427001700800704700203B
:10ED3000704721497D20000110B5086020491F4817
:10ED400008602049114C086020680078002803D131
:10ED5000FFF79BFFFFF7B9FF2068C068804710BD31
:10ED60000A4800680069004710B50C0007490968A7
:10ED7000496988472060012010BD0000B0B9020039
:10ED8000B1B90200B4B90200C4B90200ACF800C0C5
:10ED900041F4000087F4000001AD300095AC300074
:10EDA000D7F3000023F40000FBAD3000C5B902002A
:10EDB00057AF3000F7AE3000B8B90200102700009E
:10EDC000BCB90200C0B9020010B5040013F074F918
:10EDD0001F49012C0CD11F4A4A601F494B6A8022EF
:10EDE00013434B624B6A93434B6213F069F910BDB6
:10EDF000184A521CF0E70800E6E770B50400401E10
:10EE0000044223D105F03EFF20421FD005F030FF21
:10EE100020421BD0200018F07CEF104C616A60315A
:10EE2000C872FFF7D1FF606A0025603045730AF0B1
:10EE30000AF90B480560616A6031C87A8872FFF789
:10EE4000C3FF606A60300573012070BD002070BD93
:10EE5000002300800100030000A80080F058000497
:10EE6000CC2701C010B5FAF2B9FA10BDFB48807882
:10EE70007047FA48C0787047F84800697047F7490A
:10EE80001F2088807047F8B50400F44DF44F13E05C
:10EE9000A001060010F08DFA00280AD0300010F012
:10EEA00065FA2A89D300DB1903C3601C521CE88071
:10EEB0002A81641C2404240CA8888442E8D3F8BD69
:10EEC000F3B581B000240F00E44EF08800904018A4
:10EED000B18888422AD9FF20FEBDF088B1888842D7
:10EEE00003D30098FFF7CFFFF5E7019AE1008D18F3
:10EEF0006B682A68800110F03BFAF088800110F0FE
:10EF000035FA0CCD5040594008431BD1F0888001A0
:10EF100010F060FAF088800110F04BFA002811D050
:10EF2000F088401C641C2404240CF080BC42D4D320
:10EF30000098FFF7A8FFF1880098081AC01B00048A
:10EF4000000CFEBDF088401CF080C6E7F8B5012437
:10EF50000025C24FB888009070E0C149E000411818
:10EF600008784E7842065ED503003F3B0EF3DEE99B
:10EF70000B691C1C07110B0E151515171D00641CC1
:10EF80002404240C5AE088783861F8E7887878708F
:10EF9000F5E7B44820220DF3AEEF30194CE0887845
:10EFA000B870C878F870EAE7891C4A28F43F1E1048
:10EFB0000100000014EB00000004000014B6BE388D
:10EFC0001CD07F281AD04888000B01D0088815E093
:10EFD00008780200AF3A072A01D9BF280ED10A7A71
:10EFE000D303034310091B0400011B0C0002184348
:10EFF000B22803D1497A0907090D08439E4A002126
:10F0000020320BE006234B43D35A834203D16D1EBB
:10F010002D062D0E04E0491C0906090EA942F1D364
:10F02000062359435052881844804671301904040D
:10F030006D1C240C2D062D0E0AE0022801D18978C2
:10F0400039700121002800D0310008190404240C73
:10F05000009884428BD3F8BD8749002010B5087012
:10F060008348416900290FD101214161002010F03E
:10F07000AAF9002801D110F0B7F9FFF70AFF002024
:10F08000FFF70BFFFFF76CFF10BD7B4A002020321B
:10F090000DE07F2908D1062358437649801840881F
:10F0A000C000411803C97047401C202804DA06211B
:10F0B0004143515C0029ECD10020C043010070475E
:10F0C00070B506000D00FFF7E0FF0C00FCF2CCFE6F
:10F0D0000004000C30602000FCF2C6FE2860012015
:10F0E00070BD7CB504000020634A2032002C2BD078
:10F0F00025E00D2920D1062358435E498018408819
:10F10000C00040188288110B01D1811C0FE011064C
:10F11000574B120B92001833D218090E801C403A3C
:10F12000D56B6A4601ABA8476B461A790099200057
:10F130000DF3EAEE01207CBD401C202804DA0621F4
:10F140004143515C0029D4D100207CBDF8B50D00AD
:10F1500016001A000021002D3DD0474C454F2034A9
:10F16000002833D000060016401C40424401FF2016
:10F170000B3082422FD3202C2DDA010028000DF312
:10F180008AEFE000C119FF222800521C0A300DF35B
:10F19000BCEEFF200B30308013E04A2813D106204C
:10F1A000484300194088C000C1194888001F040462
:10F1B000240C94420FD8091D220028000DF3A4EE60
:10F1C00034800020F8BD491C202904DA0620484379
:10F1D000205C0028E1D10120F8BD002310B51A0001
:10F1E000837004E0845CE3181B061B0E521C8A42E9
:10F1F000F8D30121C91A817010BDFFB5C3B06846AC
:10F20000FFF76FFF00282FD06B465C88449884423C
:10F210002AD800256E4605E07059FCF225FE439978
:10F2200048512D1DA542F7D345982018FCF21CFE2D
:10F230004399486043982100FFF7CFFF0E4800270D
:10F2400020306AE0090665D50B49449B20314018FF
:10F250004088C1000748081881880A0B0E05360D42
:10F26000A1199942419209D9012047B0F0BD00008F
:10F27000C4F800C0C04101C0C04201C0002A02D190
:10F28000801C42900EE06D4B92003106D218090EA0
:10F29000801C403AD56B40AA41ABA847409840AB90
:10F2A00042901E79006880218843FCF2DDFD43997D
:10F2B0000425085109E04299A80880000858FCF28A
:10F2C000D3FD439A61192D1D5050B542F3D35C49CB
:10F2D0007D1C02E0000607D46D1C202D04D2062000
:10F2E0006843085C0028F5D10020C043202D07D0DA
:10F2F00006226A43895C002902D04598A1190818A2
:10F30000FCF2B2FD01004398001941603100FFF7A3
:10F3100064FFA4197F1C202F05D206207843484A99
:10F32000115C00298ED14698048000209DE7FFB52E
:10F33000FF2100240500491C424881B00DF380EEF6
:10F34000404A286808211060042029E02B5CE34033
:10F35000A41C9B0724069B0F240E082C03D1401CE1
:10F3600000240006000E032B12D12B5C002C04D1CC
:10F37000401C0006000E53540FE0401CE340000602
:10F38000000E082753542E5C3F1BBE401E4303E073
:10F39000FF26022B00D01E005654491C0906090EF8
:10F3A000029B9842D2D3049801700398026004989B
:10F3B0000078508005B059E7F7B500240A2307CE3E
:10F3C0000100000010EF000000040000476C6D54C5
:10F3D000160022481F4F151DFC2A36D817E04A296F
:10F3E00010D1C0194088C1001C4809184888A8429B
:10F3F00012D10198091D320012F096FB002801D1AC
:10F400000020FEBD641C2406240E202C04D20620FD
:10F410006043395C0029E2D1114C4A202070300051
:10F420000B30C008607001993200201D0DF376ED9D
:10F430002904090C6180C91DC9082000FFF754FD8B
:10F44000FF2802D0FFF796FDDAE70120FEBD00009D
:10F45000DCF800C0E04201C0C03F01C0C04101C0B3
:10F46000C04001C0AB4908220028C86801D0104341
:10F4700000E09043C8607047A749002010B548607D
:10F48000F5F7E5FB10BDF0B503252D03A148A34C0E
:10F49000C030C20D9302870C00299E4E016A0AD02B
:10F4A00011430162016A99430162A0682843A06088
:10F4B0003068384309E091430162016A19430162EF
:10F4C000A068A843A0603068B8433060F0BD38B58C
:10F4D00005000024684605F0DDFC00281AD0002D48
:10F4E0000BD16B465878C10714D0400612D59878D6
:10F4F0008007800F0CE001240CE0012D0AD16B463F
:10F500005878810706D5C00904D098788006800F06
:10F510000128F0D0200038BD73B56B4605005C793A
:10F52000600705D57C484168002901D1012141606F
:10F530002800FFF7CCFF0106090E2800FFF7A3FF04
:10F54000600703D46B461879000900D00120FFF74B
:10F5500089FF7CBD33B56B460028197902D10807B5
:10F56000000F02E0012813D108096D4A6949D4430C
:10F57000803100280DD06B4B6B4D01280DD0092830
:10F5800010D00F2804D1C817C8600861C86108628C
:10F590003CBDCA600A61CC6102E0CB600A61CD610A
:10F5A0000C623CBDCB6061480861CD616048EEE70C
:10F5B000F0B50028047A4578067947792BD00129DF
:10F5C0000CD10599012909D1012A06D16540D90735
:10F5D00000D06640990700D567402C00554B19684C
:10F5E000914200D01A6001782A0609040A432102D8
:10F5F0000A4348492243C0314A628279C3781204DF
:10F600001B021A4332438A62C279807812043B0299
:10F610001A430243CA62F0BD38B5050000246846AB
:10F6200005F038FC002803D1280000F00FF838BDA1
:10F630006B4618780007000F01D0012804D100990B
:10F64000280000F038F80400200038BD30B5002450
:10F6500085B0050021002200230001A804940EC0FB
:10F660006B46187C1C74587C012108435874987CA4
:10F670009C741C715C7180209C71D8711C725C72CE
:10F680009872D8721C7304992800FFF745FF6B46E7
:10F69000997C28000091FFF75DFF6B46187C2300E2
:10F6A0000207120F00922200210001A8FFF780FF3D
:10F6B000012005B030BDF3B585B0002507001E4818
:10F6C0002E00406A2C006030C27A380002A905F092
:10F6D000FCFB00281CD006993800FFF71DFF6B4685
:10F6E000997E38000191FFF735FF6B46587EC106C1
:10F6F00001D4800600D501256B46187E2300020741
:10F70000120F00923200290002A8FFF751FF0120DA
:10F7100007B0F0BD00A70080E0F800C0002800801E
:10F7200011DD55DD1FDF5FDFEF2FAF2FF1FDF5FDA1
:10F73000FEF2FAF238040004F0580004F94910B55A
:10F74000096812F0B8EA8905800A084301D018F068
:10F75000DAE910BDF448016A0F2211430162022068
:10F76000ECE7F148016A0909090101620120E5E7B6
:10F77000EE4970B50868082290430860EC4A50686A
:10F7800040084000506010690B2108431061E949AE
:10F7900008009369DB0601D4401EFAD29069800606
:10F7A00001D4491EFAD212F09BFCE3490A680124F5
:10F7B0006406A2430A60E04A80321368DF4D2B40A2
:10F7C00013601368ED432B4313600A68061BCA7469
:10F7D000010000000CF3000000040000F8A948E755
:10F7E00022430A6012F08AFC0120FFF7B1FFFFF705
:10F7F000BBFFFFF74BFE70BD70B5F4F232EFD54D95
:10F8000004002878022812D1A869401CA8612006AB
:10F8100004D4D148F0F7E2FE18F0E8E9802C02D1D8
:10F82000F4F21EEF70BD2000F4F224EF70BD6869A1
:10F83000002805D0C8480A38F0F7D0FE18F0D6E9FD
:10F8400002206C6128700120A861C44DAC88800240
:10F850000440A8886B26A043F600B042E6D0022000
:10F8600000F06EFA0028E1D03443AC8070BDB94995
:10F8700010B58869401E88610CD1486900224A6130
:10F88000FF2280280A7002D1F4F2EAEE10BDF4F2F1
:10F89000F2EE10BD0028FCDAF4F2E2EEAE480938D0
:10F8A000F0F79CFE18F0A2E910BD70B5A94E706982
:10F8B000002807D012F01EFCA7482438F0F78EFE6F
:10F8C00018F094E912F016FCA44D7061AC88012088
:10F8D00080020440A888A04382280BD02888F080AA
:10F8E000002000F02DFA002804D0A8883081822062
:10F8F0000443AC8070BD974910B5984A0B8948699C
:10F900009380CB88138000224A61FF220A7012F094
:10F91000F5FB10BD10B58F4C6069002807D012F0C0
:10F92000E9FB8D482338F0F759FE18F060E912F032
:10F93000E1FB8A49606188880122920210408A882E
:10F940008243022A08D00A88E2801A220A808A8822
:10F95000228102221043888010BD7E4910B57F4A63
:10F960000B8948699380CB88138000224A61FF226B
:10F970000A7012F0C3FB10BD70B505000E00FBF25B
:10F9800002FF764C20342581FBF2FDFEA680FBF2BF
:10F99000FAFE70BD70B505000E00FBF2F4FE6F4C70
:10F9A00020342581FBF2EFFEA680FBF2ECFE70BD59
:10F9B00070B50500FBF2E7FE684C20342581FBF2B0
:10F9C000E2FE207970BD70B504000D00FFF7F0FF76
:10F9D000284301002000FFF7DDFF70BD70B5040073
:10F9E0000D00FFF7E5FFA84301002000FFF7D2FF5D
:10F9F00070BD58484178002909D159490968012248
:10FA000009044270090F02002432515C8170807831
:10FA10007047504AD078002818D1106150480068CB
:10FA200011008007800F10310123002807D0012822
:10FA300007D0022807D0032807D1402004E0202067
:10FA400002E00B6001E010200860D370106970477D
:10FA5000444B59681C22914310400843586070473A
:10FA6000404B5968FF22E1329143104008435860EF
:10FA7000704770B50C00FFF7F3FF2000FFF7E8FFB9
:10FA8000384D39482860FFF70FFA384EFF2822D04A
:10FA90006868304068602C6835480440FFF704FA15
:10FAA000000702D5012080060443FFF7FDF9400757
:10FAB00002D5012080040443FFF7F6F9800702D540
:10FAC0000120C0040443FFF7EFF9C00702D0012072
:10FAD000C00604432C60FFF7EAF9FF2820D0A8688D
:10FAE0003040A8602C6823480440FFF7E0F9000785
:10FAF00002D5012080020443FFF7D9F9400701D560
:10FB000004200443FFF7D3F9800701D508200443FC
:10FB1000FFF7CDF9C00702D00120C00204432C60DA
:10FB200070BD0C4910B5486900224A61FF220A7075
:10FB300012F0E4FA10BD00009C2401C080A10080F6
:10FB400000A3008040A600808813000000210080F0
:10FB5000FFEFFFEFE8F800C0570001000008009039
:10FB6000002000800029008004FB04FBFDFF7FFFD4
:10FB7000FFFFF3F3F3F3FFFF70B57B4C60690028E0
:10FB800006D012F0B7FA7948F0F728FD18F02EE801
:10FB900012F0B0FA764D6061AC880120800204401A
:10FBA000A888B526A0433601B04206D0022000F056
:10FBB000C7F8002801D03443AC8070BD10B56A4C42
:10FBC000207900280BD101202071FFF7D5FF0620F6
:10FBD000FFF7EEFEC006C00F6071FFF70625ACAB65
:10FBE0000100000008F7000000040000AB739B8BCD
:10FBF000A2FF6079A8E7F8B50700FFF7E9FF624CBC
:10FC0000250D660D00280FD0FFF7C0FF80212620AC
:10FC1000FFF7E3FEFFF78FFFA0682843A060A0680E
:10FC20003043A060002006E0A068A843A060A06860
:10FC3000B043A060380000F0C3F8F8BD10B5040070
:10FC4000F5F72AFD00281ED15048C16809090901AD
:10FC50002143C160816809090901214381608268EB
:10FC6000010C0A43826002691209120122430261F7
:10FC700002690A43026182690A4382614449A00021
:10FC80000858444908605FE740488038008800060B
:10FC9000000E70473D48803800683F498874010C69
:10FCA0003D48203801863D494969816370473A489B
:10FCB00010B52038016A002000F057F844E73648B4
:10FCC00010B520388169002000F04FF83CE7324839
:10FCD00010B5203841688161002000F046F833E714
:10FCE0002D4810B5203881688161002000F03DF872
:10FCF0002AE7294810B52038C1688161002000F04A
:10FD000034F821E7244810B52038016981610020CA
:10FD100000F02BF818E71D48214A016811430160E3
:10FD200070471A491E4A0868904308607047164990
:10FD30008868CA0C9043886028E713488168C20C21
:10FD400011438160F7E6002070470C48C068704797
:10FD50000020704710210A2803D20849400034319E
:10FD6000095A084801800120704708000A492039D3
:10FD70004A69824201D0486160E77047E8F800C0F4
:10FD800037000100000800908028008000210080DA
:10FD9000007B02009C2401C01059000400A80080D0
:10FDA000000820880449034808600449001F0078BF
:10FDB000087070472CF900C0ACB90200A8B9020065
:10FDC00070B505002924FFF7E1FE2000FFF7FAFDDA
:10FDD00029002000FFF7E8FDFFF7ADFE70BD70477A
:10FDE000704710B5FFF770F8411C02D00006000EF6
:10FDF00010BD4A2010BD10B500F040F810BD10B580
:10FE0000FFF795FF10210420FFF7F2FD01210520E7
:10FE1000FFF7EEFDFFF791FF10BD10B5FFF787FF6D
:10FE200010210420FFF7D9FD01210520FFF7D5FDA2
:10FE3000FFF783FF10BD10B50400FFF7A7FE002CED
:10FE400015D0FFF7F0FD000702D42C21192009E09E
:10FE5000A4211920FFF7A8FD60211A20FFF7A4FDB7
:10FE60006C212820FFF7A0FDFFF765FE10BD0F21D4
:10FE70001920FFF799FDFE216620F3E7F8B500246D
:10FE8000672712F0D7FF00283DD1FFF77FFE04213E
:10FE90001620FFF7ADFD1D4D0621286811F01EEF5D
:10FEA0008905800A084301D017F040EEFFF799FF5B
:10FEB00001001F20FFF778FD10212020FFF78DFDA6
:10FEC0007D26F6002868062111F008EF8905800AD2
:10FED000084301D017F02AEE0920FFF773FD641CD8
:10FEE000000602D4B442EDD303E00820FFF76AFD18
:10FEF000070010212020FFF77BFD04211620FFF7CB
:10FF00006CFDFFF718FE3800F8BD00009C2401C00E
:10FF100003490A7FD207FCD101492031088270478A
:10FF2000000800908C4A8B49116001608B48007872
:10FF3000002800D001207047002804D00A2803D0F0
:10FF4000102803D1032070470F207047012070470D
:10FF5000F0B587B00E008446110018000D9D0C9C72
:10FF600000220E9B0096049203900592019102904C
:10FF70002A0021006046F7F2F5FA002801D0FFF7C9
:10FF8000DBFF07B0F0BD70B50C001500049A190036
:10FF90000A2C04D113002A00F4F2C6FD01E0F4F2A9
:10FFA000EFFB002801D0FFF7C7FF70BD7CB55A43B7
:10FFB000040006980D001600002801AB0AD10022AB
:10FFC00065480092006832000A21FFF7DCFF002834
:10FFD00000D0FEE7019B0122290020000096F6F2E6
:10FFE000A9FD002800D0FEE77CBD1FB5376879DD8C
:10FFF0000100000004FB0000000400005F1CEE3F55
:020000021000EC
:10000000002202A9F7F256F8002801D0FFF79EFF60
:1000100004B010BD1A0010B5F6F27EFF002801D022
:10002000FFF794FF10BD534910B54968F6F236F852
:10003000002801D0FFF78AFF10BD052A10B507D0B0
:10004000062A05D0072A01D0082A02D1002200E0A2
:100050000222F6F225F9002801D0FFF777FF10BD44
:1000600000B587B00B0003AA04A901921A00009101
:1000700006A905ABF6F2ECF8002801D0FFF766FF01
:1000800007B000BD7CB5060010001D000023069AD5
:10009000052801930BD0062807D0072803D008288D
:1000A00006D1012004E0002002E0032000E002204D
:1000B00000920200300001ABF6F262F804000198F1
:1000C0001A2C286001D0072C08D129003000FFF736
:1000D000C7FF02201A2C00D021207CBD002C01D1AA
:1000E00000207CBD2000FFF731FF7CBD0A0022A16B
:1000F00010B5F7F2C1F8002801D0FFF727FF10BDB7
:1001000010B5F7F22DF9002801D0FFF71FFF10BD41
:1001100010B5F7F2E9F9002801D0FFF717FF10BD7D
:1001200038B51400049D1A000A2905D1130011499D
:100130002200F4F295FD05E000920E4923002A000A
:10014000F4F2ACFB002801D0FFF700FF38BD0A290C
:1001500010B502D1F4F2C8FD01E0F4F2EBFB002887
:1001600001D0FFF7F3FE10BD68800200487D020059
:10017000447D02004CF900C04F53415F53656D61EF
:100180000000000070B505000C00000900F0DEF86A
:1001900020702807000F00F0D9F8607070BDF8B526
:1001A00005000C000026022875D077DC002D74D0E5
:1001B000012D7FD120000CF3EDFF001967A111F094
:1001C0006FFD20000CF3E6FF0719FFF767FD00063F
:1001D000000E3900FFF7D6FF20000CF3DBFF0019FB
:1001E00061A111F05DFD20000CF3D4FF00195FA1A7
:1001F00011F056FD20000CF3CDFF0719F4F7D4FAE7
:100200003900FFF7BFFF20000CF3C4FF00192821BD
:100210000170467020000CF3BDFF0719F4F7CCFA0B
:100220003900FFF7AFFF20000CF3B4FF00192E21B7
:100230000170467020000CF3ADFF0719F4F7C4FA03
:100240003900FFF79FFF20000CF3A4FF001948A11D
:1002500011F026FD20000CF39DFF071902F068FF46
:100260003900FFF78FFF20000CF394FF00192821BD
:100270000170467020000CF38DFF071902F055FF46
:100280003900FFF77FFF20000CF384FF00192921BC
:10029000017046700EE01CE000E00EE00A2D51D027
:1002A000632D07D134480078582803D13349200002
:1002B00011F0F6FC30480570F8BD304920002839AF
:1002C00011F0EEFC20000CF365FF00192038867752
:1002D000F0E720002AA111F0E3FC20000CF35AFF04
:1002E000011929484078FFF74DFF20000CF352FF19
:1002F00000192E270770467020000CF34BFF0119E0
:1003000021480078FFF73EFF20000CF343FF00195F
:100310001EA111F0C5FC20000CF33CFF01191E4882
:100320004078FFF72FFF20000CF334FF001907700F
:10033000467020000CF32EFF011917480078FFF7D4
:1003400021FFB7E71549B2E7154870470A2801D2DF
:10035000303000E057300006000E70474368697087
:100360005265763A000000002C20000042423A001C
:10037000292C2052463A000054F900C0CD7B0200DF
:100380004F2E522E3A000000FDF500C020204361A0
:100390006C204F2E522E3A00BE0101C0BCF500C0A9
:1003A00024440ECB07E003788B4207D04378801CAF
:1003B000D21A921E1818022AF5DA0020704700009F
:1003C0000448C1690029FCD0816A0422114381627A
:1003D00070470000003400800748002110B5006815
:1003E000C94312F04BFD002010BD034810B5006852
:1003F00012F04BFD10BD00002C2601C0AB489185CA
:100400000100000000FF0000000400000CC63D5386
:1004100070B511F08DFE0500FF48FBF291FC040061
:1004200009D02000542108300CF33CEEFA4821009A
:100430000C30FBF2AFFC280011F07EFE200070BDF6
:1004400070B5040011F074FE0500002C0DD02000E2
:10045000542108300CF326EEEF4821000C30FBF25B
:10046000D7FC0100EC48FBF295FC280011F064FE7B
:1004700070BD10B5F1F723F9002010BD704770472B
:10048000002803D02030407E0007C00F70470028AE
:1004900007D02030427EF723C9071A40090F0A43CC
:1004A00042767047002807D02030827EFB23C907A0
:1004B0001A40490F0A4382767047002806D0C26866
:1004C000C90752085200C90F0A43C260704700288A
:1004D00006D0C2680223C9079A43890F0A43C26043
:1004E0007047002806D0C2681023C9079A43C90E76
:1004F0000A43C2607047F8B500250E0017002C00B3
:10050000002824D0092189014218D16A002901D08C
:100510000D000835516A002901D00C000834330061
:10052000220029000097FDF23FF8002E06D0002D92
:1005300004D0280048210C300CF3B4ED002F06D075
:10054000002C04D0200048210C300CF3ACEDF8BD99
:1005500070B50400006800280BD0806D00250028CD
:1005600003D0FFF76DFF206885652068FFF768FFFF
:10057000256070BDF8B5040015F00DF8200014F0EA
:10058000E3FF210020314B7EF72213404B76E568D4
:100590000426B5432122E560125C97070AD509229B
:1005A0009201C56FA2185562C06FD0620820034344
:1005B0004B7605E0100701D4900601D53543E56080
:1005C000200017F0E6EB0020F8BD10B50400020093
:1005D0008034206800280FD0C17B20320907090F22
:1005E00001290AD0022908D0032905D15078C00971
:1005F00002D12000FFF7ACFF10BD51780A07FBD4F1
:100600008906F9D4FFF71CFF0020206010BD70B5EB
:1006100014001D0000290AD0012809D0022801D0A9
:10062000042804D10A00290020000CF3A0EC70BDBE
:100630001022290020000CF39AEC1035200008222B
:10064000290010300CF392EC290008310822200018
:100650001830EAE7FFB591B00B200E008001119928
:100660001A9F0818109040690C90002014001D007B
:10067000002B0B9004D0E8790007000F2030E871C0
:10068000002C04D0E0790007000F2030E071002F2B
:1006900004D0F8790007000F2030F8712100F37AB8
:1006A0000C310F9129000C310E91210030004031A6
:1006B0000E300D910CF376EE05047E7EF37E7D0008
:1006C0000700002C75D0002DFCD0B07A042870D221
:1006D000707B317B000208434007A07A02D50121DC
:1006E000084301E040084000A072E079F17A000977
:1006F00009070001090F0843E07178783978000292
:10070000084320810320A0710D98B27A0121407A1C
:10071000914008430D990D224872B07AB91C03012B
:10072000181A00190C300A90801C0CF320EC787811
:100730003978000208430D28E07A04D108210843E3
:100740000121E07203E0F72108400021E0720A98DD
:1007500041700A98B17A0170707B317B00020843C6
:10076000000702D50D98B17A0172A07AC0071FD098
:1007700011980121C068022208431043119AD060E9
:10078000A87AC20702D0EA79120711D10843A872E9
:10079000E8793F2200090001E8710320A871787808
:1007A00039780002084328810F990E980CF348EC21
:1007B0001EE2F3E1002D0A9072D0707B317B0002C3
:1007C000084381076CD54007A87A02D50121084368
:1007D00001E040084000A872E879F17A00090907B1
:1007E0000001090F0843E8710A98417A027A080269
:1007F000104328810320A871B17A5020415501216E
:10080000E972A87AC00754D011980321C64FA02BD3
:1008100001000000FC020100000400000E903B7A81
:10082000C06808431199C860002001E03C950200AF
:10083000431E2886EB62119913225201891888837E
:1008400011990922920189188B630100119B4A00BA
:10085000D21815235B010020D2181083431E119A71
:10086000880080180522D2018018491C042983625F
:10087000ECDB00206863012028871198407A022869
:1008800043D1119814F06AFE0990119814F08DFE6E
:1008900009992031497889060DD510994969803127
:1008A0000979C90707D080308068002803D001216A
:1008B00002E0E5E01BE00021119801F05CFDA87A60
:1008C000FD210840A87210984069FF306130407ED9
:1008D000002801D001200B900A980A9B417A007AE7
:1008E00009020143F07A0E9A0A33FFF79AFE002CB0
:1008F00069D0707B317B00020843C10763D0400799
:10090000A07A06D50121084305E0A87A0221084310
:10091000D8E740084000A072E079F17A00090907A1
:100920000001090F0843E0710A98417A027A08022F
:10093000104320810320A0710D99B07A0874E07AE9
:1009400002210843E072A07AC0072AD0707B317B75
:1009500000020843800614D50A9920000A78203046
:100960000274497841740A990422891C0C300CF3F2
:1009700008EB208E002804D1E06A002801D1401E37
:10098000E062707B317B00020843C00603D5002083
:1009900060630120208711980321C06808431199E2
:1009A000C8600C9880300079C00701D101200B90FD
:1009B0000A980A9B417A007A09020143F07A0F9A59
:1009C0000A33FFF72EFE002F7DD0707B317B0002B3
:1009D0000843410577D54007B87A02D5012108437D
:1009E00001E040084000B872F879F17A000909077F
:1009F0000001090F0843F8710A98417A027A080247
:100A0000104338810320B871B17A5020C155F87A6B
:100A100040210843F872B87AC00724D0707B317B3C
:100A200000020843800614D50A9938000A7820305D
:100A30000274497841740A990422891C0C300CF321
:100A4000A0EA388E002804D1F86A002801D1401E9F
:100A5000F862707B317B00020843C00603D500209A
:100A60007863012038870A980A9B417A007A090244
:100A700001433A00F07A0A330C32FFF7D2FDBDE0B1
:100A80000021099005A80A91FFA78ECF8EC00021F2
:100A90000A000B000F0001A88EC0707B317B0002A2
:100AA0000843810700D50A95C00700D00A940A9828
:100AB00000287DD00A98807AC00712D00A98006D6D
:100AC000002807D100E096E0FFF7ACFC0A99002867
:100AD000086506D00A980A99006D542208300CF374
:100AE000BAEA11990124497A2000022900D0002095
:100AF000717B327B0902114389071FD5002809D079
:100B000011981021C0686B4608431199C860187D80
:100B1000401C18750A980521C17211990A98FF3175
:100B200006224A310CF32CEA1198119AC06802216E
:100B300020430843D0600A9820304173707B317B9A
:100B400000020843C0070BD00A981221C1720A980C
:100B500006210CF3B2EA0A982030447301200B906E
:100B60000A98F17AC079090700090001090F0843C2
:100B70000A99C8710A98032181710998417C027C05
:100B800008020A99104308810999102201A810F05F
:100B9000FDFF00280DD10A9810222E3005A90CF374
:100BA000F0E90A9810223E3005A90CF3EAE90CE0BE
:100BB00035E00A98099910222E30FEF2C1FD0A98FC
:100BC000099910223E30FEF2BBFD0A98B17A0173FA
:100BD00009990A98102212311D300CF3D2E90999B3
:100BE0000A98102222310D300CF3CAE90A980A99AA
:100BF000807A204388720B98002803D01198002136
:100C0000FDF7EAFAFCF71BFD002D05D0A87AC00716
:100C100002D0119817F0C6E8002015B087A2F6227E
:100C200001000000F8060100000400005D4AE8161B
:100C3000F0BD0120FBE7F7B582B0002702983E0027
:100C4000019714F095FC0299029B0922497A9201BE
:100C50009C1802292AD1050020304078C10903D10F
:100C6000010701D480064AD52F0080373868002854
:100C700004D1FFF7E1FB002838600ED03F686762BF
:100C80000298083701F09EFB00280AD0FFF7D4FB3A
:100C9000852189000028485103D10020C04305B0B8
:100CA000F0BDFF35FF35AD1C686923E003290ED187
:100CB000A06A002803D1FFF7BFFBA06207E0616ACA
:100CC000002907D00831083054220CF3CEE9606ABD
:100CD000002804D1FFF7B0FB0028606201D0676AEA
:100CE0000837029801F06EFB002801D1206B02E06A
:100CF000FFF7A2FB2063002801D008300190E06AD2
:100D0000002804D1FFF798FB0028E06201D0E66AD2
:100D10000836019A00920499029833003A00FFF7CE
:100D2000ADFCBCE770B505000C000026081D09F0FD
:100D3000DAFF002815D1201D09F0C6FF002810D1C8
:100D40005920C00029180622201D10F029FF002874
:100D500007D0201D14F08CFC050001D1012070BDCE
:100D60000126220031002800FFF765FF70BDFFB5A6
:100D700089B004001F00129E002E77D0002CFCD0FA
:100D80002000403008902338079010380690401E0D
:100D9000059010300490083003903801C01B0019F2
:100DA000029020003E30FF29019004D1E079000933
:100DB0000228E2D0E8E00229FCD1FF209D3030700B
:100DC000000A70700A20B0700020F0700B990622A3
:100DD000301D0CF3E0E8E0790007000FF072E07AD4
:100DE000410602D50121890204E0800701D50121D5
:100DF00000E002213173090A7173E07903071B0FC8
:100E00003000190010300CF3E2EA050432323232BD
:100E10003100042F2AD2B7720899097AB94208D151
:100E2000717B327B09021143082211433173090A95
:100E300071730299497B002901D1052100E00D2140
:100E4000B173090AF173F17BB37B0A0202991A4369
:100E50000E310CF3A0E8F078B2780102F07B114378
:100E6000B27B000210430818801C35E02EE13500EB
:100E70003035032948D1217BB172202107008173CD
:100E80000020F87330000E300199102200900CF30E
:100E900082E8102230000799203007E0365C365C8B
:100EA000365C365C365C365C365C365C0CF372E87D
:100EB0000699102228000CF36EE801990098102280
:100EC000FEF248FCF078B17800020843F97BBA7B67
:100ED0000902114340181230B070000AF070A07A75
:100EE000C00708D0707B317B00020843042108430F
:100EF0003073000A7073F078B17800020843001D67
:100F00000004000C0DB0F0BD08990A7CB272228971
:100F1000B275120AF275228E21001378B3735278DB
:100F2000F27304222C310CF336E80021317571750F
:100F3000E07901073000090F1830012911D1202173
:100F4000B1750021F175059910220CF324E83000E9
:100F50000499082228300CF31EE80822039928007F
:100F600005E02189B175090AF175228905990CF30B
:100F700012E8F078B2780102F07D1143B27D0002F0
:100F8000104308180A30A7E7E079351D0007000F65
:100F90003071000A7071FF20401C3070000A00227E
:100FA0007070B270F270E07A410602D501208002C2
:100FB00004E0800701D5012000E00220A870000AAB
:100FC000E870E07901071ED1A81D042F7ED2218987
:100FD0002971090A69710899097AB94202D1012176
:100FE000417000E042700770029922890E31801C26
:100FF0000BF3D0EFF178B07809020143891CB1708E
:10100000090AF17041E00007000F012813D12020E8
:1010100028710020687105991022A81D0BF3BAEF02
:1010200028000499082216300BF3B4EFA6C5F5B7D3
:1010300001000000F40A010000040000A9259DA29F
:101040000822280003991E300AE0022801D0042853
:1010500009D1102028710020687105991022A81D5F
:101060000BF3A2EF1BE0032853D120892871000A5B
:101070006871207BA8710120E871AF1D07991022CB
:10108000B81C0BF392EF38000699102212300BF3C4
:101090008CEF3800019910222230FEF265FBA07A15
:1010A000C00708D0E878A978000208430421084363
:1010B000A870000AE870F178B278080269791043E4
:1010C0002A79090211434018801D020AB070001DE0
:1010D0000504F270E0792D0C000718D0741900E0B7
:1010E00017E0FF2121312170090A61700621A170EA
:1010F0000021E1700B990622201D0BF356EFE178D9
:10110000A278080210432D1D401905042D0C28005B
:1011100002E7002000E7FFB581B0002501980A9E94
:10112000C079000718D1042B16D3019F0024403743
:101130000120797AA04001420AD0230601A8009636
:1011400007C81B0EFFF71DFE3618281805042D0CC6
:10115000641C042CECDB05E001A8009607C8FFF72F
:1011600010FE05002800A4E5FFB583B000240500AB
:101170001E00C0680D9F40051DD5287A01281AD091
:10118000022818D1280014F0FDF90599002912D180
:10119000002810D08030006800280CD0F1073FD024
:1011A0005921C9006A180499083000230097FFF7F5
:1011B000E8FD040034E02800FF304A3002900920A6
:1011C0008001B1072D1800290BDAE86A002808D041
:1011D0000C9B029A049908300097FFF79CFF3F1878
:1011E0000400F0070DD0686A00280AD00C9B029A10
:1011F000049908300097FFF78EFF3F182018040469
:10120000240C70050CD5286B002809D00C9B029A81
:10121000049908300097FFF77EFF20180404240C7F
:10122000200007B0F0BDFFB587B0FF2100261F00EA
:10123000089CD04B35003000062C059607D20200E2
:10124000079801970091FFF78FFF06007BE01400DD
:1012500071E0C8480490FF2003900020029060785D
:10126000217800020843C11FF9390FD10399019772
:101270000091E179A0790B020343029A07980021BB
:10128000FFF772FF05003F18301844E00100FF39F6
:101290009D3942D107980690E078A1780002084372
:1012A000062829D3201D09F028FD002814D1201D6F
:1012B00009F014FD00280FD107985921C9004118E1
:1012C0000622201D10F076FC002805D0201D14F009
:1012D000D9F9069001200290E178A2780802104323
:1012E0000A2809D3A07A0390627B237BA1481102CC
:1012F000194300D0080004900698002809D00399EB
:1013000001970091049B029A06980221FFF72CFF97
:1013100005007F1970190604360CE078A1780002E8
:10132000084305998300091D41180904090C181880
:1013300004191434059108990598884203D219209C
:101340008001864285D330000BB0F0BD70B5060039
:1013500004680834E07903071B0F934201D0012091
:1013600070BD000712D1042910D22500403501229A
:10137000687A8A40904368720801401A00190C305C
:101380000F210BF3D8EE687A002804D13068FFF7FC
:1013900075F800203060002070BDFFB581B00400FA
:1013A00000201D000A9F0090E068002640050028EC
:1013B00027DA207A012824D0022801D0032820D15E
:1013C000200014F0DFF8217A032902D1617A022982
:1013D00017D1002F15D1002813D0803007000068E6
:1013E00000280ED0E90752D0C17B0A070399120FDB
:1013F0008A4202D00399FF2949D1FFF73FF83E60A6
:1014000045E00921029889016718FF281BD15A4835
:10141000854218D1F86A002802D0FFF72FF8FE6243
:10142000786A002808D0FFF729F87E62B86A002899
:1014300002D0FFF723F8BE62386B0028CE469C44EA
:1014400001000000F00E010000040000FAFF4ECE83
:1014500027D0FFF71DF83E6323E0F86A002808D084
:10146000A80706D59B208000039A02992018FFF751
:1014700077FF786A002808D0E80706D09920800016
:10148000039A02992018FFF76BFF386B002808D0E9
:10149000680506D527200001039A02992018FFF756
:1014A0005FFF00980FE4F7B586B0002707983E006D
:1014B000062864D314005EE0FF200490039000200F
:1014C00002906078217800020843304DC11FF9393D
:1014D00001D1012643E00100FF399D393FD1069833
:1014E0000590E078A1780002084306282BD3201D40
:1014F00009F00DFC002814D1201D09F0F9FB00288B
:101500000FD106985921C90041180622201D10F05C
:101510005BFB002805D0201D14F0BEF805900120CB
:101520000290E178A278080210430A280BD3A07A2F
:101530000490E07A0390617B207B0D020543124802
:10154000054000D1114D0598002808D0029A00925C
:10155000039A049905982B00FFF729FF0643E078CA
:10156000A178000208433F1DC11983000F04181819
:101570003F0C04191434079887429DD300E00126DC
:10158000300009B0F0BD000003040000FFFF0000C0
:1015900070B50C0010F0F4FD0500002C15D02000F3
:1015A00013F0FAFF002810D00D21890140180279AC
:1015B0000021012A0AD0022A04D10171C160200051
:1015C00000F06BF8280010F0DFFD70BD0171F9E745
:1015D0003EB5FF220400062101A810F022EB0022F4
:1015E000009220000E2301AA01A9F5F76FF910F06F
:1015F000C7FD0500E17AA07A14F005F807E02000A5
:1016000016F0F2EBE27AA17A2000FBF7F8F804007A
:10161000F5D1280010F0B8FD3EBDF1B582B00298BA
:1016200013F0BAFF0D21890105004418A0680028B5
:1016300028D010F0A5FD01902079352701263F0123
:10164000002820D001281AD10220E66020712069EC
:10165000FAF2ABFD00220092164A17480299EB19E4
:10166000FAF240FD019810F08FFD0298272116F044
:10167000C0EBE06801040298090C00F00EF8019834
:1016800010F082FDFEBD002200920A4A0A4802992B
:10169000EB19FAF227FD2671F1E713B5040013F0F8
:1016A0007BFF064B20001C684C21022301AAA047A7
:1016B0001CBD00000087930331100100A8BA02008E
:1016C000FFB585B004001D008F480E9F0460002008
:1016D00011F016FC8D4901200860E0784021084394
:1016E000E070280026002030017E20363170407ED8
:1016F0002900707004223431301D0BF360EC00209F
:10170000B070F07820214009400108438006800E27
:10171000B9010843F07010F033FD060060880490B2
:10172000218820000022283001AB07C32B00009045
:10173000079A04990C332000FEF215F92088103026
:101740002080300010F020FD288F401C0004000C89
:10175000288702D1686B401C686309B0F0BDF8B5FA
:10176000018943690C18E56EE66DE8790007000F02
:1017700002280ED1B0792900C207D20F180011F04B
:101780008CFC009022682B0000213000FFF798FFAE
:1017900007E0032805D122682B000021300016F055
:1017A0002CEB0020F8BDF7B58CB015000C984669FD
:1017B0000D9840300BF344ED0400408808AB0990CD
:1017C00018790007800F02280AD10C980C9980889C
:1017D000270010380004000C24378880603803E0AC
:1017E00020882700203710380A90F878800652D5D4
:1017F0000A9800284FDD3000FCF7A0FA00284DD0F1
:101800000D98434A20300B90007E41072000490F7D
:101810000C300CF33BFB3F49096888423ED308ABD0
:10182000187907AA0007800F08A910D14F20C0001F
:101830003018029201910090E879390002079F2048
:1018400080003318120F0120FFF2D6F91E2D6E2BE7
:1018500001000000EC12010000040000453A6B7D1D
:1018600016E028002C300592021D04910390E879BF
:1018700001070B98090F007E02924007400F01916B
:101880000090A0783A00030901213000EFF720FA18
:1018900000280DD0002E08D00520C00130180068A7
:1018A000002802D0416D491C416500200FB0F0BDF9
:1018B0001E4E0C98306030000D99442208300BF316
:1018C00088EB002011F026FB194901200860194817
:1018D000002205600A9803920104090C3A000832BC
:1018E00002912B0001970092326C09990C33200071
:1018F000FEF212F80120D9E710B5D37904001B07D6
:1019000000201B0F022B03D12068FFF756FF10BDEC
:10191000032BFCD1206816F07EEA10BD44040004BD
:101920003C040004FC800200DCBA020050440004C5
:101930004004000448040004F7B582B00E0010F023
:1019400029FC0024370020370190182060433949D2
:101950000A5C002A45D045187978687809098842D8
:101960003FD1281D0622B11D10F038F9002838D1CA
:10197000182161432F482E00081800210173FA78BE
:10198000BB780A36120230881A4301270D35120936
:101990003F03904219D104980069002802D02878AA
:1019A000042812D3378029700298407A02281BD16C
:1019B0000298F5F744FC002807D002980022FF3077
:1019C0004130018A029816F086E93088B8420BD07F
:1019D0002878022808D221060298090EF2F7F1F9B8
:1019E00002E0641C042CB0D3019810F0D7FB05B0C2
:1019F000F0BD10B58B7801241B09052B09D006DD3D
:101A00000B2B0DD00C2B02D1110016F008EA200090
:101A100010BD017A0229FAD116F004EA0024F6E793
:101A200020314A790B7911021943F0D016F0FEE902
:101A3000EDE700009C800200634800787047FF21BA
:101A40006248393110B50BF360EB5F490020087034
:101A500010BDFEB50020009010F09CFB0025029008
:101A6000012001905948E9004458002C41D02089B8
:101A70000619606900280DD00B21890141184969B8
:101A8000002720310F72017A032903D1FAF72BFFC7
:101A900080308762F06D80780007800F022802D1C5
:101AA0002000FCF78BFC300060300700407A3028C3
:101AB00002D1200009F046F8787A212801D10120CE
:101AC0000090F16D88780007800F07D16069427A35
:101AD000022A03D13200FFF78CFF019060690022D7
:101AE000310013F024F80198002802D020000BF3F5
:101AF000CDFF6D1C272DB3D3FFF7A1FF0098002861
:101B000001D001F043F8029810F048FBFEBDFEB58D
:101B100010F040FB009011F0D3F92B4C002811D1AC
:101B20002B480169406981420CD0009810F036FBC7
:101B3000A0680722401CA06026480121006811F01F
:101B4000D5F9FEBD01A810F032FB019BE0682178B9
:101B5000181A002920D00A281ED300221B4F10007B
:101B6000E36012E0C5007E59002E0BD0ED196D68C0
:101B7000FF265D1B491E4B36B54203D965886D1C97
:101B8000521C6580401C272801D20029EADC002A6B
:101B900002D01020EFF706FF009810F0FFFAFEBD0C
:101BA000030010B5094C00200100CA00A258002A09
:101BB00003D052699A4200D10120491C272901D241
:101BC0000028F2D010BD00006C7D0200C85900044E
:101BD00000A00080687D020030B50022AA4CE378A6
:101BE000002B0AD007E0A5182D79854202D10120EB
:101BF0000A7030BD521C9342F5D8002030BD10B59C
:101C0000A14C0020E3780B2109E0221812798A42C6
